:100000000C94BC020C9401030C9401030C940103A6
:100010000C9401030C9401030C9401030C94010350
:100020000C9401030C9401030C9401030C94010340
:100030000C9401030C94CA560C9401030C94010314
:100040000C9401030C9401030C9401030C94010320
:100050000C9401030C9401030C9401030C94010310
:100060000C9401030C94475B0C94B25B0C94010359
:100070000C9401030C9401030C9401030C940103F0
:100080000C9401030C9401030C9401030C940103E0
:100090000C9401030C9401030C9401030C940103D0
:1000A0000C9401030C9401030C9401030C940103C0
:1000B0000C9401030C9401030C9401030C940103B0
:1000C0000C9401030C9401030C940103C913CB138A
:1000D0000413CE13D913DC13DF13E213EB13EE1367
:1000E000D42695269B26A4268F26C826B026CE2663
:1000F000A026C026A0265C285C285C285E285E28F6
:10010000602867286728672867286728802F082DB8
:10011000162D752D2A2BDE2E312E102F3E2F982EC8
:100120009B2F802F9960A260A660AA60AE60C2601B
:10013000CB60CF60D3600A612F6135613B61416163
:10014000476154616761876194615D614F624F628D
:100150004F624F62DB61DF61E361FC610062166246
:100160004F621A62216225622C62306237623B6202
:1001700044626D6187617A6187614F624F624F624D
:100180004F62A061AD61B561D3610C9447610C947D
:10019000CB600C94CE130C94D11F0C943D3B0C946B
:1001A00094610C946E5A0C94F4190C94982E0C943F
:1001B000233C0C941B1E0C9405570C9421620C9448
:1001C00074600C94275A0C94DA590C94AB310C944B
:1001D0002B550C9467610C94E3610C94E0400C94F3
:1001E00000620C943B610C944F620C942D3B0C9478
:1001F000983B0C9495260C94195A0C94AC5F0C9473
:100200002F610C9404130C943B620C9437620C9491
:1002100087610C94AE5A0C947A610C94DF130C94A1
:100220009B2F0C94575A0C94D9130C94A0260C9421
:100230000A610C94A2570C94EE130C942E5C0C944F
:100240000E3C0C94102F0C942C620C94C9130C943B
:10025000802F0C94FD560C94D3610C94C8260C94FA
:10026000925E0C9430620C94D0570C9445300C94F0
:1002700067280C94DC130C94AA600C94F4570C942B
:1002800015580C948F260C949A5F0C94B0260C94FD
:10029000CD5A0C94A9400C94CB130C945E280C946A
:1002A00054610C94C0260C94AD610C94A6600C941F
:1002B000A9490C94E2130C94FC610C945C280C94F6
:1002C00095570C945D610C943A590C94CB230C9483
:1002D000B3580C94C6580C94A4260C94C0590C9492
:1002E000A2600C941A510C942E550C94A35F0C949C
:1002F0001A620C94EB130C94752D0C94DF610C9422
:10030000715B0C9400600C94FE5A0C9499600C94F0
:10031000DC5B0C94CF600C94AE600C942A2B0C9494
:1003200031550C9425620C9403030C94C2600C9418
:1003300016620C9435610C94B5610C94162D0C94D6
:10034000201A0C94A0610C94082D0C946D610C94EF
:10035000D3600C9463580C94D0490C94CA3B0C9411
:100360000C4E0C94CE260C9461620C947B4D0C9434
:100370003E2F0C94DB1C0C940D080C94F6030C948B
:10038000312E0C9444620C94D4260C94121C0C94C0
:10039000303B0C942E570C9460280C9441610C94C3
:1003A00071620C94B25E0C94DE2E0C949B260C941D
:1003B000DB610C948556696E6465782E68746D6C8B
:1003C000003C68746D6C3E0A3C686561643E3C2F7D
:1003D000686561643E0A3C626F64793E0A3C68313C
:1003E0003E576F726B733C2F68313E0A3C2F626F31
:1003F00064793E0A3C2F68746D6C3E0A3C48544D4B
:100400004C3E3C484541443E3C5449544C453E25B5
:10041000642025733C2F5449544C453E3C2F48459D
:1004200041443E3C424F44593E25642025733C2FB5
:10043000424F44593E3C2F48544D4C3E0D0A005704
:1004400057572D41757468656E7469636174653AB8
:10045000204261736963207265616C6D3D22257372
:10046000220D0A00636C6F73650D0A0D0A00436F5D
:100470006E6E656374696F6E3A2000436F6E7465CB
:100480006E742D4C656E6774683A20256C640D0A95
:1004900000436F6E74656E742D547970653A202533
:1004A000730D0A00485454502F25642E25642025CE
:1004B000642025730D0A5365727665723A2045747F
:1004C0006865726E75742025730D0A00FFFFFFFFCB
:1004D000FFFFFFFFFFFFFF3EFFFFFF3F34353637D3
:1004E00038393A3B3C3DFFFFFFFFFFFFFF000102B1
:1004F000030405060708090A0B0C0D0E0F10111254
:1005000013141516171819FFFFFFFFFFFF1A1B1C06
:100510001D1E1F202122232425262728292A2B2C93
:100520002D2E2F30313233FFFFFFFFFF4E41004EA3
:1005300041004E41004E41003031323334353637C0
:100540003839414243444546303132333435363709
:100550003839616263646566303030303030303055
:10056000303030303030303020202020202020200B
:10057000202020202020202084E880937400112453
:100580001FBECFEFD1E2DEBFCDBF00E00CBF18E051
:10059000A0E0B2E0ECEFFBEC00E00BBF02C0079084
:1005A0000D92AA38B107D9F729E0AAE8B8E001C04E
:1005B0001D92A43CB207E1F78FEF9FE79EBF8DBF6E
:1005C0008FEF9FE7845C99408138914050F04FEF66
:1005D0005EE7445C594064EC79E081EA99E00E946E
:1005E000854C0E94C85220E831E040E050E066EFC0
:1005F00073E088E895E00E9474550E9400000C9416
:10060000FC650C940000CF93DF9300D01F92CDB710
:10061000DEB780E092ECA1E0B0E089839A83AB83FF
:10062000BC8340E060E070E084E593E00E949C526F
:100630004091A6025091A70264E574E086E593E03C
:100640000E94FF3E8091A6029091A7020E94C73EA1
:10065000AE014F5F5F4F61E071E00E94593C0E9424
:10066000B04B9F938F9386E594E09F938F930E9466
:10067000FD3F81E894E09F938F9386E894E09F93F9
:100680008F930E94FD3F40E060E070E082E093E0E5
:100690000E949C520FB6F894DEBF0FBECDBF892BCF
:1006A00029F086E994E00E941140FFCF20E63AEE5F
:1006B00040E050E060E070E081E894E00E944E0E7F
:1006C000892B29F08FEB94E00E941140FFCF6091BD
:1006D0007709709178098091790990917A090E943F
:1006E00028219F938F938FEE94E09F938F930E9486
:1006F000FD3F89EF94E09F938F930E94FD3F40E080
:1007000060E070E08FE792E00E949C520F900F90A3
:100710000F900F900F900F90892B29F086E195E0B4
:100720000E941140FFCF8EE195E00E9411408DE3C1
:10073000E82E85E0F82E9AE4C92E95E0D92E2BE517
:10074000A22E25E0B22E32E2832E35E0932E0E94B7
:10075000FB1A8C01892BA9F48091A0098F938091B9
:100760009F098F939F928F920E94FD3F68EE73E0E6
:1007700080E090E00E9487500F900F900F900F90B4
:10078000E6CFFF92EF920E94FD3F60E570E0C80166
:100790000E94671BDF92CF920E94FD3F67E575E0E4
:1007A000C8010E94033E3C010F900F900F900F90E4
:1007B000009779F48091A0098F9380919F098F937E
:1007C000BF92AF920E94FD3F0F900F900F900F903D
:1007D00005C00E947F12C3010E94C43DC8010E944F
:1007E0001D1E86E795E00E941140B1CF0E94B14ED8
:1007F00020E033E040E050E063E073E083E895E020
:100800000E9474558EEF0E94D54D0E94854D0E9426
:100810009C4DE0918B08F0918C08309709F0199568
:1008200090910A029F3F89F383B723B7217F922BD0
:1008300093BF93B7916093BF889593B79E7F93BF03
:1008400093B7917F8E70892B83BFDFCF062E692FE0
:10085000902D072E782F802D0895CF93DF93EC01F4
:10086000892B69F089A59AA50E9401468BA59CA5B4
:100870000E940146CE01DF91CF910C940146DF9199
:10088000CF910895CF92DF92EF92FF920F931F9333
:10089000CF93DF931F921F92CDB7DEB77C016A0121
:1008A000FC018081918169837A830E940146C6019F
:1008B00001960E94F3458C01F70191838083698141
:1008C0007A81009751F0C114D10419F0A6010E9459
:1008D0001E65F601E00FF11F10820F900F90DF915F
:1008E000CF911F910F91FF90EF90DF90CF900895DF
:1008F0004F925F926F927F928F929F92AF92BF9230
:10090000CF92DF92EF92FF920F931F93CF93DF93DB
:100910008C017B018DE290E00E94F345EC01892B74
:1009200009F40BC18DE2DE011D928A95E9F780EC96
:1009300098EAA0E0B0E08DA39EA3AFA3B8A7F8010A
:1009400080899189A289B38989839A83AB83BC8387
:1009500000511F4FF0EFEF1AF1085E018BE2A80E75
:10096000B11C4E01A9E28A0E911CD8012C912F3F97
:1009700009F4DAC01E141F040CF0DCC0211106C0FB
:100980000F5F1F4FB1E0EB1AF108EFCFF801318193
:10099000C32ED12CEC14FD040CF4CCC0253331F45F
:1009A000313009F0C7C082818883B6C02C3031F461
:1009B000A601B8016E5F7F4FC40107C02F3041F41C
:1009C000A601B8016E5F7F4FC5010E944204A4C01A
:1009D000343008F4A1C0D801E28113966C91862FBF
:1009E00090E0A0E0B0E04427582F692F7A2FD8017B
:1009F00014968C9190E0A0E0B0E0DC019927882764
:100A0000840F951FA61FB71F8E0F911DA11DB11D2D
:100A1000F801458150E060E070E0742F66275527AB
:100A200044272A013B01480E591E6A1E7B1EC30142
:100A3000B201213029F44D825E826F8278866CC0CB
:100A40002C3129F449865A866B867C8665C0233012
:100A500029F44D865E866F86788A5EC02630D9F589
:100A6000498A5A8A6B8A7C8A383008F455C0D80182
:100A700016968C91169717964C91179750E060E058
:100A800070E0762F652F542F44272A013B01480E32
:100A9000511C611C711C18968C9190E0A0E0B0E094
:100AA000DC0199278827AC01BD01440D551D661D49
:100AB000771DF801818590E0A0E0B0E0B82FAA276B
:100AC00099278827840F951FA61FB71F8D8B9E8B94
:100AD000AF8BB88F21C0263329F4498E5A8E6B8E86
:100AE0007C8E1AC02A3339F40E9426046D8F7E8FC3
:100AF0008F8F98A311C02B3339F40E94260469A369
:100B00007AA38BA39CA308C0233331F40E9426044C
:100B10006DA37EA38FA398A7F2E0CF0ED11C0C0D7E
:100B20001D1DEC18FD0821CF8881823049F08550C9
:100B3000823030F0CE010E942D0480E090E03CC075
:100B40008D8D9E8DAF8DB8A1892B8A2B8B2B61F457
:100B50008DA19EA1AFA1B8A5B695A79597958795AC
:100B60008D8F9E8FAF8FB8A389A19AA1ABA1BCA195
:100B7000892B8A2B8B2BF9F48D8D9E8DAF8DB8A18F
:100B80008C019D013695279517950795AC01BD0100
:100B9000E2E07695679557954795EA95D1F7400F2E
:100BA000511F621F731F840F951FA61FB71F89A3B4
:100BB0009AA3ABA3BCA3CE01DF91CF911F910F915C
:100BC000FF90EF90DF90CF90BF90AF909F908F906D
:100BD0007F906F905F904F900895EF92FF920F93E8
:100BE0001F93F901E00FF11FE451FF4FAFEFA08316
:100BF0007801EDEEEE0EF11CECE2EE16E1E0FE0601
:100C000020F4ECE2EE2EFF24F394890123E430E09B
:100C10000E948C1E97FF09C083E190E090939A0890
:100C2000809399088FEF9FEF02C080E090E01F91C2
:100C30000F91FF90EF9008952F923F924F925F9205
:100C40006F927F928F929F92AF92BF92CF92DF92DC
:100C5000EF92FF920F931F93CF93DF93CDB7DEB741
:100C600060970FB6F894DEBF0FBECDBF9C878B8711
:100C70002A013B011901470158010E94E6506F8388
:100C8000788789879A8767017801A50194012A5F8F
:100C90003109410951092D873E874F87588B04E25E
:100CA00012E09101AE014B5F5F4FBE016F5F7F4F5E
:100CB0008B859C850E94D81E181619064CF000974B
:100CC000B9F124E130E030939A082093990830C0BC
:100CD000823F91057CF0D1012C91223059F4149679
:100CE0004D915D916D917C91179744155505660561
:100CF0007705F1F00E94E650DC01CB012F813885A9
:100D000049855A85821B930BA40BB50B2D853E8517
:100D10004F85588982179307A407B50738F47501E2
:100D20006401C81AD90AEA0AFB0AB9CF80E090E048
:100D300060960FB6F894DEBF0FBECDBFDF91CF91A6
:100D40001F910F91FF90EF90DF90CF90BF90AF90E9
:100D50009F908F907F906F905F904F903F902F90DB
:100D60000895EF92FF921F93CF93DF9300D01F92CD
:100D7000CDB7DEB7162F29833A834B835C830E945D
:100D800080527C0129813A814B815C81009729F056
:100D9000DC011B968C91833049F081E190E09093C7
:100DA0009A08809399088FEF9FEF46C0D7011F964E
:100DB000ED91FC915097309781F38081863069F7EF
:100DC00029833A834B835C830E94E65060938D08AD
:100DD00070938E0880938F089093900829813A81B0
:100DE0004B815C8120939108309392084093930843
:100DF0005093940810939B0880919C0890919D08B3
:100E0000892B69F420E231E0A7016DE078E08DE8FC
:100E100095E00E94745590939D0880939C0887E903
:100E200098E00E94D45140E050E0BA0185E998E092
:100E30000E94605180E090E00F900F900F900F9013
:100E4000DF91CF911F91FF90EF900895CF92DF92A5
:100E5000EF92FF920F931F93CF93DF93EC0184E205
:100E600092E0DE01FC011D923197E9F781E0888371
:100E7000898396E09A83E1E7F9E0DE015C960190D0
:100E80000D929A95E1F72C833D834E835F830C2C62
:100E9000CD2CD02CD986C886EC86FD860E871F8780
:100EA000FE01E451FF4F93E69083319622E82083C0
:100EB000319623E5208331969083319695E3908394
:100EC00031968083CE50DF4F688387E090E0DF91DA
:100ED000CF911F910F91FF90EF90DF90CF900895E9
:100EE0002F923F924F925F926F927F928F929F923A
:100EF000AF92BF92CF92DF92EF92FF920F931F9328
:100F0000CF93DF93CDB7DEB73C011A012B01490126
:100F1000A80197018601750154018CEEA80EB11C41
:100F2000CE8CDF8C63E0C4010E9426072E893F89A6
:100F3000488D598D232B242B252B81F0F501E80FAB
:100F4000F91F22E3208324E021832E893F89488DE5
:100F5000598D228333834483558306962A8D3B8D96
:100F60004C8D5D8D232B242B252B81F0F501E80F73
:100F7000F91F26E3208324E021832A8D3B8D4C8DAD
:100F80005D8D22833383448355830696F501E80FF4
:100F9000F91F27E3208323E0218331E03283238379
:100FA00026E024838C010B5F1F4FE2EBF9E00190F8
:100FB0000020E9F7AF01435B594014161506A4F46D
:100FC000F501E00FF11F8CE0808341837A01FF245B
:100FD000A70162EB79E0CF0102960E941E65A7018E
:100FE0004E5F5F4F040F151F9401B201A101C301B1
:100FF0000E94ED05DF91CF911F910F91FF90EF902F
:10100000DF90CF90BF90AF909F908F907F906F9028
:101010005F904F903F902F900895CF93DF93CDB77F
:10102000DEB7A0970FB6F894DEBF0FBECDBF8C0120
:101030000E94DD506A8F7B8F8C8F9D8F2091770966
:10104000309178094091790950917A092E8B3F8B24
:10105000488F598FD8011F960D90BC91A02DBF8F3E
:10106000AE8FFD013B96CD0107961F82188619862B
:101070001A86EF80F88409851A85702F6F2D5E2DF2
:10108000442722917A018B01E20EF11C011D111DF2
:10109000EF82F88609871A87E817F90751F700EAFF
:1010A0001FE020E030E00B831C832D833E831B86F2
:1010B0001A8A1B8A1C8A1D8A198A188A212C312CAB
:1010C000812C912C0E94DD506B017C011B8511232A
:1010D00009F12B813C814D815E81220F331F441F1A
:1010E000551F2B833C834D835E8321303A4F41054E
:1010F000510540F000E01AEF20E030E00B831C8344
:101100002D833E832FEF3FEFA9012C873D874E872C
:101110005F8749C080919B08833059F08F81988503
:10112000A985BA850196A11DB11D8F839887A987CE
:10113000BA87E0919E08F0919F083097A9F0018D41
:10114000128D238D348D0C871D872E873F87012BB1
:10115000022B032BC9F020EA3FE040E050E02B8354
:101160003C834D835E831FC08FEF9FEFDC018C8734
:101170009D87AE87BF8700EA1FE020E030E00B8349
:101180001C832D833E830FC02FEF3FEFA9012C87D7
:101190003D874E875F8780EA9FE0A0E0B0E08B83C9
:1011A0009C83AD83BE8380919B08882309F444C04F
:1011B000853009F441C08091910890919208A091E6
:1011C0009308B0919408892B8A2B8B2BA9F10E944C
:1011D000E65000918D0810918E0820918F08309173
:1011E0009008AB01BC01401B510B620B730B80914B
:1011F000910890919208A0919308B0919408481793
:1012000059076A077B0738F0A1E0B0E0B0939A086D
:10121000A09399087BC0841B950BA60BB70B0B8181
:101220001C812D813E8180179107A207B30720F40E
:101230008B839C83AD83BE8380919B08823021F099
:101240009AEF980F9230D0F4BB85BB2349F1B701D8
:10125000A6010A8D1B8D2C8D3D8D401B510B620B01
:10126000730B411551056140710508F000C59601E9
:101270004A8D5B8D241B350B398B288B853011F003
:10128000811114C08114910419F0C4010E945D1FE2
:10129000C1010E940146212C312C812C912C49C086
:1012A000CA8EDB8EEC8EFD8E198A188A80919E087C
:1012B00090919F08892B51F4EE8DFF8D8385948545
:1012C000A585B685892B8A2B8B2B01F5811491047A
:1012D00021F02114310469F508C084E490E00E94F3
:1012E0002B1E4C0121143104A1F484E292E00E94EF
:1012F000F3451C018114910411F0892B61F492E1F2
:10130000E92EF12CF0929A08E092990810929B082D
:10131000D9CE892BA1F300EC16E01A83098322E0D1
:1013200030E0AE014F5F5F4F62E070E1C4010E94A8
:101330009C1F80919B08813021F52F81388549853C
:101340005A852F5F3F4F4F4F5F4F2F833887498715
:101350005A8780917B0990917C09A0917D09B09179
:101360007E09EE88FF88088D198D8E219F21A0238C
:10137000B123892B8A2B8B2B11F482E068C284E085
:1013800066C2823009F011C17B8473940B850430EE
:1013900038F021E030E030939A082093990814C483
:1013A00021013CEE430E511CC888D988E12CF12C58
:1013B00087012F81388549855A8561E0C1010E94E6
:1013C0002607EE88FF88088D198DE114F1040105C8
:1013D000110561F0F201E80FF91F22E3208324E0F8
:1013E0002183E282F382048315830696F201E80FDB
:1013F000F91F27E3208323E02183FF24F394F28263
:10140000238326E024838C010B5F1F4FE2EBF9E07E
:1014100001900020E9F7AF01435B5940141615060F
:10142000A4F4F201E00FF11F8CE0808341837A0184
:10143000FF24A70162EB79E0CF0102960E941E65AE
:10144000A7014E5F5F4F040F151FF201E00FF11F60
:1014500089E3808382E0818380E492E0082E892FF3
:10146000902D938382830C5F1F4F91014FEF5FEFAD
:10147000BA01C4010E94ED0597FDA6C3EB80FC8074
:101480000D811E8191014F81588569857A85C4013E
:101490000E941C06181619060CF07BC000919E08CD
:1014A00010919F08BC01C1010E9478047C01009743
:1014B00009F450C0DC018C91823009F046C001155E
:1014C000110509F446C08091770990917809A0919F
:1014D0007909B0917A0940917B0950917C0960911A
:1014E0007D0970917E09482359236A237B23452B6C
:1014F000462B472BA9F0F801418152816381748109
:1015000084179507A607B70729F1F7014181528192
:101510006381748184179507A607B707D9F411C0B2
:10152000D70195964D915D916D917C919897F801B9
:1015300085A196A1A7A1B0A584179507A607B7070F
:1015400020F4C8010E942D0404C0C7010E942D048C
:1015500001C0870110939F0800939E08012B09F496
:101560008DCF8091910890919208A0919308B091AD
:101570009408803E9E42A105B10570F010EAE12E6C
:101580001FE0F12E00E010E0EB82FC820D831E8351
:1015900075CF892B09F018C380919E0890919F0800
:1015A000892B09F462C383E052C1833029F57B841F
:1015B00073940B85043020F011E010939B0855C301
:1015C000E0919E08F0919F0829892F9338893F93D5
:1015D000848D8F93838D8F93828D8F93818D8F9345
:1015E00084818F9383818F9382818F9381818F9365
:1015F000A12CB12C6501BBC1843009F069C07B848A
:10160000739403E0071540F411E010939B081E8AC1
:101610001F8A188E198E29C329892F9338893F93E1
:101620001F921F921F921F92498D4F93588D5F9367
:101630008F898F939E899F93A12CB12C6501EF8098
:10164000F88409851A8591014FEF5FEFBA01C40153
:101650000E9470070FB6F894DEBF0FBECDBF97FD96
:10166000B3C2EB80FC800D811E8191014F815885B2
:1016700069857A85C4010E941C0697FDA5C2009762
:1016800009F4F3C2BC01C1010E9478048C010097E7
:1016900009F4EBC2FC018081853071F480919E08D1
:1016A00090919F080E942D0410939F0800939E081C
:1016B00085E080939B0898C1863009F0CEC2FF2454
:1016C000F394F0929B081E8A1F8A188E198EC5C249
:1016D000853009F045C0109291081092920810923E
:1016E00093081092940885E998E00E946D52E09169
:1016F0009E08F0919F08458D568D678D70A1D7018A
:10170000C6010A891B892C893D89801B910BA20B7C
:10171000B30B84179507A607B70710F086E097C0AC
:101720008A899B89AC89BD89840F951FA61FB71F25
:101730009C01AD012C193D094E095F09283319E8B8
:10174000310711E44107510520F027E339E841E46E
:1017500050E0A8EEB3E00E945E63AB01BC0175C22D
:10176000863009F09FC000919E0810919F08D80113
:1017700091962D913D914D915C9194972C873D8749
:101780004E875F874A885B886C887D88420E531E2F
:10179000641E751E4C185D086E087F086B817C8185
:1017A0008D819E8128EE33E040E050E00E94F76298
:1017B000421653066406750650F4A8EEB3E0A30182
:1017C00092010E945E636B837C838D839E832A8952
:1017D0003B894C895D89C21AD30AE40AF50A8C85D3
:1017E0009D85AE85BF85C816D906EA06FB0670F54D
:1017F000D8011196AC9011971296BC90129713963F
:10180000CC9013971496DC90149759964D915D9156
:101810006D917C915C97B989BF93E889EF931F9292
:101820001F921F921F92DF92CF92BF92AF92EF80D2
:10183000F88409851A859101C4010E9470070FB6CA
:10184000F894DEBF0FBECDBF97FF04C087E0809342
:101850009B08FFC17B847394EB80FC800D811E810B
:1018600091014F81588569857A85C4010E941C06C3
:1018700097FDAAC1009709F4F8C1BC01C1010E94FB
:1018800078048C01009709F4F0C1DC012C9125301B
:1018900009F49CC0263009F0E0C187E080939B08E2
:1018A000712CDBC1873009F0B0C000919E08109107
:1018B0009F08D80195962D913D914D915C919897F7
:1018C0002C873D874E875F874A885B886C887D8838
:1018D000420E531E641E751E4C185D086E087F086C
:1018E0006B817C818D819E8128EE33E040E050E069
:1018F0000E94F762421653066406750650F4A8EE7D
:10190000B3E0A30192010E945E636B837C838D83AD
:101910009E832A893B894C895D89C21AD30AE40ACD
:10192000F50A8C859D85AE85BF85C816D906EA0661
:10193000FB0618F010929B088CC17B847394D8012D
:101940001196AC9011971296BC9012971396CC906A
:1019500013971496DC90B989BF93E889EF931F928F
:101960001F921F921F92DF92CF92BF92AF92EF8091
:10197000F88409851A8591014FEF5FEFBA01C40120
:101980000E9470070FB6F894DEBF0FBECDBF97FD63
:101990001BC1EB80FC800D811E8191014F81588518
:1019A00069857A85C4010E941C0697FD0DC10097C8
:1019B00009F45BC1BC01C1010E9478048C0100974D
:1019C00009F453C1DC012C912530B9F480919E08B3
:1019D00090919F0828A30E942D0410939F080093C4
:1019E0009E0828A120939B08EA8CFB8C0C8D1D8DF2
:1019F000EA8AFB8A0C8B1D8B38C1263009F02DC179
:101A0000FF24F394F0929B0828C1883009F08FC01E
:101A10007B8473940B85043008F0D6C021011CEE42
:101A2000410E511CAE8DBF8D1B96ED90FD900D911A
:101A30001C911E97C12CD12C2F81388549855A8540
:101A400068E0C1010E942607F201E80FF91F27E3B1
:101A5000208323E02183B1E0B283238326E0248323
:101A60008C010B5F1F4FE2EBF9E001900020E9F7DA
:101A7000AF01435B5940A1F0F201E00FF11F8CE090
:101A8000808341837A01FF24A70162EB79E0CF01D3
:101A900002960E941E65A7014E5F5F4F040F151F3F
:101AA000F201E00FF11F89E3808382E0818380E40B
:101AB00092E0082E892F902D938382830C5F1F4F15
:101AC00091014C855D856E857F85C4010E94ED0581
:101AD00097FD70C0EB80FC800D811E8191014F81CC
:101AE000588569857A85C4010E941C061816190656
:101AF000ACF4BC01C1010E9478048C01009771F024
:101B0000DC018C91853061F480919E0890919F0852
:101B10000E942D0410939F0800939E0800E010E09F
:101B200010929B080115110509F097C09EC08930DD
:101B300009F070C0E0919E08F0919F083097C9F1BC
:101B4000BB85BB2319F07B2E739434C0418C528C1F
:101B5000638C748CE180F28003811481C12CD12CC0
:101B60002F81388549855A8567E0C1010E94260783
:101B7000411451046104710471F0F101E451FF4F0B
:101B8000E80FF91F26E3208324E021834282538259
:101B90006482758206968C0191014C855D856E8507
:101BA0007F85C4010E94ED0597FF11C077247394CF
:101BB00001C07B84EC84FD840E851F85E122E02238
:101BC000EF20E09409F051C010929B084EC0EB80CA
:101BD000FC800D811E8191014F81588569857A8530
:101BE000C4010E941C0697FF03C010929B0839C0D5
:101BF0000097B9F1BC01C1010E9478048C010097E3
:101C000081F1DC018C91853011F0863021F5109244
:101C10009B0821C0811128C080919E0890919F0847
:101C20000E942D0410929F0810929E081092910815
:101C300010929208109293081092940885E998E007
:101C40000E946D5240E050E0BA0187E998E00E949E
:101C50006051712C0AC077247394C8010E942D042E
:101C600004C07724739401C07B847B862BCAAFEFBA
:101C7000BFEFB98BA88B02CB20919B08253029F4AC
:101C80009A01AB0169E00C94B10683E090E0909377
:101C90009A08809399088FEF9FEF08956F927F9233
:101CA0008F929F92AF92BF92CF92DF92EF92FF926C
:101CB0000F931F93CF93DF9300D01F92CDB7DEB762
:101CC0003C014B0129833A834B835C830E94805201
:101CD0005C0129813A814B815C81009769F0FC01AC
:101CE0008385833049F4078510890115110521F09A
:101CF000F8018081863019F081E190E04DC08114B7
:101D00009104B1F0F401908181818923928189232A
:101D10009381892394818923958189238F3F41F081
:101D200086E0A1E7B9E001900D928A95E1F718C02D
:101D3000F80195818681892B9781892B9085892B44
:101D40009185892B9285892B59F4C30129833A8384
:101D50004B835C830E9488235C814B813A8129817B
:101D6000A0917109F0917209E09173097091740961
:101D700060917509909176098A2F8F2B8E2B872B76
:101D8000862B892B39F0FA23EF237E2367239623B2
:101D90009F3F39F482E090E090939A0880939908ED
:101DA000C9C086E0E1E7F9E0D801159601900D92EF
:101DB0008A95E1F764EF71E080E090E029833A834F
:101DC0004B835C830E948750F80113861486158626
:101DD0001686C0907B09D0907C09E0907D09F09038
:101DE0007E09C38AD48AE58AF68A80918309909114
:101DF0008409A0918509B09186098C219D21AE218D
:101E0000BF2129813A814B815C81892B8A2B8B2BC5
:101E100071F140EE5EE260E070E0C3010E943C0EB2
:101E20002091830930918409409185095091860958
:101E300020937709309378094093790950937A0970
:101E4000A0907F09B0908009C0908109D09082094C
:101E5000E0907B09F0907C0900917D0910917E094A
:101E600061E779E0C3010E9492224C0166C061E003
:101E7000C3010E94B1064C01892B09F05BC080911F
:101E80009B08853031F5E0919E08F0919F08C5844C
:101E9000D684E784F08805811681278130854181C9
:101EA000528163817481C5010E948121E0919E0865
:101EB000F0919F08E588F6880789108D218932897D
:101EC0004389548960E070E080E090E00E94B10FA7
:101ED00034C0F80183859485A585B685892B8A2B26
:101EE0008B2B59F520917709309178094091790928
:101EF00050917A09E0907B09F0907C0900917D096E
:101F000010917E09DA01C9018E219F21A023B123FE
:101F1000892B8A2B8B2B71F0A0907F09B0908009C0
:101F2000C0908109D090820961E779E0C3010E94E5
:101F3000922203C088248A94982CC4010F900F9099
:101F40000F900F90DF91CF911F910F91FF90EF9025
:101F5000DF90CF90BF90AF909F908F907F906F90C9
:101F600008954F925F926F927F928F929F92AF925D
:101F7000BF92CF92DF92EF92FF920F931F93CF9376
:101F8000DF936C01EB0129013A014701580180916F
:101F9000550990915609009731F00E940146109220
:101FA0005609109255098091570990915809009748
:101FB00031F00E9401461092580910925709C1143D
:101FC000D10439F0C6010E940646909356098093C9
:101FD0005509209739F0CE010E9406469093580982
:101FE000809357094092590950925A0960925B09AF
:101FF00070925C0980925D0990925E09A0925F09DF
:10200000B0926009DF91CF911F910F91FF90EF90F7
:10201000DF90CF90BF90AF909F908F907F906F9008
:102020005F904F900895FC01CF012191222369F028
:10203000203211F02930C1F7FC011192CF0121911A
:102040002032E1F32930D1F308950895EF92FF9201
:102050000F931F93CF93DF937C01009729F1FC012D
:1020600001900020E9F731978F01081B190BE1F06F
:10207000CBE0D2E0688179816115710591F0FB01B7
:1020800001900020E9F73197E61BF70BC8018E1B82
:102090009F0B8E0D9F1D0E942E65892B41F0269669
:1020A000E9CF8BE092E004C081E192E001C0CE0173
:1020B000DF91CF911F910F91FF90EF9008950F93B3
:1020C0001F93CF93DF9300D01F92CDB7DEB7182FA9
:1020D000092F61157105C1F07F936F9381E994E039
:1020E0009F938F930F931F9329833A834B835C8332
:1020F0000E9437400F900F900F900F900F900F900D
:102100005C814B813A81298157FD11C05F934F93C8
:102110003F932F938BE794E09F938F930F931F939D
:102120000E9437400FB6F894DEBF0FBECDBF612FBF
:10213000702F8EE694E00E944740612F702F84E656
:1021400094E00F900F900F900F90DF91CF911F911F
:102150000F910C9447400F931F93CF93DF93CDB70C
:10216000DEB728970FB6F894DEBF0FBECDBF182F8D
:10217000092F2F8338874D835E830E94B04B9F9336
:102180008F9338853F932F812F935E815F934D818D
:102190004F931F9281E08F931F928F9384EA94E074
:1021A0009F938F930F931F930E9437408091A008B5
:1021B0000FB6F894DEBF0FBECDBF80FF1EC080E01B
:1021C00090E00E94CF4369837A838B839C83CE0106
:1021D00001960E940C420E9411189F938F9383E9ED
:1021E00095E09F938F930F931F930E94C93F0F9089
:1021F0000F900F900F900F900F9028960FB6F894B5
:10220000DEBF0FBECDBFDF91CF911F910F9108951B
:10221000AF92BF92CF92DF92EF92FF920F931F93F4
:10222000CF93DF93F82EE92E6B01EA01413981E06B
:102230005807C9F054F44033E1E05E0701F140393A
:102240005140D1F40FEA15E01CC0443F81E058072B
:1022500069F0453F91E0590761F04439514061F41C
:1022600008EC15E00EC00BEB15E00BC002ED15E01D
:1022700008C001EE15E005C00BED15E002C002EA52
:1022800015E09801AE01B6018F2D9E2D0E94AB1076
:10229000C139F1E0DF0741F5F601A084B1846FE2B6
:1022A00070E0C5010E948D656C01009719F0FC017A
:1022B000108204C085E5A82E85E0B82EBF92AF92AB
:1022C0008FE394E09F938F93EF92FF920E943740A9
:1022D0000F900F900F900F900F900F90C114D1049A
:1022E00019F08FE2F60180832FEF3FEFA90161EF34
:1022F00075E08F2D9E2D0E945F101F930F93DF932B
:10230000CF931F930F93DF93CF938CEF93E09F9323
:102310008F93EF92FF920E943740EDB7FEB73C9645
:102320000FB6F894FEBF0FBEEDBFDF91CF911F91A6
:102330000F91FF90EF90DF90CF90BF90AF900895F6
:102340000E942610FC018281938108950E9426102C
:10235000FC01848195810895DF92EF92FF920F93A3
:102360001F93CF93DF9300D0CDB7DEB78C011B82D4
:102370007C0180E2D82EF8018081882309F18B321C
:1023800019F4F701D08216C0853291F4F8018181E9
:10239000898382818A8340E150E060E070E0CE0171
:1023A00001960E947163F70160830E5F1F4F02C0A8
:1023B000F70180830F5F1F4FFFEFEF1AFF0ADBCF9C
:1023C000F70110820F900F900F90DF91CF911F9126
:1023D0000F91FF90EF90DF900895EF92FF920F938F
:1023E0001F93CF93DF93EC01EA84FB84E114F104A3
:1023F00009F47EC081E090E09F8B8E8B8701F7010E
:102400008191882341F08632D9F78E899F89019680
:102410009F8B8E8BF5CF8E899F89880F991F880F90
:10242000991F0E94F3459D8B8C8B009719F41F8A8E
:102430001E8A5EC0FC01F182E0821382128222E0D9
:1024400030E0F80181918F018823C1F08632C9F70D
:10245000C901880F991FEC89FD89E80FF91F1183C5
:1024600000834C895D89FA01E80FF91F13821282FB
:10247000F801319710822E5F3F4FE3CF00E010E06C
:10248000E12CF12C8E899F89E816F9068CF58C8950
:102490009D89FC01E00FF11F0190F081E02DDF012B
:1024A00021912223B9F02D33D1F798012E5F3F4FB0
:1024B000FC01E20FF31FAD014F5F5F4F518340837B
:1024C0001C928C899D89FC01E20FF31F8081918110
:1024D0000E94AC11EC89FD89E00FF11F8081918190
:1024E0000E94AC11FFEFEF1AFF0A0C5F1F4FCACF1B
:1024F000DF91CF911F910F91FF90EF9008952F9250
:102500003F924F925F926F927F928F929F92AF9283
:10251000BF92CF92DF92EF92FF920F931F93CF93D0
:10252000DF93CDB7DEB76F970FB6F894DEBF0FBE5F
:10253000CDBF4C011B8A1A8A212C312CC1010E946B
:102540002C1664E270E081E090E00E94D7451C0107
:10255000009709F4CEC2EBE0F0E0DC011396FC93A7
:10256000EE9312972A893B892115310519F0C9018B
:102570000E94014680E091E00E94F3459B8B8A8B8C
:10258000009709F4B6C2A40160E071E00E94993F8F
:10259000892B09F4AEC26DE070E08A899B890E94A4
:1025A0004C65009711F0DC011C926AE070E08A89AA
:1025B0009B890E944C65009711F0FC01108280E01D
:1025C00091E00E94F3457C01892B09F492C29101AC
:1025D0002E5E3F4F3D8B2C8B265F3F4F3F8B2E8BCC
:1025E0002E5F3F4F398F288F205131093B8F2A8F23
:1025F000225031093D8F2C8F2C5F3F4F3F8F2E8F04
:10260000310132E2630E711CC4010E94673F8C01EC
:102610008D309105C9F30A97E1F4C7010E94014684
:102620008A899B890E9413108C010E9413107C01DF
:102630000E9413106BEF75E08A899B890E942E65BA
:10264000892B09F0CEC081E090E0F1019183808375
:10265000E4C0A12CB12C512C4A2C0F3F8FEF18074E
:1026600021F4C7010E94014644C20A30110509F451
:1026700054C00A33110519F5852D90E0FC01EE0FC9
:10268000FF1F8E0F9F1FFC01E651FC4F80818A11B6
:1026900044C04EC0C8010E94DA64D6011196ED9183
:1026A000FC911297EA0DFB1D2081022E000C330BCA
:1026B0002817390799F05394BAE05B1679F0C52CC6
:1026C000D12CC601880F991F8C0D9D1DDC01A651D0
:1026D000BC4F6D018C91481670F7DCCFC4010E948D
:1026E000673F8C010D97D1F3E0E1AE16B10431F0F4
:1026F000FFEFAF1ABF0A2AE05212AECF0F3F3FEFF3
:10270000130709F4AECF0115110509F486CF0A337A
:10271000110519F48AE058120BC0C4010E94673FEA
:102720008F3FAFEF9A0709F46FCF0A97B1F76CCFDD
:10273000A40160E071E0C7010E94993F892B09F470
:1027400090CF6AE070E0C7010E944C65009759F491
:10275000C4010E94673F8F3FBFEF9B0709F454CF2E
:102760000A97B1F751CFFC011082E816F90620F460
:1027700082918D3009F41082852D90E08A30910588
:1027800008F042CFFC018827EA59FF4F8F4F0C9485
:1027900038638301D1C10E8D1F8DCEC1C7010E9448
:1027A0009F64D10114966D937D938D939C9317979D
:1027B0002BCF0C8D1D8DC0C10A8D1B8DBDC1088D09
:1027C000198DBAC1C7010E948917F101608F718FFD
:1027D000828F938F19CF0E891F89AEC10C891D89F5
:1027E000ABC16FEF75E08A899B890E942E65892BAA
:1027F00019F4E3E0F0E00AC064E076E08A899B899E
:102800000E942E65892B31F4E2E0F0E0D101ED93D6
:10281000FC9303C045EF51E006C0D8018C918111B3
:1028200007C040E951E0B101C4010E94081161C133
:10283000F70180818823A9F369E076E0C7010E944F
:102840002E65892B39F48AE090E0D10113969C9390
:102850008E93129781E090E0F10191A380A36FE342
:1028600070E0C8010E944C65009771F0DC011D9278
:10287000CD010E940646F10193878287892B09F4D6
:1028800038C1C1010E94ED11C8010E940646D10164
:1028900019969C938E931897009709F42AC10E9469
:1028A0009519892B19F440E951E044C0C1010E94F7
:1028B0008318892B19F041E951E03CC0B101C401F2
:1028C0000E942919892B09F00BC10BE612E0A12CFB
:1028D000B12CEE24EA94FE2CD8016D917D918D01EE
:1028E0006115710509F1F101808591850E94CB1573
:1028F0005C01009719F444EF51E01CC060E070E8FF
:102900000E947F3C7C018F3FFFEF9F0749F00E94B0
:10291000853E672B682B692B91F4C7010E94263CEA
:10292000C5010E940146D8CFBFEFEB16FB0639F474
:1029300044E951E0B101C4010E940811D1C0C501B0
:102940000E94A0118C01C5010E94A6116C01892B67
:1029500009F046C08091A00881FF42C0BE016F5FB0
:102960007F4FC5010E94E03A892B49F48A859B85F7
:10297000AC85BD858E879F87A88BB98B08C082E107
:1029800096E00E9489176E877F87888B998BF1016B
:10299000808D918DA28DB38D0097A105B105B1F009
:1029A0004A855B856C857D8584179507A607B707E3
:1029B0006CF0C7010E94263C40E351E0B101C40124
:1029C0000E940811C5010E9401468AC0CE010E96E0
:1029D0000E940C420E9411180E9406463C0102C04F
:1029E000612C712CC5010E9401462BE236E048ECB7
:1029F00050E0B101C4010E94AB106114710499F060
:102A00007F926F92AEE2B6E0BF93AF939F928F92A8
:102A10000E94C93FC3010E9401460F900F900F9082
:102A20000F900F900F90C7010E94853E2B013C0133
:102A3000C114D10491F02FEF3FEFA901B801C401F7
:102A40000E945F1020916109309162098101A20109
:102A5000B701C401F601199540C09B01AC01B80152
:102A6000C4010E945F10D1018D919C910397A9F13F
:102A700080E092E00E94F3456C01892B71F1A12C5A
:102A800082E0B82E411451046104710481F04114B4
:102A9000B2E05B06610471040CF45201A501B601B9
:102AA000C7010E949D3D8C011816190624F0C6012D
:102AB0000E94014612C09401AC0161E070E0C601C1
:102AC0000E94D93F892B99F3012E000C220B330B66
:102AD000401A510A620A730AD5CFC7010E94263CE8
:102AE000C4010E94713EF10180A191A1019709F0FA
:102AF00025CDC1010E942C162A893B89211531055B
:102B000089F1C9016F960FB6F894DEBF0FBECDBF35
:102B1000DF91CF911F910F91FF90EF90DF90CF90B9
:102B2000BF90AF909F908F907F906F905F904F90ED
:102B30003F902F900C940146D8018D919C91892B48
:102B400009F062CDF701CF0121912032E1F3293064
:102B5000D1F30E940646D8018D939C93892B09F0EE
:102B600053CD7FCD6F960FB6F894DEBF0FBECDBFAD
:102B7000DF91CF911F910F91FF90EF90DF90CF9059
:102B8000BF90AF909F908F907F906F905F904F908D
:102B90003F902F900895AF92BF92CF92DF92EF9225
:102BA000FF920F931F93CF93DF935C017B01C09043
:102BB0006109D0906209C114D10421F48FE7C82EB5
:102BC00087E0D82EE50109900020E9F72197CA197E
:102BD000DB09D6010D900020E9F7F70101900020F4
:102BE000E9F73197EE19FF09CE018C199D098A0F7B
:102BF0009B1F8E0F9F1F0E94F3458C01009701F1D0
:102C0000B6010E946065B501C8010E944165F701E7
:102C100080818823A9F0209761F0CA0DDB1D2197E0
:102C200091E080E028812F3209F090E0692F782F21
:102C300002C061E070E06E0D7F1DC8010E94416519
:102C4000C801DF91CF911F910F91FF90EF90DF901E
:102C5000CF90BF90AF900895CF93DF93EC01892B75
:102C600009F441C088859985009711F00E940146BA
:102C70008A859B85009711F00E9401468C859D8571
:102C8000009711F00E9401468E859F85009711F0F4
:102C90000E94014688899989009711F00E94014697
:102CA0008A899B89009711F00E9401468C899D8931
:102CB000009711F00E9401468C8D9D8D009711F0B8
:102CC0000E9401468E8D9F8D009711F00E94014653
:102CD0008AA19BA1009711F00E940146CE01DF91CD
:102CE000CF910C940146DF91CF910895FC01CF0163
:102CF00021912032E1F32930D1F30895CF93DF936E
:102D0000FB01118210826AE0DC012C9130E020533B
:102D100031092A303105A8F420813181629FA00158
:102D2000639F500D11245183408301962C91022EF4
:102D3000000C330B20533109240F351F31832083BE
:102D4000E3CFDF91CF910895CF93DF93EB010E9402
:102D50007E1628813981263431051CF42C593F4FC9
:102D600006C02D3647E0340724F02C56374039830F
:102D70002883DF91CF9108950F931F93CF93DF9313
:102D8000FC01DB018081813489F49F012F5F3F4F7B
:102D900081818F7D803519F483E090E002C087E067
:102DA00090E08D939C93F901EF0149C0843419F4AC
:102DB0008BE090E039C0863419F481E090E034C0B3
:102DC0008A34C1F4CF0101962181322F3F7D313405
:102DD00019F41D921C921DC0222349F0CF010296C6
:102DE00022812F7D2C3419F426E030E010C025E03C
:102DF00030E00DC08D34A1F48181813661F4CF01C2
:102E0000029622812F7D223541F422E030E02D937D
:102E10003C93FC01C9CFCF01019624E030E0F7CF0D
:102E20008E3429F48AE090E08D939C93BDCF8F344B
:102E300019F489E090E0F8CF88E090E0F5CF8E01BA
:102E40002196F801808190E00E94C964892BB9F72E
:102E5000C801DF91CF911F910F910895CF92DF921A
:102E6000EF92FF920F931F93CF93DF937A01890123
:102E70000E947E16EC01DC2ECD2E8991811107C0B7
:102E8000B7018D2D9C2D0E94BC16FC010CC090E05A
:102E90000E94C964892B79F3F3CF30E020533109C4
:102EA0002A30310520F0CF0121912111F6CFB80150
:102EB000DF91CF911F910F91FF90EF90DF90CF9016
:102EC0000C94A4160F931F93CF93DF93EA0189010B
:102ED0000E947E16FC0120812A33A1F4BE010196D6
:102EE0000E947E16FC0120812A3341F4B80101962C
:102EF000DF91CF911F910F910C947E16F8011182F2
:102F0000108202C019821882DF91CF911F910F9118
:102F10000895DF92EF92FF920F931F93CF93DF9369
:102F2000CDB7DEB762970FB6F894DEBF0FBECDBF48
:102F30009E012F5F3F4F790122E1F70111922A95FF
:102F4000E9F721E030E038872F830E9476168C0164
:102F5000FC01808190E00E94C964892B69F0F8012E
:102F6000CF012191322F3F7D21F40E9476168C01F2
:102F700003C02930A9F7F9CFF801D0808D2D90E05A
:102F80000E94C964892BA9F0BE01675F7F4FC80109
:102F90000E94BC160E947616BE01695F7F4F0E9498
:102FA0007E160E947616BE01655F7F4F0E94A416B2
:102FB0000EC0DD20C1F09E01255F3F4FAE01475F8F
:102FC0005F4FBE01695F7F4FC8010E942E170E94AC
:102FD00076169701AE014D5F5F4FBE016B5F7F4F6D
:102FE0000E9462178C01C8010E94761669EE77E094
:102FF0000E945765892B21F4C7010E94C74303C073
:10300000C7010E94CB4362960FB6F894DEBF0FBE95
:10301000CDBFDF91CF911F910F91FF90EF90DF9087
:103020000895FC0181818F9380818F9383818F9399
:1030300082818F9385818F9384818F9382859385FD
:103040008459984F9F938F93A085B185AA0FBB1F7A
:10305000A85FBB4F11968C9111978F938C918F9392
:1030600087818F9386818F930484F585E02DEE0F01
:10307000FF1FE05EFB4F81818F9380818F938DEEE8
:1030800097E09F938F9384EA98E09F938F930E9499
:1030900099408DB79EB742960FB6F8949EBF0FBE6B
:1030A0008DBF84EA98E00895EF92FF920F931F93EB
:1030B000CF93DF938C017B01C091C408D091C508E8
:1030C0002097C9F00115110541F06A817B81C80183
:1030D0000E9498650817190751F4E114F10459F09A
:1030E0006C817D81C7010E945765892B21F0099071
:1030F000D881C02DE5CFCE01DF91CF911F910F91E7
:10310000FF90EF900895CF92DF92EF92FF920F938E
:103110001F93CF93DF937C01FC01008511856FE243
:1031200070E0C8010E948D65EC01892B11F01882B6
:1031300002C005E515E060E070E0C8010E94541887
:10314000892B31F1F701C088D188C114D10419F15C
:1031500046E050E069E578E0C6010E947F65892B72
:10316000D1F4C60106960E949D3AF70160897189E3
:103170006A5F7F4FC8010E94541821E030E0892B1C
:1031800011F020E030E088279927821B930B05C0BF
:1031900080E090E002C08FEF9FEF209711F02FE2C8
:1031A0002883DF91CF911F910F91FF90EF90DF90D7
:1031B000CF900895CF92DF92EF92FF920F931F93DB
:1031C000CF93DF937C01EB016A018881998101979C
:1031D000029718F045EF51E01AC00091C80810910D
:1031E000C9080115110589F0688579856C0D7D1D6B
:1031F000D80112968D919C9113970E942E65892B70
:1032000091F0F80100811181ECCF44E951E0BE0159
:10321000C701DF91CF911F910F91FF90EF90DF9049
:10322000CF900C940811D8011496ED91FC9115974C
:10323000BE01C7011995892B19F044EF51E0E7CF82
:10324000DF91CF911F910F91FF90EF90DF90CF9082
:103250000895CF92DF92EF92FF920F931F93CF9337
:10326000DF936C017B01E091C608F091C7083097AD
:1032700069F4E0E6F8E00AC0DE018D010C1B1D0BCD
:103280008D91811110C00115110581F48081882371
:1032900011F1EF01FE019E012F5F3F4F88818B33BB
:1032A00059F7E901F7CF8B3341F7EDCFA801BE0104
:1032B000F701808591850E946765892B41F4A801FB
:1032C000B701C6010E94DA1881E090E006C0FE0155
:1032D000E00FF11FDBCF80E090E0DF91CF911F91F5
:1032E0000F91FF90EF90DF90CF90089590ED980FA1
:1032F0009A3028F4082E000C990BC09708959FE986
:10330000980F963030F4082E000C990B87559109D0
:1033100008959FEB980F963028F4082E000C990B17
:10332000C79708958FEF9FEF08958F929F92AF9266
:10333000BF92CF92DF92EF92FF920F931F93CF93A2
:10334000DF938C01FC01B080FFE2BF123EC06C0134
:10335000EC018FE2A82E7E019FEFE91AF90A89811C
:103360008823C1F08532D1F48A810E9476194C01FC
:1033700097FD14C08B810E94761997FD0FC07E01C6
:1033800023E0E20EF11CE0E18E9E800D11248B8380
:10339000811104C0F6011082C80119C0F7018081B3
:1033A0008C3509F4A082F701908182ED8B0D82307B
:1033B00020F482ED890F823030F0B92EF60190832F
:1033C000C60101966C01E701C6CF80E090E0DF9175
:1033D000CF911F910F91FF90EF90DF90CF90BF9012
:1033E000AF909F908F9008956B307105C9F06C304D
:1033F000710519F06A30710501F5FC01E65BFF4FBC
:10340000DC01A25BBF4F208131818D919C91B9017C
:10341000681B790BCB01092E000CAA0BBB0B05C056
:10342000FC0187859089A0E0B0E0FA018083918358
:10343000A283B38380E090E008958FEF9FEF08951B
:10344000CF92DF92EF92FF920F931F93CF93DF9370
:10345000EC018B017A016901AB0141705527B7017D
:103460008B5A9F4F0E94473DA801427055279601F5
:10347000B701CE01CE960E94473D8D898430D9F4A4
:10348000FE01E65BFF4F808191813496208131817E
:10349000821B930B31E020E0181619060CF030E087
:1034A000832F922F4F8558892B893C8942175307C8
:1034B00020F4826002C080E090E02D89222331F068
:1034C0002D89253019F02D892B3011F483E090E0FF
:1034D00080239123DF91CF911F910F91FF90EF9067
:1034E000DF90CF9008950F931F93CF93DF93EC015C
:1034F0008C010F5A1F4FF80180819181009749F08C
:10350000FC0120813181F801318320830E94105316
:10351000F2CF8AAD9BAD009741F0FC012081318153
:103520003BAF2AAF0E941053F4CFC95ADF4F8881B6
:103530009981009741F0FC012081318139832883F2
:103540000E941053F4CFDF91CF911F910F910895F6
:10355000CF93DF93EC010E94731A8F859889892B92
:1035600021F089899A890E940146CE01DF91CF918D
:103570000C9401468F929F92AF92BF92EF92FF926E
:10358000E090CA08F090CB08F7013097E9F0A28DDF
:10359000B38DA817B907A1F4848C958CA68CB78C31
:1035A00082169306A406B50659F4A0A1B1A1A617E8
:1035B000B70731F4A589AA2319F0A589AB3099F48E
:1035C0000280F381E02DE1CFF701309761F025898A
:1035D000213029F4228D338D8217930721F0028048
:1035E000F381E02DF2CFCF01FF90EF90BF90AF902D
:1035F0009F908F900895CF93DF938091CC08811195
:1036000010C06BEC73E286E00E940120892B09F068
:1036100059C00E941729892B09F054C081E080937A
:10362000CC0869E770E081E090E00E94D745EC01AA
:10363000892B09F447C01D8A84E08C838BE19EE1CD
:103640009E838D8382E19CE198878F838BED9CE143
:103650009A87898784EF99E19C878B8780E29AE13A
:103660009E878D870E94734F6BA37CA38DA39EA31F
:103670006FA378A789A79AA76BA77CA78DA79EA7FA
:10368000FE01E85BFF4F80E99CE0918380833496E4
:10369000918380833D9688E192E091838083369682
:1036A00028EE33E0318320832091CA083091CB0883
:1036B0003B832A839C8B8B8BD093CB08C093CA0807
:1036C000CE0102C080E090E0DF91CF910895062EF8
:1036D000672F702DFC01738F628F0C94D62F8F9201
:1036E0009F92AF92BF92CF92DF92EF92FF920F9391
:1036F0001F93CF93DF93EC017B018A010E94854DDC
:10370000209729F1E114F10419F480E090E051C010
:1037100001151105D1F36E0149E5C40ED11CF60166
:10372000808191818017910708F48C014E01F1E7A7
:103730008F0E911C5E014CE3A40EB11C8D89843068
:1037400049F0C959DF4F89E390E0998388838FEF6F
:103750009FEF2FC08BA59CA52FA138A5821B930B93
:10376000AC015695479556954795F60120813181D4
:103770004217530740F42FA938ADA901481B590B34
:103780004017510758F4F4014081518162817381DF
:10379000C5010E946051892B89F2B7CF8AA180614F
:1037A0008AA3A801B701CE010E940724892B79F6CC
:1037B000C801DF91CF911F910F91FF90EF90DF90A3
:1037C000CF90BF90AF909F908F900895CF92DF924F
:1037D000EF92FF920F931F93CF93DF937C016B01C6
:1037E0008A01C0E0D0E0C017D1077CF4A8014C1BCF
:1037F0005D0BB6016C0F7D1FC7010E946F1B181671
:1038000019062CF4C80FD91FEECFCE0102C08FEFDE
:103810009FEFDF91CF911F910F91FF90EF90DF907D
:10382000CF900895AF92BF92CF92DF92EF92FF9226
:103830000F931F93CF93DF93EC017B018A01892BB8
:1038400049F08D89843049F0C959DF4F89E390E010
:10385000998388838FEF9FEFA3C08F859889411547
:103860005105A9F4009709F497C069897A89AC01D8
:10387000CE010E94E61B29893A8997FF02C0C9013F
:1038800073C0C9010E940146188A1F8685C06B89D2
:103890007C89009749F546175707A8F0CA010E948E
:1038A000CF626C015801A81AB90AA501B701CE016F
:1038B0000E94E61B97FDCECFC114D10409F46FC05E
:1038C000EA0CFB1C01C06A018B899C890E94F345AC
:1038D0009A8B898B009709F4BDCFA601B7010E948E
:1038E0001E65D88ACF865BC0E989FA899C01240FBE
:1038F000351F2617370760F4B7018E0F9F1F0E94F0
:103900001E658F859889800F911F988B8F8747C080
:103910006B01C81AD90AA601B7018E0F9F1F0E941A
:103920001E65EC0CFD1C4B895C8969897A89CE0186
:103930000E94E61B97FD16C098012C193D096B8962
:103940007C8926173707C0F0C9010E94CF625C014D
:103950006901C81AD90AA601B701CE010E94E61B67
:1039600097FF07C089899A890E940146188A1F8695
:1039700071CFEC0CFD1C01C0590189899A89A114F1
:10398000B10429F0A501B7010E941E6502C00E9482
:103990000146B88AAF8603C080E090E001C0C8014C
:1039A000DF91CF911F910F91FF90EF90DF90CF901B
:1039B000BF90AF900895CF92DF92EF92FF920F9356
:1039C0001F93CF93DF937C016B018A014115510551
:1039D00069F0BA0181EA99E00E94B34BEC010097CB
:1039E00039F0A801B6010E94E26402C0C0E0D0E054
:1039F000A801BE01C7010E94121C8C01209729F06A
:103A0000BE0181EA99E00E941B4CC801DF91CF9171
:103A10001F910F91FF90EF90DF90CF9008952F921C
:103A20003F924F925F926F927F928F929F92AF924E
:103A3000BF92CF92DF92EF92FF920F931F93CF939B
:103A4000DF93CDB7DEB728970FB6F894DEBF0FBE71
:103A5000CDBF98878F831B018A010E94854D8F817E
:103A60009885009709F4CAC0FC018589843061F00B
:103A70008589853049F0EF81F885E959FF4F89E361
:103A800090E091838083BAC02114310419F480E05E
:103A900090E0B8C001151105D1F34F805884FAE4C5
:103AA0004F0E511C8F819885825B9F4F9E838D8323
:103AB000AF80B8849DE6A90EB11CCF80D884E3E521
:103AC000CE0ED11CF20180819181ED81FE81E080DA
:103AD000F1808E159F0581F4EF81F885858984300A
:103AE00051F6F5014081518162817381C6010E94C6
:103AF0006051892B39F3CBCF8E199F09801791071D
:103B00001CF4009721F28C01C12CD12C8F81988557
:103B10008F5A9F4F9A838983EF81F885E05BFF4F2F
:103B2000FC83EB83C016D106E0F5E981FA81608061
:103B30007180F301818892888E189F08C8018C19C2
:103B40009D0954018815990508F45C01F301678506
:103B500070896E0D7F1DA501C1018C0D9D1D0E94F8
:103B60001E65CA0CDB1CEA0CFB1CA814B904D0F2BD
:103B7000F30180819181E981FA8191838083F2014F
:103B8000808191818E199F0991838083C3010E9456
:103B90001053EB81FC81808181508083E12CF12CDA
:103BA000C1CFED81FE81F182E082EF81F8858589C8
:103BB000843039F5E85BFF4F40815181AF81B88592
:103BC000A45BBF4F2D913C91CA01800F911F281714
:103BD00039070CF4C901AF81B885A75ABF4F2D91A1
:103BE0003C91918380832417350758F028173907B3
:103BF00040F48F8198850E94772803C08FEF9FEF54
:103C000001C0C80128960FB6F894DEBF0FBECDBF25
:103C1000DF91CF911F910F91FF90EF90DF90CF90A8
:103C2000BF90AF909F908F907F906F905F904F90DC
:103C30003F902F9008950C940F1DCF93DF93EC01CC
:103C400040E050E060E070E00E94121CCE01DF9185
:103C5000CF910C944928CF93DF93EC018091CF084A
:103C600081110BC06BEA71E381E10E940120892B75
:103C700009F04DC081E08093CF08209771F50E9434
:103C8000E6502091D0083091D1082115310529F056
:103C90006E7077276160620F731F7093D108609315
:103CA000D008C091D008D091D108D06CD093D10861
:103CB000C093D008CE01082E892F902DE091630982
:103CC000F0916409309749F0228133812817390730
:103CD000B1F20190F081E02DF5CF64E170E081E078
:103CE00090E00E94D745FC01892B89F00C2ECD2F46
:103CF000D02DD383C283809163099091640991830D
:103D00008083F0936409E0936309CF0102C080E0EF
:103D100090E0DF91CF9108956F927F928F929F9262
:103D2000AF92BF92CF92DF92EF92FF920F931F93C9
:103D3000CF93DF936C014A015B013901FC0184855B
:103D40009585892B21F5A70160E880E090E00E942D
:103D50004D53EC01892B31F48CE090E0F60195870E
:103D6000848715C0A701B8018F8598890E941E65B8
:103D70008E019301B501A401C6010E94293200976A
:103D800041F4CE010E94105380E090E002C08FEF1A
:103D90009FEFDF91CF911F910F91FF90EF90DF90F8
:103DA000CF90BF90AF909F908F907F906F9008952D
:103DB0004F925F926F927F928F929F92AF92BF923B
:103DC000CF92DF92EF92FF920F931F93CF93DF93E7
:103DD000EC013B014A0159012801B701A6018C857C
:103DE0009D85892B19F08FEF9FEF56C08C819D81A7
:103DF000892B21F4CE0106960E9460518C859D8509
:103E0000892B89F7EC80FD80E114F10409F442C0AC
:103E1000D7018D919C9111979D838C831796ED917D
:103E2000FC91189784859585A685B785F3018083D5
:103E30009183A283B383D7011B96ED91FC911C97CC
:103E400080819181082E892F902DF40191838083A8
:103E500051968D919C915297982E192F481659067C
:103E600014F4942C152D28853985F901E81BF90BDC
:103E7000F987E887D7011F966D917C915097492D5E
:103E8000512FC5010E941E65C7010E941053892D44
:103E9000912F02C080E090E0DF91CF911F910F91B0
:103EA000FF90EF90DF90CF90BF90AF909F908F905A
:103EB0007F906F905F904F900895CF93DF93EC01C8
:103EC000E0916309F0916409A3E6B9E03097F1F05D
:103ED000EC17FD07B1F4888199818D939C938C81B7
:103EE0009D81009741F0FC01208131813D832C832D
:103EF0000E941053F4CFCE010E94014680E090E072
:103F000007C0DF010190F081E02DE0CF8FEF9FEF40
:103F1000DF91CF910895E0916309F09164093097A2
:103F200049F0228133812817390721F00190F0816F
:103F3000E02DF5CFCF010895009791F062307041E8
:103F400079F44115510561F02230310549F4FA0147
:103F500020813181FC013387228780E090E0089541
:103F60008FEF9FEF08950F931F93FC01892B89F02A
:103F700046875787608B718B338B228B158704871D
:103F800086819781892B41F0CF0106960E942352AA
:103F900003C08FEF9FEF02C080E090E01F910F9170
:103FA0000895CF92DF92FF920F931F93CF93DF93E9
:103FB0006C018B01DB011796ED91FC911897F18450
:103FC000C091D208D091D308209789F08A81F81641
:103FD00021F00990D881C02DF7CFEB81FC8130977B
:103FE000C1F3B801C6011995009799F702C08FEF88
:103FF0009FEFDF91CF911F910F91FF90DF90CF90B6
:104000000895EF92FF921F93CF93DF93182F7B01B8
:10401000C091D208D091D308FE01309739F0828147
:104020008117D1F00190F081E02DF7CF65E070E0CD
:1040300081E090E00E94D745FC01892BC9F01283F2
:10404000209779F4F093D308E093D20881ED9FE1B3
:1040500090938C0980938B09F482E38280E090E056
:1040600009C0D183C083F093D308E093D208F4CF82
:104070008FEF9FEFDF91CF911F91FF90EF90089509
:104080004F925F926F927F928F929F92AF92BF9268
:10409000CF92DF92EF92FF920F931F93CF93DF9314
:1040A00000D01F92CDB7DEB74B015C01270138016C
:1040B000E0906509F090660905E619E0E114F10465
:1040C00079F0F70186819781A085B1852817390796
:1040D0004A075B0728F48701D701ED90FC90EECFEB
:1040E00080E190E029833A834B835C830E94F3450F
:1040F000FC0129813A814B815C810097D1F08222B9
:104100009322A422B52282829382A482B58226833E
:104110003783408751874286538664867586D78663
:10412000C686F182E082D8018D939C9380E090E076
:1041300002C08FEF9FEF0F900F900F900F90DF91C5
:10414000CF911F910F91FF90EF90DF90CF90BF9094
:10415000AF909F908F907F906F905F904F90089559
:104160008F929F92AF92BF92CF92DF92EF92FF9287
:104170000F931F938B019C014115510531F0DA011A
:104180001D921D921D921C9213976091650970916A
:1041900066090F3FBFEF1B072B073B0781F0D901D3
:1041A000C801082E8B2FB02D092E9A2FA02D8827FD
:1041B0009927AA27B07F0097A105B04E21F4FB01F3
:1041C000309781F538C084E0FB013097A1F1C680BB
:1041D000D780E084F184C022D122E222F3228280BF
:1041E0009380A480B580C814D904EA04FB0421F0AC
:1041F0000190F081E02DE9CF4115510579F002855C
:10420000138524853585011511052105310531F00A
:10421000DA010D931D932D933C93139726853785D3
:10422000232B19F08685978508C002851385248580
:104230003585815049F680E090E01F910F91FF9005
:10424000EF90DF90CF90BF90AF909F908F900895A8
:10425000EF92FF920F931F93CF93DF93CDB7DEB70B
:1042600027970FB6F894DEBF0FBECDBF6C837D835A
:104270008E839F83FE0134968F010C5F1F4F46EEA5
:1042800058E08AE0E82E9EE2F92E808120E06E2D33
:104290000E94C36231E0320FA1E0B0E0AC0FBD1F5D
:1042A000A20FB11D905D9C93232F8111F0CF11922D
:1042B000BA01215060F081E090E08C0F9D1F820FC9
:1042C000911DDC018C91DB018D93BD01F2CFDA01F0
:1042D000A30FB11DAD014F5F5F4FFC92E017F107D7
:1042E000A1F61C9286EE98E027960FB6F894DEBFF2
:1042F0000FBECDBFDF91CF911F910F91FF90EF9037
:1043000008952F923F924F925F926F927F928F9279
:104310009F92AF92BF92CF92DF92EF92FF920F9354
:104320001F93CF93DF9300D000D0CDB7DEB71C0131
:104330002A013B0148015901C982DA82EB82FC82E1
:10434000DC011F960D90BC91A02DBE83AD83452B43
:10435000462B472B71F44090770950907809609074
:10436000790970907A09411451046104710409F4C7
:10437000BEC0ED81FE8143865486658676868114B3
:104380009104A104B10429F488248A94982CA82CBF
:10439000B12CAD81BE8153968D929D92AD92BC920F
:1043A00056976101E12CF12C8701A5019401C3010D
:1043B000B201682179218A219B210E9440208981B4
:1043C0009A81AB81BC810097A105B10551F07C01B8
:1043D0008D0120E030E0A90160E070E0CB010E9497
:1043E000402089E0F1013296A8E6B9E001900D92F3
:1043F0008A95E1F7AD81BE8115966C911597169659
:104400005C91169717964C91179718963C911897B0
:1044100019962C9119971A969C911A97862F852395
:1044200084238323822389238F3F79F0562B452BC6
:10443000342B232B922B49F086E0FD013596A1E722
:10444000B9E001900D928A95E1F740927709509278
:1044500078096092790970927A0980927B0990922A
:104460007C09A0927D09B0927E0989819A81AB81F5
:10447000BC81892B8A2B8B2BA1F480917F09909191
:104480008009A0918109B0918209482659266A269F
:104490007B2684209520A620B72089288A288B286F
:1044A00061F089819A81AB81BC8180937F0990936F
:1044B0008009A0938109B093820926960FB6F894DB
:1044C000DEBF0FBECDBFDF91CF911F910F91FF9047
:1044D000EF90DF90CF90BF90AF909F908F907F90A4
:1044E0006F905F904F903F902F900C94B5238FEF7B
:1044F0009FEF26960FB6F894DEBF0FBECDBFDF91BB
:10450000CF911F910F91FF90EF90DF90CF90BF90D0
:10451000AF909F908F907F906F905F904F903F9063
:104520002F9008954F925F926F927F928F929F92F9
:10453000AF92BF92CF92DF92EF92FF920F931F93B1
:10454000CF93DF93CDB7DEB72A970FB6F894DEBFCF
:104550000FBECDBF4B012F83388749875A8727016C
:104560003801760165010E9480529E838D830097F9
:1045700019F48FEF9FEFB5C0DC011B962C911B97B0
:104580002330B9F71F960D90BC91A02D2C912630A9
:10459000E9F5FC01258936892115310549F1AE017E
:1045A0004F5F5F4F64E070E1F90119958D819E8145
:1045B000DC015596ED91FC915697A40165E070E100
:1045C000199589819A81AB81BC81816089839A83A5
:1045D000AB83BC838D819E81DC015596ED91FC916E
:1045E0005697AE014F5F5F4F63E070E1199507C0CA
:1045F000159686E0F40101900D928A95E1F79301FA
:1046000082014F81588569857A8567C0273109F015
:10461000B0CFFC01A188B2888F819885A985BA8521
:10462000F50181A392A3A3A3B4A34114510461048F
:10463000710429F0342D252D962D872D04C03FEFD0
:104640002FEF9FEF8FEFD50199963C9399979A960C
:104650002C939A979B969C939B979C968C938114F2
:10466000910451F0F40180819181A281B381F5011F
:1046700085A396A3A7A3B0A7C5010E946D52AE0162
:104680004B5F5F4F67E171E0F501FF96808191819B
:104690000E94593C40E65AEE60E070E0C5010E947D
:1046A0006051892B09F065CFD501DC968C91DC97A0
:1046B000893009F05ECF9596CD90DD90ED90FC901D
:1046C000989799960D911D912D913C919C9791965B
:1046D0004D915D916D917C9194978D819E810E9409
:1046E00081212A960FB6F894DEBF0FBECDBFDF91B1
:1046F000CF911F910F91FF90EF90DF90CF90BF90DF
:10470000AF909F908F907F906F905F904F900895A3
:10471000CF93DF93EC0140E250E067E679E080E47C
:1047200090E00E942755892B59F4809167098032C7
:1047300039F4BE0188E699E00E945765009791F030
:1047400080E2E7E6F9E0DF011D928A95E9F786E06D
:10475000EEE2F4E0A1E7B9E001900D928A95E1F76D
:104760008FEF9FEFDF91CF91089580E280936709EB
:1047700040E250E067E679E080E490E00E9429554D
:1047800021E030E0892B11F420E030E088279927E0
:10479000821B930B0895FB01A385B485109751F1FB
:1047A000828183FF27C01C962C911C9722952F7025
:1047B000220F220F2431F0F030E085859685821794
:1047C0009307C4F0821B930B928B818B892B61F032
:1047D0001C968C911C9782958F7094E0899FA00DF8
:1047E000B11D1124B08BA78736872587CF010E9482
:1047F000AC2803C0CF010E94105380E090E00895E0
:10480000062E692F902D072E782F802D08956F92F8
:104810007F928F929F92AF92BF92CF92DF92EF9250
:10482000FF920F931F93CF93DF931F921F92CDB7E9
:10483000DEB76C017B013A01DC0192968C91452B2D
:1048400021F4982F9B7009F47DC181FF02C018E10B
:1048500001C014E1412F50E060E480E090E00E944C
:104860004D534C01009741F4F601E959FF4F87E39E
:1048700090E09183808369C1FC01A384B484D60154
:104880005A968D919C915B97F501918380839096C8
:104890008D919C91919793838283110F110F1487AF
:1048A00092968C919297877F92968C9392979B96F3
:1048B0006D917D918D919C919E970E940024D501D0
:1048C00014966D937D938D939C931797F60182A117
:1048D00084FF16C080E11D968C9382A18F7E82A3F7
:1048E000EC5BFF4F60817181828193810E94002483
:1048F000D50118966D937D938D939C931B9706C05D
:10490000F50115861086118612861386F60182A19E
:1049100081FF29C0E75AFF4F80819181082E892F9E
:10492000902D9A838983D5011D969C911D97926045
:104930001D969C93F60192A19D7F92A343A554A539
:1049400065A576A54F5F5F4F6F4F7F4F43A754A775
:1049500065A776A792E0F501948B94E0958B868B02
:104960008A81878B46C06114710439F1A30160E824
:10497000C4010E944D534C01009709F475CFA30167
:10498000B701DC011F968D919C9150970E941E6586
:10499000F60183A594A5A5A5B6A5860D971DA11D15
:1049A000B11D83A794A7A5A7B6A7D5011D968C9185
:1049B0001D9788601D968C931CC080FF1AC0F5015E
:1049C000858581608587D60192968C9192978E7F9E
:1049D00092968C9392979B968D919D910D90BC9100
:1049E000A02D0196A11DB11DF60183A794A7A5A72F
:1049F000B6A7F601E85BFF4F808191817196208117
:104A000031818217930730F4D5011F961C921E92B4
:104A10001E9706C0082E892F902DF501978786874F
:104A2000D50151961C921E92509753961C921E923D
:104A30005297F401E584F68481899289E80EF91E83
:104A40000E2CEF2CF02CD6015C962D913D914D91C2
:104A50005C915F9756966D917D918D919C91599740
:104A600006E00E94F432DC01CB01F4014585568555
:104A7000B5010E94C932D40151964D915C91529773
:104A80001F966D917C9150970E94EF32F501918BAA
:104A9000808B672821F48585837009F441C0D40197
:104AA0001D921C92D601DA96ED91FC91DB9730971E
:104AB00069F4DB969C928E92DA970E94E650F6019A
:104AC000EB59FF4F61607183608308C080819181E1
:104AD000009711F0FC01FACF918280828601055A7D
:104AE0001F4FF80180819181A281B381892B8A2B8C
:104AF0008B2B71F4D50114966D917D918D919C91C4
:104B000017970E940024F801608371838283938346
:104B100060E0C4010E94C0534C01892B09F4A4CE6B
:104B2000D6015C964D915D916D917C915F9794015A
:104B300086E00E9466348C01892B39F4C4010E94FE
:104B4000105305C000E010E002C00FEF1FEFC801D6
:104B50000F900F90DF91CF911F910F91FF90EF90E9
:104B6000DF90CF90BF90AF909F908F907F906F908D
:104B70000895AF92BF92CF92DF92EF92FF920F9380
:104B8000CF93DF936C01FC01C385D4858D8582FFB3
:104B900004C0C6010E9410536BC0F601A780B08408
:104BA000128A118A84E190E09687858788819981AD
:104BB0002A813B81398328839B838A832D8524FF27
:104BC0000FC084E08D8788859985AA85BB858C83F5
:104BD0009D83AE83BF83188619861A861B8618C0EC
:104BE0006C817D818E819F8121FF08C00E940024FD
:104BF0006F5F7F4F8F4F9F4F0E9400246887798798
:104C00008A879B871C821D821E821F8284E18D877A
:104C100080E58C871F861E861B8A1A8A198A188A45
:104C2000F601E584F6840E2CEF2CF02CF50124859A
:104C3000358546855785608971898289938906E023
:104C40000E94F432DC01CB01F60145855685BE0198
:104C50000E94EF32998B888BF501448555856685D6
:104C60007785960186E00E946634892B09F491CFFE
:104C700080E090E0DF91CF910F91FF90EF90DF9077
:104C8000CF90BF90AF900895062E692F902D072EDC
:104C9000782F802D0895FB01258536852531310536
:104CA00058F143855485FA017496DC01A75ABF4F29
:104CB0008081882309F1BF01641B750B621773079C
:104CC000DCF4813019F0823019F012C03196F0CF47
:104CD000828193819827892798276D917C911197DC
:104CE0008617970718F411969C938E933496E0CF0D
:104CF0008181E80FF11DDCCF08951F93CF93DF93DF
:104D0000EC01162F8D8990E08B30910508F057C08B
:104D1000FC018827E059FF4F8F4F0C9438636530B2
:104D200061F1663009F090C036C0633049F48AA161
:104D300082618AA34EC06330D1F3D0F16430E9F0D0
:104D40001B3009F081C03EC0643009F480C080F19E
:104D5000653009F1663009F077C08AA18160E9CF3A
:104D6000673059F020F4663009F471C06DC087EFE8
:104D7000860F833008F068C022C08AA18861D9CF2D
:104D80006B3001F18AA188618AA36A3011F15CC09D
:104D9000683009F059C08AA18161CBCF86EF860FB8
:104DA000823008F051C055C0623031F06B3051F0A4
:104DB000113009F049C04BC08AA18260BACF1B30C4
:104DC00009F045C081E090E09093F7088093F608E1
:104DD0003EC081E01D8B8823C1F040E050E060E0E0
:104DE00070E0CE010E940724892B79F0123069F41B
:104DF000FE01E959FF4F80E490E091838083CE016A
:104E000085599F4F0E94D4511FC0153039F5CE01EE
:104E10008D5A9F4F0E946D52CE0187599F4F0E941D
:104E20006D52CE0185599F4F0E946D52FE01EB5A83
:104E3000FF4F61E0808191810E94013D62E08EAD73
:104E40009FAD0E94013D0AC08FEF9FEF09C080E037
:104E5000C1CF6B3009F4B6CF8AE08D8B80E090E053
:104E6000DF91CF911F9108956F927F928F929F92C1
:104E7000AF92BF92CF92DF92EF92FF920F931F9368
:104E8000CF93DF93EC01FB013C0181E5680E711CBF
:104E9000D3018D919C91009749F0DC012D913C91BB
:104EA00011972115310519F0C901F7CFD301ED9301
:104EB000FC9321893289CE01865B9F4FDC016D9185
:104EC0007C911197620F731F6D937C930697690114
:104ED000032E000CEE08FF08DC018D909D90AD9034
:104EE000BC901397C80CD91CEA1CFB1CCD92DD9218
:104EF000ED92FC921397AE01485B5F4FDA018D9102
:104F00009C9111972817390718F01D921C9205C023
:104F1000821B930BDA018D939C938AA1982F906149
:104F20009AA320813181232B19F01182108202C0B3
:104F300088618AA38E01005B1F4FF80190819F5FFB
:104F400090839930E4F0D301ED91FC913097B9F062
:104F5000218932892F3F310509F044F4CF010E94A5
:104F60009F54F8019081981B908309C0915097300D
:104F700031F0621B730B0190F081E02DE7CF40E030
:104F800050E060E070E0CE01DF91CF911F910F9172
:104F9000FF90EF90DF90CF90BF90AF909F908F9059
:104FA0007F906F900C940724EF92FF920F931F93C2
:104FB000CF93DF93EC018B017A01FB01808991890A
:104FC000A289B3898E8B9F8BA88FB98FDA018D91BF
:104FD0009C9199A388A384859585A685B7858C8F98
:104FE0009D8FAE8FBF8FFA01648175818681978115
:104FF0000E944426FE01E05CFF4F60837183828340
:1050000093836FA778AB89AB9AAB3496DC01CB0165
:105010000196A11DB11D80839183A283B383D70123
:105020001E968D919C911F97082E892F902D98AFD9
:105030008FABF801648575858685978540E050E0E3
:105040000E94B0200097F1F0DC011F96ED91FC91D9
:1050500050978789908D8897FE01E75AFF4F2081EE
:1050600031812115310519F08217930710F49183CE
:105070008083808191812B893C898217930710F46A
:105080009C8B8B8BDF91CF911F910F91FF90EF90B5
:105090000895CF93DF93EC01892B21F10E94854D78
:1050A0008D8990E08B309105B8F4FC018827E55894
:1050B000FF4F8F4F0C9438636BE003C066E001C074
:1050C00068E0CE010E947D2680E090E00DC0C959C5
:1050D000DF4F85E290E004C0C959DF4F89E390E0DB
:1050E000998388838FEF9FEFDF91CF910895009789
:1050F00069F0FC0122A1286122A340E050E060E0B9
:1051000070E00E94072480E090E008958FEF9FEF09
:1051100008950F931F93CF93DF93E091CA08F09106
:10512000CB08CAECD8E0309791F025898281938131
:105130002B3049F49983888302811381CF010E9427
:10514000A81AF801F0CFEF012296FC01ECCFDF9115
:10515000CF911F910F910895CF92DF92EF92FF921E
:105160000F931F93CF93DF93EC01198218828091E4
:10517000120990911309892B59F4CE01DF91CF9137
:105180001F910F91FF90EF90DF90CF900C94B92575
:10519000C0908709D0908809C114D10429F4D09314
:1051A0008809C09387092CC009851A858D859E853D
:1051B000080F191F89899A89080F191FE09014098F
:1051C000F090150988EFF81AE00EF11E81EA99E0D7
:1051D0000E94924CE816F906F8F480911409909117
:1051E0001509080F191F1093150900931409F601EA
:1051F00080819181009711F06C01F9CFD183C08338
:1052000089E899E0DF91CF911F910F91FF90EF9086
:10521000DF90CF900C942352CE01DF91CF911F915C
:105220000F91FF90EF90DF90CF900C9410538091EE
:10523000120990911309892BC9F420E031E040E074
:1052400050E065E470E389E698E00E94745590931D
:1052500013098093120921E030E0892B11F020E03E
:1052600030E088279927821B930B089580E090E017
:105270000895FF920F931F93CF93DF93EC018B015F
:10528000FD88FC01E959FF4F7183608332971182D9
:1052900010823297118210828D89863018F08AE050
:1052A0008D8B01C01D8ACE010E94731ACE018D5ACA
:1052B0009F4F0E946D52CE01CC960E946D52CE013E
:1052C00087599F4F0E946D52CE0185599F4F0E9472
:1052D0006D5282E0F81203C00C33110569F0FE0133
:1052E000EB5AFF4F61E0808191810E94013D62E0B5
:1052F0008EAD9FAD0E94013D80E090E0DF91CF91A7
:105300001F910F91FF900895EF92FF920F931F93BB
:10531000CF93DF93EC01FC01EF59FF4F8081918126
:105320009C012F5F3F4F31832083089718F06CE377
:1053300070E013C02AAD3BADF901E080F1804C8DE7
:105340005D8D6E8D7F8D86E00E9466348C01892B89
:1053500051F0FBAEEAAE62E370E0CE010E94392963
:105360000FEF1FEF17C00E94E650FE01EB59FF4FF1
:10537000616071836083C15ADF4F88819981803178
:10538000F7E29F0718F4880F991F02C080E29EE49D
:1053900099838883C801DF91CF911F910F91FF906E
:1053A000EF9008954F925F926F927F928F929F92AB
:1053B000AF92BF92CF92DF92EF92FF920F931F9323
:1053C000CF93DF93EC018B015A01DB0118966D91AD
:1053D0007D918D919C911B970E9444266B017C01CD
:1053E0008BA59CA5ADA5BEA58C199D09AE09BF09CD
:1053F000B7FF04C08AA188618AA3EAC08FA198A5DB
:10540000A9A5BAA5C816D906EA06FB06C1F5F80192
:1054100064817581868197810E944426AB01BC011D
:105420008FA598A9A9A9BAA92C013D01441A550A2A
:10543000660A770A77FC11C0481759076A077B0785
:10544000F1F48BA99CA9ADA9BEA936014701681A40
:10545000790A8A0A9B0A97FC12C0D8011E968D9180
:105460009C911F97082E892F902D98AF8FAB4FA737
:1054700058AB69AB7AABCBAADCAAEDAAFEAA8FA186
:1054800098A5A9A5BAA5B701A601481B590B6A0B97
:105490007B0B77FD9DC0C816D906EA06FB0611F501
:1054A0008AAD9BAD892B09F493C0AB2809F090C05D
:1054B000F8018585837009F08BC089AD8F5F8330DB
:1054C00010F489AF85C019AECE010E94842921E075
:1054D00030E0892B11F420E030E088279927821BE7
:1054E000930B78C019AECFA2D8A6E9A6FAA6D80128
:1054F0001E968D919C911F97082E892F902D98AF05
:105500008FAB8E01055A1F4FF80180819181A281D6
:10551000B3810097A105B10549F08C199D09AE0929
:10552000BF09B7FF03C0CE010E947831D8011D9298
:105530001D921D921C9213970AAD1BAD011511050A
:1055400049F1D8011B96ED91FC911C9764817581FE
:10555000868197810E944426F80181889288092CCF
:10556000000CAA08BB08DC01CB01880D991DAA1DFF
:10557000BB1D23853485F9012585237019F001961B
:10558000A11DB11D36014701681A790A8A0A9B0AD2
:1055900097FE0EC08AAD9BAD8E010B591F4F892B14
:1055A00081F00E94E6506160F801718360830CC055
:1055B000D8018D919C919BAF8AAFC8010E94105376
:1055C000BBCFD8011D921C92CF59DF4F1982188290
:1055D00080E090E0DF91CF911F910F91FF90EF90CD
:1055E000DF90CF90BF90AF909F908F907F906F9003
:1055F0005F904F9008952F923F924F925F926F92DB
:105600007F928F929F92AF92BF92CF92DF92EF9252
:10561000FF920F931F93CF93DF9300D000D0CDB7AD
:10562000DEB79E838D838B01DB011B96CD90DC90D2
:105630001C97F601F584DC0155968C9190E08C3036
:10564000910508F078C4FC018827EA57FF4F8F4F77
:105650000C943863ED81FE8127A830AC27A130A5DA
:1056600041A552A529833A834B835C83F2FE0AC08D
:10567000CB010E94105366E370E08D819E810E94F1
:10568000392982C1F1FE18C0F601648175818681D5
:1056900097810E944426ED81FE81E05CFF4FC0802F
:1056A000D180E280F3806C157D058E059F0531F079
:1056B000C8010E94B92568C1F4FC04C0C8010E9459
:1056C000105362C1DB0151964D915C915297B60126
:1056D0008D819E810E94D229AD80BE80B4E4AB0E44
:1056E000B11CF5014080518062807380D601149610
:1056F0006D917D918D919C9117970E944426461A39
:10570000570A680A790A77FE80C0F8012189328930
:105710002115310509F465C08091F8089091F908C8
:10572000889645815681840F951F820F931F909311
:10573000F9088093F80881399C40D0F0C8010E9494
:1057400010538091F8089091F9088897D801159620
:105750002D913C911697821B930B51962D913C9164
:105760005297821B930B9093F9088093F8083CC0E2
:10577000ED81FE81E95AFF4F808091805F018114A5
:10578000910409F4F3C3F401E384F484D60114967C
:105790006D917D918D919C9117970E9444262B01CC
:1057A0003C01F70164817581868197810E944426BE
:1057B000A3019201261B370B480B590B57FF07C05B
:1057C000D5010D931C93F801918280820DC046167D
:1057D00057066806790629F05401F401808091800B
:1057E000CECFC8010E941053AD81BE8192968C919C
:1057F0009297886192968C93929740E050E060E097
:1058000070E0CD010E940724BFC0F601648175815C
:10581000868197810E944426D5014D905D906D90C0
:105820007C906415750586059705F1F0ED81FE8184
:1058300082A1886182A3EB58FF4F80819181A28170
:10584000B3810196A11DB11D80839183A283B3838F
:10585000C8010E94105340E050E060E070E08D818C
:105860009E810E9407247DC0D80151968D919C9104
:105870005297892B09F472C0B8018D819E810E94D4
:1058800034278D809E80B7E58B0E911CF40100813A
:10589000118101151105A9F0F801C384D484D50143
:1058A0004D905D906D907C90F6016481758186814C
:1058B00097810E944426461A570A680A790A77FE99
:1058C00010C08D819E818D5A9F4F0E94235261E0AE
:1058D000ED81FE81EB5AFF4F808191810E94013D55
:1058E00040C0D8018D919C911197F40191838083E0
:1058F0008091F8089091F908889715962D913C9120
:105900001697821B930B51962D913C915297821BB7
:10591000930B9093F9088093F808D60114966D9133
:105920007D918D919C9117970E944426F5014080AE
:10593000518062807380641575058605970551F462
:10594000B8018D819E810E943427D6011D968C91CD
:10595000F82A9CCFC8010E94105398CFC8010E941A
:105960001053F0FE11C0F50180819181A281B381B5
:105970000196A11DB11D80839183A283B38365E04D
:105980008D819E810E947D26AD81BE8155968C9130
:1059900055978430B9F4D7968D919C91D897281655
:1059A000390680F097968D919D910D90BC91A02D18
:1059B00029813A814B815C81281739074A075B07A7
:1059C00009F4DBC28D819E81CC960E946D5262E00B
:1059D000AD81BE81DE968D919C91DF9726960FB6A4
:1059E000F894DEBF0FBECDBFDF91CF911F910F9115
:1059F000FF90EF90DF90CF90BF90AF909F908F90EF
:105A00007F906F905F904F903F902F900C94013D4E
:105A10008F2D8671823009F073C2FB01678170851A
:105A2000A6018D819E810E94D4275DC0FF2DF0715B
:105A3000EF2EF4FE2AC0D60118966D917D918D91BE
:105A40009C911B970E944426ED81FE8183A094A027
:105A5000A5A0B6A0AB01BC01481959096A097B0988
:105A60004F5F5F4F6F4F7F4F83A594A5A5A5B6A548
:105A70000196A11DB11D88199909AA09BB098417AE
:105A80009507A607B70708F43BC2F2FE0AC0EE204E
:105A900009F451C26DE370E08D819E810E94392925
:105AA0004AC2F1FE48C2D80117966D917C911897B1
:105AB000A6018D819E810E94D427EE20A1F0F801DD
:105AC00041895289B6018D819E810E94D22964E06C
:105AD0008D819E810E947D268D819E8185599F4F5B
:105AE0000E94235228C263E0C4C1F2FE39C0ED8196
:105AF000FE81E759FF4F80819181892B31F061E070
:105B00008D819E810E947D2606C06DE370E08D81AF
:105B10009E810E943929C8010E941053ED81FE81A7
:105B2000EB59FF4F118210828D819E8126960FB610
:105B3000F894DEBF0FBECDBFDF91CF911F910F91C3
:105B4000FF90EF90DF90CF90BF90AF909F908F909D
:105B50007F906F905F904F903F902F900C94731AAE
:105B6000F1FCE9C1F4FEE7C1D60118966D917D9173
:105B70008D919C911B970E944426ED81FE8187A008
:105B800090A4A1A4B2A4AB01BC01481959096A09A7
:105B90007B094F5F5F4F6F4F7F4F83A594A5A5A5EE
:105BA000B6A50196A11DB11D88199909AA09BB09BD
:105BB00084179507A607B70708F4A2C1D801519624
:105BC0004D915C915297B601CF010E94D229F80104
:105BD00081899289892B31F0B8018D819E810E9443
:105BE000342703C0C8010E941053F0FE11C0ED819C
:105BF000FE81EC5BFF4F80819181A281B381019690
:105C0000A11DB11D80839183A283B38365E05CC134
:105C100064E08D819E810E947D268D819E818759C1
:105C20009F4F0E9423528D819E8185599F4F2696BA
:105C30000FB6F894DEBF0FBECDBFDF91CF911F919D
:105C40000F91FF90EF90DF90CF90BF90AF909F901B
:105C50008F907F906F905F904F903F902F900C941B
:105C60002352F2FE04C0C8010E9410532CC1F1FC63
:105C700047C1F4FE60C1DB0151964D915C91529792
:105C8000B6018D819E810E94D229ED81FE8143A5BE
:105C900054A565A576A587A190A5A1A5B2A548178D
:105CA00059076A077B0721F469E0CF010E947D262E
:105CB000D80151968D919C915297892BA9F0B801EA
:105CC0008D819E810E9434278D819E818D5A9F4FA8
:105CD0000E94235261E0ED81FE81EB5AFF4F8081EB
:105CE00091810E94013D03C0C8010E941053F0FE43
:105CF00044C1ED81FE81EC5BFF4F80819181A281E7
:105D0000B3810196A11DB11D80839183A283B383CA
:105D1000ED81FE81ED59FF4F11821082ED81FE81F0
:105D20008589893019F46AE0CF01D0C067E0CCC022
:105D3000F2FC99CFF1FCE4C0F4FEFDC0DB0151960A
:105D40004D915C915297B6018D819E810E94D2291E
:105D5000F80181899289892BA9F0B8018D819E81F2
:105D60000E9434278D819E818D5A9F4F0E9423521D
:105D700061E0ED81FE81EB5AFF4F808191810E94AD
:105D8000013D03C0C8010E941053F0FEF6C0ED8132
:105D9000FE81EC5BFF4F80819181A281B3810196EE
:105DA000A11DB11D80839183A283B383ED81FE8108
:105DB000ED59FF4F118210826AE086C0F2FE21C0C9
:105DC000CB010E94105366E370E08D819E81269680
:105DD0000FB6F894DEBF0FBECDBFDF91CF911F91FC
:105DE0000F91FF90EF90DF90CF90BF90AF909F907A
:105DF0008F907F906F905F904F903F902F900C947A
:105E00003929F1FC7DC0F4FE96C0DB0151964D911D
:105E10005C915297B6018D819E810E94D2298BC0E0
:105E2000F2FC21CFF1FC6CC0F4FE85C0FB0141897E
:105E30005289B6018D819E810E94D229AD81BE8199
:105E40009B964D915D916D917C919E9797968D91CA
:105E50009D910D90BC91A02D481759076A077B07AB
:105E600009F069C0ED81FE81ED59FF4F118210826A
:105E70006AE08D819E810E947D265DC0F2FCF3CE9A
:105E8000F1FC3EC0F4FE57C0FB0141895289B601C6
:105E90008D819E810E94D229C8010E941053AD813C
:105EA000BE819B964D915D916D917C919E97979649
:105EB0008D919D910D90BC91A02D481759076A07AF
:105EC0007B0709F05AC06BE08D819E8126960FB644
:105ED000F894DEBF0FBECDBFDF91CF911F910F9120
:105EE000FF90EF90DF90CF90BF90AF909F908F90FA
:105EF0007F906F905F904F903F902F900C947D26F5
:105F0000C80126960FB6F894DEBF0FBECDBFDF9155
:105F1000CF911F910F91FF90EF90DF90CF90BF90A6
:105F2000AF909F908F907F906F905F904F903F9039
:105F30002F900C94B925C80126960FB6F894DEBFB1
:105F40000FBECDBFDF91CF911F910F91FF90EF90CA
:105F5000DF90CF90BF90AF909F908F907F906F9089
:105F60005F904F903F902F900C941053F501118348
:105F70000083D8011D921C9237CC26960FB6F89458
:105F8000DEBF0FBECDBFDF91CF911F910F91FF906C
:105F9000EF90DF90CF90BF90AF909F908F907F90C9
:105FA0006F905F904F903F902F9008950F931F93A5
:105FB000CF93DF93EC018D89882329F0C959DF4FF6
:105FC00088E390E059C061E0CE010E947D266A8D91
:105FD0007B8D42E059E0AAEFB8E018E080E0FA01DA
:105FE00021913191AF0121153105A9F0F9012385E6
:105FF0003485F901228133816217730761F4183007
:1060000049F0212F30E02650374F0C91F901908153
:10601000901708F4182F8F5F1196883001F7183009
:10602000C1F0E12FF0E0EE0FFF1FEE5FF64F0081B1
:106030001181118210820115110559F0B801CE01AC
:106040000E944B26B801CE010E94FB2A80E090E01E
:1060500017C0FE01E359FF4F408151816281738176
:10606000CE0187599F4F0E946051009749F01D8AC9
:10607000C959DF4F8CE390E0998388838FEF9FEFBE
:10608000DF91CF911F910F91089580E20E94D54D2D
:10609000F12CCC24C3948091F6089091F708892BB9
:1060A00031F01092F7081092F6080E948928F394B4
:1060B00083E08F1538F4C2E0D9E0AAEFB8E0E8E059
:1060C00080E020C048EC50E060E070E089E899E0B2
:1060D0000E946051892B79F7C0918709D091880976
:1060E00010928809109287091092150910921409CC
:1060F0009CC09C91953058F49F5F9C938F5F119644
:10610000883039F029913991232B99F7F7CFE82F6F
:10611000F5CFE83069F0F0E0EE0FFF1FEE5FF64FCD
:106120008081918111821082009711F00E94B9251F
:10613000C091CA08D091CB08209709F456C08AA113
:1061400084FF09C088608AA340E050E060E070E00E
:10615000CE010E9407248AAD9BAD892BC9F08E0128
:106160000B591F4FF80180819181892B89F00E9482
:10617000E650F801208131812E7F621B730B369728
:10618000808191816817790718F0CE010E948429D7
:106190008D898A3019F08D89893089F4FE01ED5995
:1061A000FF4F808191819C012F5F3F4F318320837E
:1061B0000997B8F06BE0CE010E947D2616C08D894C
:1061C000833079F4FE01ED59FF4F808191819C016C
:1061D0002F5F3F4F318320838D9718F0CD8A118236
:1061E00010820A80DB81C02DA7CFF12C54CFEB8524
:1061F000FC85AF81B8851C962D913D914D915C91A8
:106200001F9760817181828193810E94BA1A8C01EB
:10621000E880D980009761F0BE010E944B26BE0144
:10622000C8010E94FB2ACE2DDD2D209701F733CF28
:106230002F813885AB85BC851D968C911D97867105
:10624000823009F051C042E0842E49E0942E00E0F3
:1062500010E058E0B52EF401819191914F01009723
:1062600029F4F8E0BF122AC0B02E28C0FC014781F3
:106270005085FA014484558466847784F901448505
:106280005585668577854416550666067706B1F40A
:10629000FC0143855485FA01608171814D915C91C7
:1062A00011976417750751F40E941053000F111FC6
:1062B000F801EE5FF64F1182108216C00F5F1F4F7C
:1062C0000830110541F6F8E0BF1671F08B2D90E013
:1062D000FC01EE0FFF1FEE5FF64FD183C083FC0180
:1062E000E650F74F10829FCFCE010E94B9259BCF79
:1062F0000F931F93CF93DF938C01EC01CB59DF4FAA
:1063000088819981892B11F10E94E650F801E15AA8
:10631000FF4F20813181220F331F488159814E7FE9
:10632000241B350B620F731FCB01880F991F880F39
:10633000991F803D27E0920728F06AE070E00E94F4
:10634000CF6202C068EC70E071836083DF91CF910F
:106350001F910F9108950F931F93CF93DF93EB013C
:10636000EB85FC85309729F08D859E8588309105D9
:1063700020F4CE010E94105365C008979A8B898B38
:1063800028E030E03E872D87892B21F0CF01089649
:10639000988B8F87828193810E948B1F8C0100973D
:1063A00071F48A8183FFE5CF8E0120E030E0A901FE
:1063B00063E083E00E945837892BD9F243C0DC01A7
:1063C0001A962D913C911B972115310501F11896D4
:1063D0004D915C91199789899A89840F951F281787
:1063E00039073CF21496ED91FC911597309751F0D6
:1063F000208131812115310511F0F901F9CFD183C7
:10640000C08303C0F801D583C483D8010EC0FC014A
:1064100084819581009711F00E941053D801159640
:10642000DC93CE93149789899A8919969C938E93BD
:106430001897F80186819781892B21F0C80106966B
:106440000E94235280E090E0DF91CF911F910F9145
:1064500008954F925F926F927F928F929F92AF9228
:10646000BF92CF92DF92EF92FF920F931F93CF9341
:10647000DF9300D01F92CDB7DEB77C012A013B012C
:106480004901C80148E050E060E40E944D536C01AE
:10649000009709F467C0DC011B96AD90BC901C9777
:1064A000F70182819381D5018D939C939401022EF3
:1064B000232F302DF50133832283D6011D962D9194
:1064C0003C911E9751968D919C915297820F931FEC
:1064D000082E892F902D95838483AE014F5F5F4FE7
:1064E000C301B2010E94B020009771F0DC011F9639
:1064F000ED91FC91509783859485A585B685898318
:106500009A83AB83BC8304C019821A821B821C82CB
:10651000F50117821682E480F58069817A818B818A
:106520009C8101E1A30192010E94F432DC01CB01C4
:1065300048E050E0B5010E94C932D60151964D9114
:106540005C9152971F966D917C9150970E94EF320B
:10655000F501978386839601B301A20181E10E9430
:10656000663402C08FEF9FEF0F900F900F900F9047
:10657000DF91CF911F910F91FF90EF90DF90CF901F
:10658000BF90AF909F908F907F906F905F904F9053
:106590000895FB01A0E0B0E0423051054CF021919C
:1065A0003191820F931FA11DB11D42505109F4CFAB
:1065B000452B29F02081820F911DA11DB11DAD0138
:1065C00066277727411551056105710539F0AA271E
:1065D000BB27840F951FA61FB71FF1CF08950E94F8
:1065E000C932809590950895EF92FF920F93CF93C3
:1065F000DF93CDB7DEB72C970FB6F894DEBF0FBE92
:10660000CDBF69837A838B839C832D833E834F83A5
:10661000588719860A87FC86EB864CE050E0BE015D
:106620006F5F7F4F80E090E00E94C932BC0180E044
:1066300090E02C960FB6F894DEBF0FBECDBFDF9171
:10664000CF910F91FF90EF9008956F927F928F926C
:106650009F92AF92BF92CF92DF92EF92FF920F93F1
:106660001F93CF93DF931F92CDB7DEB77C013B0121
:10667000DB0117960D911C911897F8018081807F9E
:10668000803409F092C086819781082E892F902D41
:106690009F73892B09F089C0E0911609F0911709C1
:1066A000309759F0D8011C966D917D918D919C91F8
:1066B0001F971995892B09F078C0F80180818F7098
:1066C000880F880F843108F470C090E0D3011996C8
:1066D000CD90DC901A97C816D9060CF466C0408994
:1066E000518962897389F701A785B0894F3FFFEF10
:1066F0005F076F077F0709F46EC04A015B0120EF57
:1067000082229924AA24BB24E0EE8E169104A104CF
:10671000B104B9F45D960D90BC91A02D109709F4C9
:1067200044C018968D909D90AD90BC901B974815D5
:1067300059056A057B0509F44AC00D90BC91A02D4E
:10674000EDCF1B968D909D90AD90BC901E978114BF
:106750009104A104B104E9F1481559056A057B05C6
:1067600041F4D30112962C911297286012962C9323
:1067700030C053968D909D90AD90BC905697BFEFD2
:106780008B169B06AB06BB0669F080949094A09490
:10679000B094482159216A217B2184169506A606CA
:1067A000B706C9F0C3010E942336C3010F90DF91E1
:1067B000CF911F910F91FF90EF90DF90CF90BF90FE
:1067C000AF909F908F907F906F900C94105342E009
:1067D00003C040E001C041E0F80122813381022E74
:1067E000232F302DD3011E963C932E931D972817EF
:1067F0003907DCF2C216D306C4F21A969C938E9324
:106800001997281B390B1E963C932E931D97232B0B
:1068100031F0800F911F1C969C938E931B97E091F3
:106820008B09F0918C093097C9F4F801818581308A
:10683000E9F0823071F5B301C7010F90DF91CF917C
:106840001F910F91FF90EF90DF90CF90BF90AF908E
:106850009F908F907F906F900C940038B301C70188
:10686000498319954981892B01F720C0B301C701DC
:106870000F90DF91CF911F910F91FF90EF90DF90DC
:10688000CF90BF90AF909F908F907F906F900C941F
:10689000263641118ACF830120E030E0A90162E071
:1068A00083E00E945837892B09F47FCF0F90DF9146
:1068B000CF911F910F91FF90EF90DF90CF90BF90FD
:1068C000AF909F908F907F906F9008957F928F925E
:1068D0009F92AF92BF92CF92DF92EF92FF920F936F
:1068E0001F93CF93DF93CDB7DEB72E970FB6F894F3
:1068F000DEBF0FBECDBFD82E4B875C876D877E87EE
:10690000C90122E0D21649F044E150E060E20E9461
:106910004D537C01009721F4FCC048E150E0F6CFD4
:10692000DC0117960D911C911897F80180818F70EA
:1069300080648083807FF2E0DF1204C08660D8012B
:106940008C9303C08560F8018083D80111961C9256
:106950001197F7012185328585859685820F931FD2
:1069600021893289820F931F082E892F902D13962B
:106970009C938E93129717961C921E921697B2E0D4
:10698000DB1204C081E0F801808704C080E4D801F4
:1069900018968C93F801D1868B849C84AD84BE8438
:1069A000808A918AA28AB38AB2E0DB120EC080E0AC
:1069B00090E0A4E0B4E9082E8B2FB02D092E9A2F79
:1069C000A02D848B958BA68BB78BFFEF8F169F0620
:1069D000AF06BF0609F4A0C0D501C401082E8B2F55
:1069E000B02D092E9A2FA02D88279927AA27B07F8E
:1069F0000097A105B04E09F405C1AE01495F5F4F94
:106A0000C501B4010E94B0205C01009709F47EC06A
:106A1000DC011F96CD90DC905097F601818D928D10
:106A20009C01022E232F302DD80115963C932E93D6
:106A300014970196928F818F83859485A585B6855D
:106A4000F80184879587A687B78713861286D701B2
:106A500019964D915C911A9717966D917C911897A4
:106A600080E090E00E94EF32F80193878287D601A0
:106A70008C918630E1F54F81588569857A8541157D
:106A8000510561057105E1F44B855C856D857E8559
:106A900053968D919D910D90BC91A02D842B952B9B
:106AA000A62BB72B8F3F9F4FAF4FBF4F49F446E008
:106AB00050E06FEF70E0CE0101960E9427650BC099
:106AC0009E012F5F3F4FC5010E943E39892B19F06F
:106AD00080E090E0A4C0D6019396ED91FC9194974C
:106AE0009701AE014F5F5F4F60E078E00CC08731E7
:106AF00069F4D6019396ED91FC919497970140E04B
:106B000050E061E270E0C501199589C0C7010E949B
:106B100010538FEF9FEF83C046E050E06FEF70E0BF
:106B2000CE0101960E94276500914C0910914D09F4
:106B3000772473940115110559F2D8011B968C9195
:106B4000833009F05BC060E2C7010E94C0536C0152
:106B5000F801A784B088DC0117968D909C90189757
:106B6000F501818D928D9C01022E232F302DD401B1
:106B700015963C932E9314970196928F818F83855F
:106B80009485A585B685F40184879587A687B78700
:106B9000708613861286D60119964D915C911A97CC
:106BA00017966D917C91189780E090E00E94EF32EB
:106BB000F40193878287D5018C91863059F493969E
:106BC000ED91FC9194979601AE014F5F5F4F60E0AD
:106BD00078E010C0873121F0C6010E9410530EC02A
:106BE000D5019396ED91FC919497960140E050E089
:106BF00061E270E0C8011995892B71F3F8010081F9
:106C0000118198CF81E089831A828EE58B838C85F0
:106C10008F778C838D858D838E858E8385CF2E9601
:106C20000FB6F894DEBF0FBECDBFDF91CF911F919D
:106C30000F91FF90EF90DF90CF90BF90AF909F901B
:106C40008F907F90089580E090E00895CF92DF923A
:106C5000EF92FF920F931F93CF93DF938C016B0101
:106C6000DB011B96CD91DC911C97209709F48DC018
:106C70001D962D913C911E972830310508F485C052
:106C800028503109FB01328B218B232B41F0CE019F
:106C90000896908B878788E090E096878587988113
:106CA000933029F1983009F070C0D6011796ED9114
:106CB000FC9118974485558566857785D8011F9680
:106CC0008D919C915097DC011B960D911D912D91FA
:106CD0003C911E9704871587268737878FEF80871B
:106CE000960180E00E94D936892B09F059C0C981EC
:106CF000D0E0F601818992894C9708F446C0E78478
:106D0000F088D70119968C91863019F0813119F1EC
:106D10003CC0F7012485358546855785E057FE4FF1
:106D200060817181828193810E94BA1A009769F112
:106D3000DC0155962C915597223021F055962C91D7
:106D4000243019F5CC0FDD1FCC5CDB4F68817981D5
:106D50000E9439291AC0F701868997890E948B1FE2
:106D6000009799F0CC0FDD1FCC5CDB4F08811981B7
:106D7000D70156962D913C91579750964D915D9124
:106D80006D917C9153970E94B31FC601DF91CF9103
:106D90001F910F91FF90EF90DF90CF900C941053C4
:106DA000DF91CF911F910F91FF90EF90DF90CF90E7
:106DB0000895CF92DF92EF92FF920F931F93CF939C
:106DC000DF936A017B01E9010B851C85F801808353
:106DD000138212824D855E856B857C8580E090E014
:106DE0000E94C93249895A896F8578890E94EF3299
:106DF000F801938382839E01B701A60181E0DF91B0
:106E0000CF911F910F91FF90EF90DF90CF900C9456
:106E100066344F925F926F927F928F929F92AF9261
:106E2000BF92CF92DF92EF92FF920F931F93CF9377
:106E3000DF93C82FD62F49015A01C60148E050E020
:106E400060E40E944D53009701F1DC011B96ED9127
:106E5000FC911C97D18384829582A682B7829C0183
:106E6000B801A7018C2FDF91CF911F910F91FF9057
:106E7000EF90DF90CF90BF90AF909F908F907F90DA
:106E80006F905F904F900C94D9368FEF9FEFDF910A
:106E9000CF911F910F91FF90EF90DF90CF90BF9017
:106EA000AF909F908F907F906F905F904F900895DC
:106EB0002F923F924F925F926F927F928F929F920A
:106EC000AF92BF92CF92DF92EF92FF920F931F93F8
:106ED000CF93DF93382E262E29013A01C801D8011D
:106EE0001796ED91FC91189784849584A684B784B5
:106EF0004CE150E060E80E944D53EC01892BE9F031
:106F0000AF85B889EF81F88584E101900D928A956B
:106F1000E1F7AF85B8895496EB85FC8588E0019050
:106F20000D928A95E1F76E0185017401A30192012A
:106F3000622D832D0E94093702C08FEF9FEFDF91F2
:106F4000CF911F910F91FF90EF90DF90CF90BF9066
:106F5000AF909F908F907F906F905F904F903F90F9
:106F60002F900895BF92CF92DF92EF92FF920F93EE
:106F70001F93CF93DF93B82E6A017B0148E050E066
:106F800060E480E090E00E944D53EC01892B59F1C0
:106F90000B851C8588E090E09E878D87F801B08284
:106FA0001182C482D582E682F782138212824D85D5
:106FB0005E856B857C8580E090E00E94EF32F80171
:106FC000938382839E0140EE50E060E076E182E0B0
:106FD000DF91CF911F910F91FF90EF90DF90CF90B5
:106FE000BF900C946634DF91CF911F910F91FF9069
:106FF000EF90DF90CF90BF90089586E10C94B23768
:107000000F931F93CF93DF938C01CB01DB011B9672
:10701000ED91FC911C97309749F11D962D913C9173
:107020001E972830310514F120812231F9F02631E4
:10703000E9F02131D9F4F801C785D0890E941053B5
:107040000D8CDE8DC02D2097B9F0488559856A8555
:107050007B85403E51056105F1E07F0719F0C801CD
:107060000E94FD370990D881C02DEDCFDF91CF91DF
:107070001F910F910C941053DF91CF911F910F919D
:1070800008950F931F93CF93DF93FC01C38DD48D8D
:107090008C01055E1F4F2097C1F08C8580FF10C0CA
:1070A000CE010E960E94365288819981F801918313
:1070B0008083CE010E940146F801C081D181EBCFCF
:1070C0008E010990D881C02DE6CFDF91CF911F911D
:1070D0000F9108950F931F93CF93DF930E94DD507C
:1070E000009118091091190920911A0930911B0972
:1070F000DC01CB01801B910BA20BB30BCC97A1053C
:10710000B105D0F10E94DD50609318097093190900
:1071100080931A0990931B09C0914C09D0914D0995
:10712000209751F18B85833019F58F8598890097C9
:10713000F9F0DC012C912630D9F45B96ED91FC91AD
:107140005C9730E0309789F0248522FD08C04585A2
:1071500051E0540F5587493010F021602487248571
:10716000322B0190F081E02DEDCF30FD0E944138AF
:107170000990D881C02DD4CFDF91CF911F910F916D
:107180000895EF92FF920F931F93CF93DF9300D058
:107190001F92CDB7DEB77901FC0107851089F80190
:1071A000238D348D2115310561F1F901828193819F
:1071B000A481B581481759076A077B0719F0208118
:1071C0003181F0CFF901848582FD0DC0F90115866A
:1071D00096E0F701D901169601900D929A95E1F784
:1071E0008260F9018487C9010E960F900F900F906D
:1071F0000F90DF91CF911F910F91FF90EF900C9422
:107200006D5249835A836B837C830E946A3880E184
:1072100090E00E94F3459C0149815A816B817C81F9
:10722000892B09F180E1F90111928A95E9F7F901B9
:107230004283538364837583E114F10459F086E03B
:10724000F701D901169601900D928A95E1F782E037
:10725000F9018487F801838D948DF90191838083EE
:10726000F801348F238F0F900F900F900F90DF91C4
:10727000CF911F910F91FF90EF9008954F925F92E1
:107280006F927F92AF92BF92CF92DF92EF92FF9276
:107290000F931F93CF93DF935C012A013B01690198
:1072A000DC011F96ED90FC9050970E946A38F70120
:1072B000C38DD48D209709F459C08A819B81AC81FC
:1072C000BD81481659066A067B0621F00990D881CF
:1072D000C02DF0CF00E010E08C8581FD2FC001159E
:1072E000110571F444EF51E060E070E0CE010E96BC
:1072F0000E946051D7015B96CD91DC915C9718C0DC
:10730000B801C5010E946E3A892B61F3D7015B96E3
:10731000ED91FC915C9727C08A819B81AC81BD81F6
:10732000481659066A067B0631F00990D881C02DAF
:10733000209791F751C08C8581FF55C02C96F6019E
:1073400036968A918293CE16DF06D9F73CC08281A9
:107350009381A481B581481659066A067B0669F1B6
:107360000190F081E02D309791F749C00E946A3872
:1073700080E190E00E94F345EC01892B09F43FC0C5
:1073800080E1DE011D928A95E9F74A825B826C8278
:107390007D82F701838D948D99838883D48FC38FE9
:1073A00020E030E0B301A20181E090E00E94103AB9
:1073B0008C01892B09F090CF1CC0848581FD1FC0F2
:1073C0008160848719C00115110519F0C8010E9458
:1073D000105380E090E015C00115110581F0C8013F
:1073E0000E9410530CC00115110549F0C8010E94FC
:1073F00010538C8581608C87C7010E9441388FEFC4
:107400009FEFDF91CF911F910F91FF90EF90DF9051
:10741000CF90BF90AF907F906F905F904F90089506
:107420008F929F92AF92BF92CF92DF92EF92FF9294
:107430000F931F93CF93DF938C014A015B01690186
:107440004CE150E060E280E090E00E944D537C010E
:10745000009709F434C0FC01C781D08581E090E039
:10746000082E892F902D9983888380E098E0082E3C
:10747000892F902D9B838A8386E08C8384E08D8383
:10748000C801082E892F902D9F838E83CE014296AE
:10749000C114D10441F026E0F601DC0101900D9207
:1074A0002A95E1F706C046E050E06FEF70E00E94D9
:1074B0002765888E998EAA8EBB8EC70102C080E098
:1074C00090E0DF91CF911F910F91FF90EF90DF90AF
:1074D000CF90BF90AF909F908F9008950F931F9380
:1074E000CF93DF939B01DB011796CD91DC91189729
:1074F000FC0107851089DE011896F801359646E0F3
:1075000001900D924A95E1F7D8011B964D915D913E
:107510006D917C911E974E875F87688B798BAE014A
:107520004E5E5F4F9396ED91FC91949766E078E004
:10753000DF91CF911F910F911994CF93DF93C82FB3
:10754000D92FDC0120E03FEFE991EE23A9F1E032F1
:1075500074F10E2E000CFF0BE455FB4FE491EF3F4E
:1075600031F141E0420F223059F02330B9F021309F
:1075700001F52E2F2073522F52955F7064E006C0E4
:107580002E2F2C73522F5695569560E1360290019E
:107590001124252B2C93242F11960CC040E4340287
:1075A000900111242E2B2C93119620E003C0E32F81
:1075B00001C0242F3E2FC8CF1C92DF91CF91089598
:1075C000EF92FF920F931F93CF93DF93CDB7DEB768
:1075D0002D970FB6F894DEBF0FBECDBF7B01FC0127
:1075E000DE01119690E0AD018F012191222339F047
:1075F0002A3329F0983019F02D939F5FF5CFFA01C7
:10760000E90FF11D1082CA010E9480520097B1F06B
:10761000D8012C912A3311F40F5F1F4F1B870A8763
:10762000FD86EC86DC015596ED91FC915697AE01F6
:10763000465F5F4F61E071E1199502C08FEF9FEFE8
:107640002D960FB6F894DEBF0FBECDBFDF91CF9160
:107650001F910F91FF90EF9008958FEF9FEF089586
:10766000DC011296ED91FC9113970190F081E02DD1
:107670006481758180E090E00895CF92DF92EF926F
:10768000FF920F931F93CF93DF936C017B0184E0F4
:1076900090E00E94F345EC01892B39F48CE090E0F6
:1076A0009093A00980939F0938C0F70180818F32A1
:1076B00019F4FFEFEF1AFF0A009100021091010286
:1076C0000115110561F0F80162817381C7010E9403
:1076D000EB64892B71F0F80100811181F1CF82E018
:1076E00090E09093A00980939F09CE010E940146EB
:1076F00014C064E070E081E090E00E94D7450097FC
:1077000049F0FC0111830083D982C8829B838A835C
:10771000CE0105C08CE090E0E4CF8FEF9FEFDF91CA
:10772000CF911F910F91FF90EF90DF90CF90089530
:107730000F931F93CF93DF939B01EA01DC01129615
:107740000D911C911397D801ED91FC911197129610
:107750006D917C91139784819581861B970B84177B
:10776000950708F4EC01209779F086819781680FDE
:10777000791FAE01C9010E94E264F8018281938100
:107780008C0F9D1F93838283CE01DF91CF911F9138
:107790000F9108950F931F93CF93DF93EA01633204
:1077A0007141A9F52A813B81E881F9810281138128
:1077B000F80140815181F90180819181A281B381D9
:1077C0006C817D816130710539F06230710559F449
:1077D000FA016481758103C0F80162817381860FAB
:1077E000971FA11DB11DB7FD12C0FA01448155813B
:1077F00060E070E0481759076A077B0744F0F8011A
:1078000093838283F90180839183A283B3838FEF73
:107810009FEFDF91CF911F910F910895CF93DF9349
:10782000EC0101978E3F9F4F48F48A819B8100971E
:1078300011F00E940146CE010E94014680E090E0D6
:10784000DF91CF9108958FEF9FEF0895CF93DF934E
:107850008830910548F089E090E09093A0098093EA
:107860009F098FEF9FEF22C0880F991FEC01C45E24
:10787000D64F88819981009771F3DC01ED91FC91DD
:107880001197309769F4198218821796ED91FC913F
:10789000189740E050E060E070E0DF91CF911994DC
:1078A000078CF0A1E02D199519821882DF91CF91F4
:1078B000089588309105D0F4880F991FFC01E45E8B
:1078C000F64FA081B181109789F08D919C9111970D
:1078D000009731F41B96ED91FC911C97CD0105C0EA
:1078E000DC015596ED91FC915697199489E090E052
:1078F0009093A00980939F098FEF9FEF0895AF9217
:10790000BF92CF92DF92EF92FF920F931F93CF938C
:10791000DF93CDB7DEB729970FB6F894DEBF0FBE61
:10792000CDBF5B01FC01DE01119690E0AD016F015E
:107930002191222339F02A3329F0983019F02D9320
:107940009F5FF5CFFA01E90FF11D1082CA010E9475
:107950008052009719F482E090E011C0ECE1F9E068
:10796000E12CF12C21913191232B81F02FEFE21AA0
:10797000F20AA8E0EA16F104A9F788E190E09093F2
:10798000A00980939F098FEF9FEF2AC08701000F06
:10799000111FF801E45EF64F2FEF3FEF3183208394
:1079A000F60120812A3321F4B6016F5F7F4F02C0B8
:1079B00060E070E0DC015D96ED91FC915E9720E067
:1079C00030E0A5011995F801E45EF64F8F3FBFEF57
:1079D0009B0719F411821082D6CF91838083C7014F
:1079E00029960FB6F894DEBF0FBECDBFDF91CF91C1
:1079F0001F910F91FF90EF90DF90CF90BF90AF90CD
:107A000008950F931F93CF93DF931F92CDB7DEB7E7
:107A10008C010115110571F0F8018481862331F084
:107A20008281938169830E94D4516981F801008128
:107A30001181EFCF0F90DF91CF911F910F9108959A
:107A4000CF93DF93FC012FEF3FEF3097E9F0848174
:107A50008623B1F0C281D381A881B981109719F42E
:107A6000398328830DC0AF3F8FEFB80749F01496D4
:107A70008D919C911597019615969C938E931497D2
:107A80000190F081E02DE1CFDF91CF910895EF9249
:107A9000FF920F931F93CF93DF93EC018B017A0139
:107AA0002115310509F442C0892B09F43FC0672B29
:107AB00009F43CC0452B09F439C02130310541F0AF
:107AC0002230310509F032C00FB6F8940F921EC073
:107AD00085E090E00E94F345FC0113830283E48279
:107AE0000FB6F8940F928881998191838083F983EE
:107AF000E8830F900FBE1AC0FC01428153812081A0
:107B00003181398328830417150721F088819981F1
:107B1000009791F70F900FBE009741F0DF91CF9142
:107B20001F910F91FF90EF900C940146DF91CF9140
:107B30001F910F91FF90EF9008958830910538F0D4
:107B400089E090E09093A00980939F091AC0880F64
:107B5000991FFC01E45EF64F80819181009781F3CB
:107B6000DC01ED91FC911197309729F41596ED9178
:107B7000FC91169705C00788F08DE02D309709F02D
:107B800019948FEF9FEF0895EF92FF920F931F9339
:107B9000CF93DF937C01892B49F489E090E09093A7
:107BA000A00980939F090FEF1FEF25C0E4EAF2E0E0
:107BB000C0E0D0E081919191E816F90629F0219674
:107BC000C830D105B9F7E9CFF701808191810E94D2
:107BD000263C01E010E0892B11F400E010E0119543
:107BE00001951109C7010E940146CC0FDD1FCC553C
:107BF000DD4F19821882C801DF91CF911F910F913B
:107C0000FF90EF900895EF92FF920F931F93CF9301
:107C1000DF938C01CB010E94CB3E7C018FEFE816F5
:107C2000F80609F455C00830110510F1D8018D91FE
:107C30009C911197892BE1F414968C9114978430C0
:107C4000B9F4ECE1F9E080E090E08C012191319110
:107C5000232B39F0019688309105B9F788E190E03F
:107C600015C0FC01EE0FFF1FE45EF64FB183A08349
:107C7000E4EAF2E0C0E0D0E081919191892B59F0E3
:107C80002196C830D105C1F787E190E09093A00913
:107C900080939F091DC087E090E00E94F345FC019E
:107CA000CC0FDD1FCC55DD4FF983E883309741F0D1
:107CB00011830083F382E28214821682158206C049
:107CC0008CE090E09093A00980939F09CF0102C0BF
:107CD00080E090E0DF91CF911F910F91FF90EF90A6
:107CE000089540E050E060E070E0FC018081918107
:107CF0000E94A94921E030E0892B11F420E030E016
:107D000088279927821B930B0895CF93DF9300D088
:107D10001F92CDB7DEB78830910550F089E090E032
:107D20009093A00980939F096FEF7FEFCB0128C04C
:107D3000880F991FFC01E45EF64F808191810097C6
:107D400069F3DC01ED91FC911197309799F41B9642
:107D5000ED91FC911C97309709F3AE014F5F5F4F97
:107D60006AE070E01995892BC9F669817A818B8167
:107D70009C8106C001A0F2A1E02D309779F21995FF
:107D80000F900F900F900F90DF91CF910895FC010D
:107D9000808191810895FC012081223771F027377D
:107DA00039F0213699F46AE071E049E051E009C008
:107DB00062E073E041E053E004C062E070E040E064
:107DC00050E0FC01319620E030E40CC086E190E008
:107DD0009093A00980939F098FEF9FEF08958B32B6
:107DE00029F4AB0181918111FACF05C0823671F778
:107DF00020E030E8F7CFCA01822B932B08959F92A1
:107E0000AF92BF92CF92DF92EF92FF920F931F93A8
:107E1000CF93DF935C01CB018A010E94CB3E7C01B2
:107E2000019699F0E4EAF2E0C0E0D0E0819191910E
:107E30008017910769F02196C830D105B9F789E01C
:107E400090E09093A00980939F09E0E0F0E032C0B9
:107E500087E090E00E94F3456C018E01000F111F36
:107E60000C551D4FF801D182C082C114D10469F3B1
:107E7000B701C5010E947F3C9C01F601918380837C
:107E8000F801808191812F3F3F4F71F40E9401469C
:107E900042E04C1728F02196F801D183C083D5CF5A
:107EA000F80111821082D1CFFC01F382E2821482A8
:107EB00016821582CF01DF91CF911F910F91FF9014
:107EC000EF90DF90CF90BF90AF909F9008950F9369
:107ED0001F93CF93DF931F92CDB7DEB78C01FC01C8
:107EE000848183FF05C0877F8483858196811BC041
:107EF00041E050E0BE016F5F7F4FF80180819181CA
:107F00000E949D3D9C01019761F0F8019481232B13
:107F100011F0906102C09062F80194838FEF9FEF9F
:107F200002C0898190E00F90DF91CF911F910F9156
:107F30000895CF92DF92EF92FF920F931F93CF930A
:107F4000DF938C016A017B01C02FD12F82E0E816FC
:107F5000F104A4F0C6010E94673F8F3F2FEF920704
:107F600021F4188280E090E00BC02196FE01319749
:107F7000808321E0E21AF1080A9741F71882C801CC
:107F8000DF91CF911F910F91FF90EF90DF90CF90F5
:107F90000895CF93DF93CDB7DEB7AE01465F5F4F55
:107FA000688579858E819F810E942640DF91CF91DF
:107FB0000895CF93DF93EB016230710540F0BA0171
:107FC0006C9FA0016D9F500D7C9F500D1124BC0132
:107FD000F901808191810E94A9491816190644F47B
:107FE000C230D10538F0BE010E94CF62CB0102C081
:107FF00080E090E0DF91CF910895CF93DF93CDB7EC
:10800000DEB7AE014A5F5F4FFA0161917191AF0136
:108010008091A6029091A7020E942640DF91CF9105
:1080200008956091A6027091A7020E94144A8F3FA2
:108030002FEF920751F06091A6027091A7028AE09B
:1080400090E00E94F44980E090E008950F931F9320
:108050009B01FC01808191818A01AC0160ED79E492
:1080600089EA99E40E947A461F910F910895CF936F
:10807000DF93CDB7DEB7AE01465F5F4F6885798588
:108080008E819F810E945A40DF91CF9108950F9376
:108090001F93CF93DF93EC018B010E94FB64AC0133
:1080A000BE01F80180819181DF91CF911F910F91E5
:1080B0000C94D049AF92BF92CF92DF92EF92FF9291
:1080C0000F931F93CF93DF935C01EB018A01CB01E8
:1080D0000E94FB6401966C01BC0181EA99E00E9458
:1080E000B34B7C010097C1F0A601BE010E94E2647F
:1080F000F50140815181970160ED79E489EA99E4C5
:108100000E947A46D82FC92FB70181EA99E00E94D0
:108110001B4C8D2F9C2F02C08FEF9FEFDF91CF91D3
:108120001F910F91FF90EF90DF90CF90BF90AF9095
:108130000895CF93DF93CDB7DEB7AE01465F5F4FB3
:10814000688579858E819F810E94C140DF91CF91A2
:1081500008950F931F93CF93DF938C01EA01FC01E5
:10816000808191810E941E65F801808191818C0F30
:108170009D1F91838083CE01DF91CF911F910F913D
:1081800008950F931F93CF93DF931F921F92CDB744
:10819000DEB79A8389839B018A01AE014F5F5F4FEF
:1081A00060EE70E489EA90E40E947A46E981FA81FF
:1081B00010820F900F90DF91CF911F910F91089532
:1081C0000F931F93CF93DF938C01EA01FC01808111
:1081D00091810E94E264F801808191818C0F9D1F42
:1081E00091838083CE01DF91CF911F910F910895EC
:1081F0004F925F926F927F928F929F92AF92BF92B7
:10820000CF92DF92EF92FF920F931F93CF93DF9362
:10821000EB01FC014080518062807380209709F45B
:10822000E8C0C301B20120E83FE146E857E00E9400
:10823000F76249015A0160E87FE186E897E00E9411
:10824000B36293018201061B170B280B390BB9018E
:10825000A80168017901D501C40132E0880F991F96
:10826000AA1FBB1F3A95D1F7403813E3510711EE0F
:10827000610711E071072CF48A5B9F4FAF4FBF4F2E
:108280003AC04A015B0120E8821A23E3920A21EEF8
:10829000A20A21E0B20A30E8831633E3930631EEF6
:1082A000A30631E0B30638F4895B9F4FAF4FBF4F51
:1082B0007501640120C0E7E6DE1AE2ECEE0AE3E0B5
:1082C000FE0AC114F5E8DF06F2EEEF06F1E0FF0664
:1082D00030F4885B9F4FAF4FBF4F11E00DC0875BFD
:1082E0009F4FAF4FBF4F6A017B010CEED01A04EADB
:1082F000E00A05E0F00A10E09B878A87C701B60113
:1083000020E831E541E050E00E94F76249015A015E
:10831000F9013F872E87D90120E831E541E050E09F
:108320000E946963C61AD70AE80AF90A111103C044
:1083300084EB92E002C08EEC92E0DC01129641E008
:1083400050E060E070E02D913D912E173F072CF436
:108350004F5F5F4F6F4F7F4FF6CF4150510961091B
:10836000710959874887440F551FFC01E40FF51F19
:1083700080819181881A990A9F828E82C301B201FD
:1083800020E831E541E050E00E94F762C90104961F
:1083900067E070E00E94E3629D878C87C701B601A9
:1083A00020E13EE040E050E00E9419633D832C83D1
:1083B000A0EFB1EF0E944063C60ED71EE81EF91E63
:1083C000C701B6012CE330E040E050E00E941963A1
:1083D0003B832A8314EC1203B001139F700D112408
:1083E000C60ED71ED982C882198A188A80E090E00A
:1083F00002C08FEF9FEFDF91CF911F910F91FF9000
:10840000EF90DF90CF90BF90AF909F908F907F9034
:108410006F905F904F9008956DE879E00E94F8406A
:10842000892B19F48DE899E0089580E090E0089593
:108430004F925F926F927F92AF92BF92CF92DF92F4
:10844000EF92FF920F931F93CF93DF9300D01F9271
:10845000CDB7DEB78C015B01FC01828593856C0191
:10846000092E000CEE08FF08C982DA82EB82FC823A
:10847000855491098734910520F06FEF7FEFCB0190
:1084800073C1F801808591858C309105E8F4F8017D
:1084900080859185FC01EE0FFF1FEC54FD4FC080DD
:1084A000D1802601DD0C66087708C980DA80EB8070
:1084B000FC80B701A6014370552766277727452B17
:1084C000462B472B99F139C06CE070E00E94E362C3
:1084D000AB01770F660B770BC40ED51EE61EF71E99
:1084E000C982DA82EB82FC8297FD04C0F801918791
:1084F00080870DC00C96F80191878087F1E0CF1A34
:10850000D108E108F108C982DA82EB82FC82898114
:108510009A81AB81BC8185549109A109B109873445
:108520009105A105B10508F4B2CFA7CF02972CF0B1
:108530002FEF421A520A620A720AA70196012654C4
:10854000310941095109ADE6B1E00E945E63E1E005
:10855000CE1AD108E108F10822E0F594E794D79407
:10856000C7942A95D1F7DC01CB018C0D9D1DAE1D62
:10857000BF1D4197A109B10973016201C80ED91E3F
:10858000EA1EFB1EF80186819781092E000CAA0BBA
:10859000BB0B26013701480E591E6A1E7B1EF7FCD5
:1085A00005C0B7FD07C077FE05C067CFB7FF02C0A3
:1085B00077FE63CFA8E1B0E0A30192010E945E6361
:1085C0006B017C0145284628472841F00E94196329
:1085D000283131054105510509F04FCFF80184815B
:1085E0009581092E000CAA0BBB0B26013701480E02
:1085F000591E6A1E7B1EF7FC05C0B7FD07C077FE3B
:1086000005C03BCFB7FF02C077FE37CFACE3B0E089
:10861000A30192010E945E636B017C0145284628FC
:10862000472841F00E9419632C333105410551055B
:1086300009F023CFF80182819381092E000CAA0B47
:10864000BB0B26013701480E591E6A1E7B1EF7FC24
:1086500005C0B7FD07C077FE05C00FCFB7FF02C04A
:1086600077FE0BCFACE3B0E0A30192010E945E6302
:108670006B017C0145284628472841F00E94196378
:108680002C3331054105510509F0F7CEF801408141
:108690005181052E000C660B770BD701C601840FA4
:1086A000951FA61FB71F89839A83AB83BC83F7FCF2
:1086B00005C077FD07C0B7FF05C0DFCE77FF02C05A
:1086C000B7FFDBCEAB28F1F14091E8025091E9020F
:1086D0006091EA027091EB02840F951FA61FB71FED
:1086E00089839A83AB83BC83CE0101960E94A44BFD
:1086F000009709F4C2CEF8012089318912161306B9
:1087000044F0232B31F1FC01208931891216130624
:1087100004F549815A816B817C818091EC029091B2
:10872000ED02A091EE02B091EF02840F951FA61FFB
:10873000B71F89839A83AB83BC83CE0101960E94C5
:10874000A44B07C0CE0101960E940C42009709F489
:1087500094CE22E1FC01D80101900D922A95E1F717
:1087600069817A818B819C810F900F900F900F907F
:10877000DF91CF911F910F91FF90EF90DF90CF90FD
:10878000BF90AF907F906F905F904F90089561E0A1
:1087900070E00C94184260E070E00C941842CF92A4
:1087A000DF92EF92FF92CF93DF93EC01C0902C0900
:1087B000D0902D09E0902E09F0902F090E94DD50F5
:1087C0006C0D7D1D8E1D9F1D209721F06883798380
:1087D0008A839B83DF91CF91FF90EF90DF90CF90C2
:1087E00008958F929F92AF92BF92CF92DF92EF92B5
:1087F000FF920F931F93CF93DF937C018091F00240
:108800009091F102892B11F480E0ADC1D7011A9645
:108810000D911C911B978091FA029091FB02081711
:10882000190741F48091F2029091F3020817190799
:1088300009F41FC16801B3E0CB22DD24C114D104C7
:1088400049F48091D2029091D3024C01EFEF8E1A3D
:108850009E0A08C08091B8029091B9024C01FFEFC6
:108860008F1A9F0A9801265431098DE691E0289FBE
:10887000E001299FD00D389FD00D1124580121E02F
:10888000A21AB108B594A794B594A794BE01680D37
:10889000791D6A0D7B1DCB01770FAA0BBB0BBC01A9
:1088A000CD016D5071098109910927E030E040E068
:1088B00050E00E94196316161706180619061CF0D8
:1088C0002CE130E002C023E230E0C901861B970BA7
:1088D000880D991DC114D10441F42091D402309126
:1088E000D5022817390744F040C12091BA023091CF
:1088F000BB02281739070CF507979093FD02809368
:10890000FC0280E09DEDADE6B0E08093FE02909326
:10891000FF02A0930003B09301031093FB020093A6
:10892000FA02C114D104E9F4E091E002F091E1020D
:108930004F018FEF881A980A1CC09093FD02809314
:10894000FC0280E09DEDADE6B0E08093FE029093E6
:10895000FF02A0930003B09301031093FB02009366
:10896000FA02E091C602F091C7024F01AFEF8A1AF6
:108970009A0AC80DD91DCA0DDB1DCE01DD0FAA0B49
:10898000BB0BBC01CD016D5071098109910927E034
:1089900030E040E050E00E941963161617061806F2
:1089A00019061CF0ECE1F0E002C0E3E2F0E0E61BA7
:1089B000F70BE80DF91DCD2829F48091E202909182
:1089C000E30204C08091C8029091C9028E179F07EC
:1089D0000CF43797F093F502E093F4022091EC0247
:1089E0003091ED024091EE025091EF02A8EEB3E01B
:1089F0000E945E634B015C01BDED9B0EBDE6AB1EAC
:108A0000B11CB7FE0FC0DC01CB01975CAB46BA4F7F
:108A10008093F6029093F702A093F802B093F902C4
:108A200031971FC081142CE5920626E2A20625E0AC
:108A3000B2064CF48092F6029092F702A092F802ED
:108A4000B092F90212C0DC01CB019F57A84BB44091
:108A50008093F6029093F702A093F802B093F90284
:108A60003196F093F502E093F4021093F302009331
:108A7000F202C091FC02D091FD028091F40290912B
:108A8000F502D7011E96ED91FC911F97C817D907E3
:108A90007CF4EC17FD070CF4B7CE8E179F070CF48F
:108AA000B3CECE17DF079CF4E817F90784F45AC059
:108AB000E817F9070CF456C0CE17DF070CF452C0C4
:108AC0008E179F0724F4EC17FD070CF49DCED701F9
:108AD00012968D919C91139714964D915C911597D8
:108AE000CD90DC900D2C000CEE08FF082CE330E05C
:108AF000DC010E945763C60ED71EE81EF91E20E156
:108B00003EE0DA010E945763A7019601260F371F46
:108B1000481F591FA8EEB3E00E945E6351E040E099
:108B2000CE17DF0771F40091FE021091FF02209131
:108B300000033091010360177107820793077CF4EB
:108B40000DC00091F6021091F7022091F8023091C9
:108B5000F90260177107820793070CF050E0852F28
:108B6000942F18C081E090E015C09093FD0280938F
:108B7000FC0280E09DEDADE6B0E08093FE029093B4
:108B8000FF02A0930003B09301031093FB02009334
:108B9000FA02CACEDF91CF911F910F91FF90EF9013
:108BA000DF90CF90BF90AF909F908F9008950F93DC
:108BB0001F93CF93DF93689F8001699F100D789F6B
:108BC000100D1124C8010E94F345EC01009729F013
:108BD000A80160E070E00E942765CE01DF91CF918F
:108BE0001F910F910895BC0181EA99E00E94B34B57
:108BF000009731F42CE030E03093A00920939F09D6
:108C00000895BC0181EA99E00C941B4CEF92FF920D
:108C10000F931F93CF93DF937C01EC010990002009
:108C2000E9F7C81BD90BCE010E94F3458C010097D0
:108C300021F0AE01B7010E941E65C801DF91CF91FE
:108C40001F910F91FF90EF900895CF92DF92EF92D6
:108C5000FF920F931F93CF93DF938C017B016A01E7
:108C6000E901C131D10544F040E150E0B601C7014E
:108C7000F80119956097F5CF1C161D066CF4AE012E
:108C8000B601C701F801DF91CF911F910F91FF90BD
:108C9000EF90DF90CF901994DF91CF911F910F91BA
:108CA000FF90EF90DF90CF900895DB01ED91FC9164
:108CB000119783FF09C0CF0104968D939C93608127
:108CC000718182819381089586FF09C0CF01029648
:108CD0008D939C936081718180E090E00895CF0135
:108CE00002968D939C9360817181072E000C880BF6
:108CF000990B08952F923F924F925F926F927F92BD
:108D00008F929F92AF92BF92CF92DF92EF92FF929B
:108D10000F931F93CF93DF93CDB7DEB7A6970FB610
:108D2000F894DEBF0FBECDBF9DA38CA37BA36AA327
:108D300058A34F8F59011B8F0A8F212C312CCE0144
:108D400001962C01DE015996BD8FAC8FF5017F0194
:108D5000BFEFEB1AFB0AD080DD2029F025E2D21606
:108D600011F0F701F4CF8F010A191B0949F0A8018E
:108D7000B5018F8D98A1ECA1FDA11995200E311E92
:108D8000DD2009F4CCC2D701198EEA8DFB8D30E0CD
:108D900050E040E0EE24EA94FE2C612C712C1E8EF3
:108DA0005D012FEFA21AB20A1C9119A3103229F407
:108DB000411107C051E040E204C01B3221F451E0F0
:108DC0004BE2D501EDCF1D3221F46E8D64606E8FC4
:108DD000F8CF133219F48E8D816017C0103321F44F
:108DE0009E8D90619E8FEDCF1C3689F411968C91EB
:108DF00011978C3641F42E8D20622E8F5D0162E03A
:108E0000A60EB11CDECF8E8D88608E8FDACF1A371A
:108E1000C1F21A3279F4CF0102966080718077FE38
:108E200006C0AE8DA460AE8F719461947108FC0190
:108E300031E0C7CF1E32A9F511968C9111978A3275
:108E400021F0C501E12CF12C12C05D0122E0A20E3F
:108E5000B11CCF010296E080F180F7FE06C0FC0154
:108E600031E0EE24EA94FE2CACCF31E018C05C0176
:108E7000DC012C91019660ED620F6A3078F4AAE073
:108E8000AE9DB001AF9D700D1124E22E220FFF08A0
:108E9000B0E3EB1AF108E60EF71EE9CFCF01FC01B3
:108EA00090CF8FEC810F8930E0F4612E712CB0E30C
:108EB0006B1A7108D5015D012D9180ED820F8A300A
:108EC00008F07FCF6AE0669DC001679D900D112478
:108ED000622E220F770820E3621A7108680E791E4D
:108EE000EACF5111498F332311F0FB8FEA8F1836E7
:108EF000ACF415360CF081C11035B1F13CF41534E9
:108F000009F47BC1173409F478C18DC1133619F106
:108F10000CF06BC0183509F40DC185C1103709F488
:108F200009C13CF4193609F460C01F3609F4B3C016
:108F30007AC1153709F455C0183709F4FBC0133747
:108F400009F071C1EA8DFB8DCF0102969B8F8A8F4C
:108F5000008111811EC0EA8DFB8DCF0102969B8F8F
:108F60008A8F8081898363C1EA8DFB8DCF01029650
:108F70009B8F8A8FC080D180C114D10471F0C6014B
:108F80000E94FB6401960E94F3458C01B6010E9489
:108F9000F4640115110529F402C063E769A30FE623
:108FA00018E08FEFE816F80679F0A70160E070E0AE
:108FB000C8010E940465009779F0801B910B8E1503
:108FC0009F0554F47C0108C0F80101900020E9F7E6
:108FD00031977F01E01AF10A198E6701E12CF12C1B
:108FE0002FC1198E9E8D90649E8FAE8DA5FF08C0F7
:108FF0008A8D9B8D08969B8F8A8F65E375E0A4C050
:10900000BE01665E7F4FBE8D8B2F90E00E9455465D
:10901000153759F097FF09C0909580957095619527
:109020007F4F8F4F9F4F2DE2298FEFEFEE16FE06F9
:1090300069F0FE8DFF7EFE8F61157105810591053A
:1090400051F4E114F10409F44AC00AC06115710534
:109050008105910529F06A3071058105910530F48B
:10906000605D688F8E01085E1F4F61C08E01075ED4
:109070001F4F2AE030E040E050E00E94F762605D60
:10908000D8016E938D01B901CA0161157105810581
:10909000910579F74CC0BE8DB5FF08C08A8D9B8DB8
:1090A00008969B8F8A8F62E375E04EC0BE01665EB4
:1090B0007F4FEE8D8E2F90E00E945546198EFFEF68
:1090C000EF16FF0681F02E8D2F7E2E8F6115710514
:1090D0008105910571F4E114F10409F019C18E01C3
:1090E000075E1F4F24C0611571058105910509F4C4
:1090F0000FC18E01075E1F4F262F2770205DD801FC
:109100002E938D01E3E09695879577956795EA957F
:10911000D1F7611571058105910571F7BE8DB0FF1D
:1091200006C0203321F0F80180E382938F01CC8CBC
:10913000DD8C60C0EE8DE5FF0EC08A8D9B8D08969C
:109140009B8F8A8F6FE275E0C2010E94F46452E047
:10915000C52ED12C64C0103789F4EA8DFB8DCF0168
:1091600002969B8F8A8F40815181BA0180E090E006
:10917000FE8DF160FE8F28E729A308C0BE01665E60
:109180007F4FAE8D8A2F90E00E945546198EBFEF1B
:10919000EB16FB0619F0EE8DEF7EEE8FF9A1F83796
:1091A00019F428E435E002C028E335E08E01075EBB
:1091B0001F4F6801FB01EF70FF27E20FF31FE491DF
:1091C000D801EE938D0144E0969587957795679544
:1091D0004A95D1F7611571058105910559F7BE8D45
:1091E000B0FF08C0F801319729A12083319780E3AF
:1091F00080838F01C01AD10A23C08A8D9B8D04966B
:109200009B8F8A8F6CE275E0C2010E94F464F201C8
:1092100001900020E9F731976F01C418D508E12CBF
:10922000F12C82010DC0112309F479C01983198E24
:10923000CC24C394D12CE12CF12C8E010F5F1F4F55
:109240004701EC14FD040CF44601898D882319F0C4
:109250006FEF861A960A8E8D84718EA381110BC0D2
:1092600093012819390948E655E06F8D78A18AA144
:109270009BA10E942546898D882351F041E050E052
:10928000BE01675E7F4F8F8D98A1ECA1FDA119955E
:10929000FEA1F03159F493012819390948E555E048
:1092A0006F8D78A18AA19BA10E94254697012C1958
:1092B0003D0948E555E06F8D78A18AA19BA10E94E8
:1092C0002546C114D10439F0A601B8018F8D98A1AB
:1092D000ECA1FDA11995F9A1F03519F4C8010E947E
:1092E00001462E8D22FF0BC093012819390948E64B
:1092F00055E06F8D78A18AA19BA10E942546681434
:1093000079041CF0260C371C21CD280C391C1ECDED
:1093100080E3888F20E38E01085E1F4FFFCEC101DE
:10932000A6960FB6F894DEBF0FBECDBFDF91CF91EA
:109330001F910F91FF90EF90DF90CF90BF90AF9073
:109340009F908F907F906F905F904F903F902F9065
:1093500008958830910538F089E090E09093A00955
:1093600080939F091AC0880F991FFC01E45EF64F95
:1093700080819181009781F3DC01ED91FC9111973F
:10938000309729F41796ED91FC91189705C0018C40
:10939000F28DE02D309709F019948FEF9FEF08952B
:1093A00088309105C0F4880F991FFC01E45EF64FE8
:1093B00080819181009779F0DC01ED91FC9111970A
:1093C000309729F41996ED91FC911A9703C0038CFC
:1093D000F48DE02D199489E090E09093A00980939A
:1093E0009F098FEF9FEF08950F931F93CF93DF9304
:1093F0001F92CDB7DEB7182F092FFB01898341E0FB
:1094000050E0BE016F5F7F4F808191810E94A9492A
:10941000019711F01FEF0FEF812F902F0F90DF9129
:10942000CF911F910F910895DB01FC010190002065
:10943000E9F73197AF01481B590BBC018D919C9105
:109440000C94A9498F929F92AF92BF92CF92DF92D4
:10945000EF92FF920F931F93CF93DF9300D01F9251
:10946000CDB7DEB78B01FC014081518162817381F0
:109470006A017B01F1E8CF1AF4EFDF0AF3E0EF0AAB
:10948000F1082EEFC21626E1D20628EFE2062FE7FA
:10949000F20608F041C08091E8029091E902A091A3
:1094A000EA02B091EB02481B590B6A0B7B0B498314
:1094B0005A836B837C83B801CE0101960E94F840E9
:1094C0008091F0029091F102892B09F42AC1C80120
:1094D0000E94F143892B09F424C189819A81AB81CF
:1094E000BC814091EC025091ED026091EE027091CE
:1094F000EF02841B950BA60BB70B89839A83AB8372
:10950000BC83B801CE0101960E94F84081E090E052
:10951000F801918B808B05C1B8010E94F840C80109
:109520000E94F1434091E8025091E9026091EA0201
:109530007091EB02F801C080D1800D2C000CEE0878
:10954000FF08892B89F08091EC029091ED02A091A7
:10955000EE02B091EF02840F951FA61FB71FC81A25
:10956000D90AEA0AFB0A04C0C41AD50AE60AF70AAD
:10957000C701B6012CE330E040E050E00E941963DF
:1095800097FD04C0F801718360830AC0645C7F4F5B
:10959000F80171836083FCE3CF1AD108E108F10878
:1095A0008CE3882E912CA12CB12CC701B601A5010A
:1095B00094010E941963F801C280D3800D2C000C25
:1095C000EE08FF08C20ED31EE41EF51EC701B60149
:1095D000A50194010E94196397FD04C0F8017383EB
:1095E00062830AC0645C7F4FF80173836283FCE38B
:1095F000CF1AD108E108F108C701B6012CE330E029
:1096000040E050E00E941963F801C480D5800D2C21
:10961000000CEE08FF08C20ED31EE41EF51EC701A3
:10962000B60128E130E040E050E00E94196397FD68
:1096300004C0F801758364830AC0685E7F4FF80137
:1096400075836483F8E1CF1AD108E108F108C701F6
:10965000B60128E130E040E050E00E941963690162
:109660007A011216130614061506ECF4F801648547
:109670007585CB01770FAA0BBB0BBC01CD01620F27
:10968000731F841F951F27E030E040E050E00E94E8
:109690001963F80175876487868197818C0D9D1DFC
:1096A0009783868338C02115310541055105C9F1DD
:1096B000F80164857585695F7F4FCB01770FAA0B31
:1096C000BB0BBC01CD01620F731F841F951F27E0E8
:1096D00030E040E050E00E941963F801758764872C
:1096E000868197818C0D9D1D978386831816190698
:1096F0008CF04F96978386838CE691E097878687D8
:109700008BE090E09187808782859385019793878E
:10971000828707C0F80186859785C80ED91ED7862F
:10972000C68680E090E00F900F900F900F90DF9131
:10973000CF911F910F91FF90EF90DF90CF90BF904E
:10974000AF909F908F9008956DE879E00E94224A33
:10975000892B19F48DE899E0089580E090E0089550
:1097600086E798E00895CF93DF93EC016E5F7F4F1B
:109770006430710510F464E070E06F5F7F4F6E7FBE
:10978000E881F98130E020E0A0E0B0E03097C9F056
:10979000808191818617970770F0109731F04D9175
:1097A0005C9111978417950730F46817790771F069
:1097B0003C2F2D2FDF01EF0122960280F381E02D57
:1097C000E5CF1097F9F0C32FD22FFD018081918151
:1097D000861B970B228133818430910578F0DF015D
:1097E000A60FB71F11969C938E9313963C932E93BE
:1097F000129771836083B983A88302C03983288359
:10980000DF011296CD01DF91CF9108950F931F9341
:10981000CF93DF938B010E94B34BEC01009729F0AB
:10982000A80160E070E00E942765CE01DF91CF9132
:109830001F910F910895CF93DF93EC01611571058E
:1098400009F454C0FB013297A881B981109709F43B
:1098500053C08D919C9111979C012A0F3B1FE217D9
:10986000F307F9F420813181820F931F11969C93A5
:109870008E931296ED91FC9113979D01280F391F3D
:10988000E217F307E9F520813181820F931F1196CA
:109890009C938E938281938113969C938E931297BF
:1098A0002FC0EA17FB07C0F4F983E88320813181D8
:1098B000AF01420F531FA417B50759F4280F391FE2
:1098C0003183208312968D919C9113979383828389
:1098D00017C0B383A28314C0E217F30750F0ED0161
:1098E000229612960D90BC91A02DB0CF8DEF9FEFD8
:1098F00009C08FEF9FEF06C013821282F983E883BD
:1099000080E090E0DF91CF910895FB013196EE7FEA
:10991000460F571F4E1B5F0B4E7F41935193BF0164
:109920000C941B4CDC01ED91FC9180E090E03097B1
:1099300051F02081318122503109820F931F028022
:10994000F381E02DF4CF0895CF93DF93FC01708F66
:10995000678B158214820FB6F8940F92EB01A881E1
:10996000B981AF3FDFEFBD0741F484819581019656
:1099700095838483A0E0B0E016C01097A1F00F900B
:109980000FBE828952969C915297891748F0BD016B
:109990006E5F7F4F12960D90BC91A02D109791F79E
:1099A0000FB6F8940F92B383A283DB011196FC9358
:1099B000EE93A281B3811097A1F014968D919C91A2
:1099C0001597892B71F014962D913C9115978481F0
:1099D0009581820F931F9583848315961C921E9206
:1099E00014970F900FBEDF91CF910895CF93DF931F
:1099F000FC010FB6F8940F92EB01A881B9810F908A
:109A00000FBEAF3FDFEFBD0769F1109759F1AE17F9
:109A1000BF0701F50FB6F8940F9282819381DB01A5
:109A200011969C938E9384819581892B61F0A281FC
:109A3000B381109731F08481958115969C938E9314
:109A40001497158214820F900FBE13821282108E0B
:109A5000178A08C0BD016E5F7F4F12960D90BC91B2
:109A6000A02DD3CFDF91CF910895CF93DF93C091F5
:109A7000A309D091A409209711F10FB6F8940F9281
:109A80008C819D810F900FBE892BA9F08F89988DB5
:109A90000FB6F8940F922C813D81215031093D83FE
:109AA0002C830F900FBEFC01208131812F3F3F4F4F
:109AB00011F00E94D4510990D881C02DDCCF0E94B2
:109AC000814FE091A709F091A8098091A509909193
:109AD000A609E817F90761F08785813011F482E063
:109AE00087870FB6F8940F920E9439550F900FBEDA
:109AF000DF91CF910895CB01FB01168A158A22E0F0
:109B0000278765EA79E00C94A44C8091A70990918D
:109B1000A809FC0122813381232B61F065EA79E0F9
:109B20000E94F64C65EA79E08091A7099091A80916
:109B30000E94A44C0C94354DE091A909F091AA091A
:109B4000309751F06389748981EA99E00E941B4C37
:109B50001092AA091092A9090895CF93DF93C0919A
:109B6000A309D091A4090E949C4D8091A7099091CE
:109B7000A809E3EAF9E0209769F0C817D90729F4A2
:109B8000888199819183808305C0FE010990D881E5
:109B9000C02DF1CF8091A7099091A8099093AA09AF
:109BA0008093A909DF91CF910895CF93DF93C82FB8
:109BB0008091A7099091A809FC01D28965EA79E012
:109BC0000E94F64C8091A7099091A809FC01C28BD4
:109BD000CF3F29F065EA79E00E94A44C02C00E94C0
:109BE000AD4DE091A709F091A8098091A509909148
:109BF000A609E817F90719F481E0878709C082E010
:109C000087870FB6F8940F920E9439550F900FBEB8
:109C10008D2FDF91CF910895809140099091410956
:109C2000A0914209B09143090196A11DB11D8093F5
:109C3000400990934109A0934209B0934309409190
:109C40003C0950913D0960913E0970913F09809116
:109C5000340990913509A0913609B0913709840FE4
:109C6000951FA61FB71F80933C0990933D09A093B1
:109C70003E09B0933F0980913C0990913D09A09124
:109C80003E09B0913F0981349244AF40B1053CF1A7
:109C90008091380990913909A0913A09B0913B0916
:109CA0000196A11DB11D8093380990933909A093A5
:109CB0003A09B0933B0980913C0990913D09A091EC
:109CC0003E09B0913F0980549244AF40B10980935E
:109CD0003C0990933D09A0933E09B0933F09089534
:109CE000CF92DF92EF92FF929B01AC01A091AD0960
:109CF000B091AE090E945E63C72ED82EE92EFF24D4
:109D000041E3C416D104E104F10430F180E3C81A40
:109D1000D108E108F108D701C60120E030E0009742
:109D200041E0A407B10528F0F9013197F1F7119747
:109D3000F6CF970144275527A0E0B0E00E946C635E
:109D4000C60ED71EE81EF91EC114D104E104F104A9
:109D500019F0C6010197F1F7FF90EF90DF90CF90D7
:109D600008958CE09EE40E9437560E945B569B014A
:109D7000AC0160E472E48FE090E00E94F76220930F
:109D80003409309335094093360950933709E0E799
:109D9000F0E08081826080838FEA93E09093AE0947
:109DA0008093AD090895CF93C82FCC2341F068EE7E
:109DB00073E080E090E00E94704EC150F6CFCF91EA
:109DC00008950F931F93FC0113821282A091AB0997
:109DD000B091AC09109741F140855185628573853A
:109DE00018960D911D912D913C911B97401751078D
:109DF0006207730758F4041B150B260B370B1896D4
:109E00000D931D932D933C931B970EC0401B510B3C
:109E1000620B730B4087518762877387B383A2837A
:109E20000D90BC91A02DD6CFB183A083109721F0C7
:109E30001396FC93EE931297A281B381109719F0B9
:109E4000ED93FC9304C0F093AC09E093AB091F9130
:109E50000F9108950F931F93CF93DF93FC0114820A
:109E60001582168217821586148640855185628573
:109E70007385411551056105710581F1C281D38159
:109E800080819181209719F09983888304C09093F1
:109E9000AC098093AB09A081B1811097A1F0139612
:109EA000DC93CE93129718960D911D912D913C91B4
:109EB0001B97400F511F621F731F18964D935D93A0
:109EC0006D937C931B971086118612861386CF01A3
:109ED000DF91CF911F910F910C94E14EDF91CF91C3
:109EE0001F910F9108950FB6F8940F926091400959
:109EF0007091410980914209909143090F900FBEE2
:109F00000895CF92DF92EF92FF92CF93DF930E945A
:109F1000734FC0904809D0904909E0904A09F090E9
:109F20004B099B01AC012C193D094E095F096901E0
:109F30007A01609348097093490980934A09909384
:109F40004B09C091AB09D091AC09209709F458C0D6
:109F5000C114D104E104F10409F452C08885998543
:109F6000AA85BB85C816D906EA06FB0660F48C19DB
:109F70009D09AE09BF0988879987AA87BB87C12C2D
:109F8000D12C760108C0C81AD90AEA0AFB0A188639
:109F900019861A861B8688859985AA85BB85892B93
:109FA0008A2B8B2B71F6EC85FD85309721F06E8521
:109FB0007F85CE011995E091AB09F091AC09019034
:109FC000F081E02DF093AC09E093AB09309711F0EC
:109FD000138212828C819D81AE81BF81888799878F
:109FE000AA87BB87892B8A2B8B2B31F4BE0181EA90
:109FF00099E00E941B4CA5CFCE010E94E14EA1CF5B
:10A00000DF91CF91FF90EF90DF90CF9008954F9226
:10A010005F926F927F928F929F92AF92BF92CF92F8
:10A02000DF92EF92FF920F93CF93DF934B015C018E
:10A030006A01790160E170E081EA99E00E94B34B26
:10A04000EC01892B49F10E94734F409048095090D0
:10A05000490960904A0970904B09A501940124199F
:10A06000350946095709DC01CB01820F931FA41F54
:10A07000B51F88879987AA87BB8700FF05C01C8208
:10A080001D821E821F8204C08C829D82AE82BF828E
:10A09000DD86CC86FF86EE86CE01DF91CF910F91D3
:10A0A000FF90EF90DF90CF90BF90AF909F908F90F8
:10A0B0007F906F905F904F9008950F93CF93DF93B1
:10A0C0000E940750EC01009711F00E94E14ECE0172
:10A0D000DF91CF910F9108950F93CF93DF9300D02D
:10A0E0001F92CDB7DEB72B833C8349835A830E94EE
:10A0F00060562B813C8149815A810E945D500F90AE
:10A100000F900F900F90DF91CF910F910895CF9204
:10A11000DF92EF92FF920F93CF93DF936B017C015D
:10A12000672B682B692B09F43FC065EA79E08091C1
:10A13000A7099091A8090E94F64CC091A709D09157
:10A14000A80983E08F8701E09E014BE75DE4C7012A
:10A15000B6010E946C509E8B8D8B892B49F0DF914C
:10A16000CF910F91FF90EF90DF90CF900C94354DF1
:10A17000E091A709F091A80985EA99E0908F878B73
:10A180008091A5099091A6099383828381E08787B6
:10A19000F093A609E093A509DF91CF910F91FF906D
:10A1A000EF90DF90CF900895DF91CF910F91FF90C6
:10A1B000EF90DF90CF900C94854D609138097091AD
:10A1C000390980913A0990913B0908958F929F92A5
:10A1D000AF92BF92CF92DF92EF92FF92E8E3F9E065
:10A1E000208131814281538184809580A680B7800F
:10A1F000A8EEB3E00E945E636B017C01C501B4016F
:10A2000028EE33E040E050E00E941963C701B60138
:10A21000620F731F841F951FFF90EF90DF90CF9008
:10A22000BF90AF909F908F90089560E070E081EEB6
:10A2300090E00895CF93DF93FB010FB6F8940F924F
:10A24000C081D1810F900FBECF3F2FEFD207A9F170
:10A25000209799F14D895E892A813B8148175907DA
:10A2600041F50FB6F8940F92318320838C819D8144
:10A27000892B89F0AA81BB81109739F08C819D814F
:10A2800015969C938E93149704C08FEF9FEF918344
:10A2900080831D821C820F900FBE82E08F8765EA4B
:10A2A00079E0CE010E94A44C8FEF9FEF9E8B8D8BA7
:10A2B00004C0FE013296E901CBCFDF91CF91089522
:10A2C0008F929F92AF92BF92EF92FF920F93CF9394
:10A2D000DF93EC014A015B010FB6F8940F9288817D
:10A2E00099810F900FBE019651F40FB6F8940F921A
:10A2F000198218820F900FBE0E94854D39C065EA01
:10A3000079E08091A7099091A8090E94F64CBE01BE
:10A310008091A7099091A8090E94A44CE090A709F8
:10A32000F090A80983E0F701878781149104A104C4
:10A33000B10461F001E09E014AE151E5C501B401BB
:10A340000E946C50F701968B858B03C0F701168A2B
:10A35000158A0E94354DE091A709F091A8098589D9
:10A360009689019629F4168A158A8FEF9FEF02C00D
:10A3700080E090E0DF91CF910F91FF90EF90BF9040
:10A38000AF909F908F9008950FB6F8940F92FC01B4
:10A39000208131812F3F3F4F19F4FC01118210823F
:10A3A0000F900FBE0C946051CF93DF93FC010FB65A
:10A3B000F8940F92C081D1810F900FBECF3F8FEFE5
:10A3C000D80709F43BC0209781F10FB6F8940F929B
:10A3D0008A819B81918380838C819D81892B89F0E7
:10A3E000AA81BB81109739F08C819D8115969C9331
:10A3F0008E93149704C08FEF9FEF918380831D820B
:10A400001C820F900FBE8D899E89009721F00E94BB
:10A410002A4F1E8A1D8A82E08F8765EA79E0CE0185
:10A420000E94A44C81E090E00BC00FB6F8940F920C
:10A430008FEF9FEF918380830F900FBE80E090E0BD
:10A44000DF91CF910895CF93DF931F921F92CDB7E5
:10A45000DEB70E94D45189839A830E94854D8981F9
:10A460009A810F900F90DF91CF9108950F931F93D2
:10A47000CF93DF938C010FB6F8940F92FC0180818B
:10A4800091810F900FBE8F3FFFEF9F0759F40FB6DA
:10A49000F8940F92F801118210820F900FBEC0E065
:10A4A000D0E015C0C0E0D0E0892B89F0C8010E943F
:10A4B000D451C80FD91F0FB6F8940F92F8018081BC
:10A4C00091810F900FBE01978E3F9F4F78F3CE0181
:10A4D000DF91CF911F910F910895CF93DF931F923A
:10A4E0001F92CDB7DEB70E94365289839A830E94AD
:10A4F000854D89819A810F900F90DF91CF910895BA
:10A500000F931F93CF93DF938C01C0914C09D0918F
:10A510004D09209759F0B801CE0102960E94576567
:10A52000892B21F00990D881C02DF3CFCE01DF9186
:10A53000CF911F910F910895CF93DF93EC01611597
:10A54000710511F07D876C8741114E87CE0102960F
:10A550000E948052892B19F08FEF9FEF16C0EB8974
:10A56000FC89309769F480914C0990914D09998349
:10A570008883D0934D09C0934C0980E090E005C0DA
:10A58000CE011995892B79F3E7CFDF91CF9108950B
:10A5900043E150E06FEA79E080E090E00E942755C7
:10A5A000892B71F48091AF09833151F442E050E07E
:10A5B0006EE778E080EB99E00E941165009741F02A
:10A5C00061E878E082EB99E00E9460658FEF9FEF91
:10A5D0000895EF92FF920F931F93CF93DF938C0117
:10A5E0007B01EA01640F751F81EA99E00E94B34B79
:10A5F000009731F4F801118210828FEF9FEF09C0AC
:10A60000C80FD91FF801D183C083F382E28280E0B2
:10A6100090E0DF91CF911F910F91FF90EF900895FF
:10A62000CF93DF93EC018A81982F977029F08150A6
:10A630008A83DF91CF91089584FF07C06B817C816D
:10A640006E7F81EA99E00E941B4C8A8185FF06C0DB
:10A650006F81788581EA99E00E941B4C8A8186FF90
:10A6600006C06B857C8581EA99E00E941B4C8A813B
:10A6700087FF06C06F85788981EA99E00E941B4CAC
:10A680008B899C89009711F00E941053BE0181EACA
:10A6900099E0DF91CF910C941B4CCF92DF92EF9217
:10A6A000FF920F931F93CF93DF93EC01062F6A0164
:10A6B000862F807F803121F0162F209771F403C000
:10A6C000209789F410E165E170E081EA99E00E9449
:10A6D000064CEC01892B09F449C0103251F01034BA
:10A6E00069F0103181F47E0183E0E80EF11C10E185
:10A6F0000EC07E01E7E0EE0EF11C09C07E01FBE01A
:10A70000EF0EF11C04C07E018FE0E80EF11C8A817F
:10A710008123F70191F0828193818C159D054CF482
:10A72000608171816E7F81EA99E00E941B4CF70184
:10A7300004C0F701D382C28202C013821282F701E1
:10A7400082819381892B91F4402F50E04F70B601A4
:10A75000C7010E94E952892B31F0CE010E941053AB
:10A76000C0E0D0E003C08A81182B1A83CE01DF91AC
:10A77000CF911F910F91FF90EF90DF90CF900895B0
:10A78000AF92BF92CF92DF92EF92FF920F931F93FF
:10A79000CF93DF938C01C62EFC01828187708730B6
:10A7A00011F480EFC82E65E170E081EA99E00E9423
:10A7B000064CEC01009709F4B6C0F801A580B680FC
:10A7C000A114B10411F143815481C4FE15C041703C
:10A7D0005527B50103960E94E9527C01892BB9F4F3
:10A7E000F80163817481A5018B819C810E941E65A3
:10A7F0008A8180618A830BC05C834B83BE82AD8279
:10A80000E12CF12CDD24D39403C0E12CF12CD12CCC
:10A81000F801A184B284A114B10421F1E114F1047E
:10A8200009F5C5FE16C040E050E0B501CE0107961F
:10A830000E94E9527C01892BA9F4F8016781708597
:10A84000A5018F8198850E941E658A8180628A8316
:10A8500009C0F8018781908598878F83BA86A98679
:10A86000DD24D394F801A584B684A114B10421F1A8
:10A87000E114F10409F5C6FE16C040E050E0B50150
:10A88000CE010B960E94E9527C01892BA9F4F801B4
:10A8900063857485A5018B859C850E941E658A81D0
:10A8A00080648A8309C0F801838594859C878B879F
:10A8B000BE86AD86DD24D394F801A188B288A114A8
:10A8C000B10409F1EF2851F5C7FE15C040E050E092
:10A8D000B501CE010F960E94E952892BF9F4F801D7
:10A8E00067857089A5018F8598890E941E658A8178
:10A8F00080688A830AC0F80187859089988B8F8742
:10A90000BA8AA98A04C0EF2849F4DD2061F01C8BC3
:10A910000B8BF80182818F5F828305C0CE010E947C
:10A920001053C0E0D0E0CE01DF91CF911F910F9185
:10A93000FF90EF90DF90CF90BF90AF9008956F920F
:10A940007F928F929F92AF92BF92CF92DF92EF92BF
:10A95000FF920F931F93CF93DF9300D01F92CDB739
:10A96000DEB77C015B0140E050E0CE0101960E9421
:10A97000E952892B09F055C089809A80F7016785D3
:10A98000708941895289C4010E941E65F70181893D
:10A9900092899C838B8300811181C12CD12C01155C
:10A9A000110529F18B819C81F801418952899C0113
:10A9B000240F351FA216B306D4F0F8016080718011
:10A9C00067857089880D991D0E941E652B813C81C9
:10A9D000F80181899289820F931F9C838B83C80120
:10A9E0000E941053FFEFCF1ADF0A8301D8CFF7017F
:10A9F00011830083828187FF07C06785708981EAA0
:10AA000099E00E941B4C03C08068F7018283898112
:10AA10009A81F701908B87878B819C81928B818BA8
:10AA200002C0C12CD12CC6010F900F900F900F9037
:10AA3000DF91CF911F910F91FF90EF90DF90CF901A
:10AA4000BF90AF909F908F907F906F9008950C94DF
:10AA5000EC5A0C94F45A80E090E0089580E090E085
:10AA600008959F918F910F900BBE0F900FBE1F9076
:10AA70001895E091A709F091A8092F923F924F9263
:10AA80005F926F927F928F929F92AF92BF92CF927E
:10AA9000DF92EF92FF920F931F93CF93DF938DB7C7
:10AAA0009EB7918B808BE091A509F091A609F09358
:10AAB000A809E093A70981E08787808991898DBFE4
:10AAC0009EBFDF91CF911F910F91FF90EF90DF908C
:10AAD000CF90BF90AF909F908F907F906F905F903E
:10AAE0004F903F902F9008958F929F92BF92CF9258
:10AAF000DF92EF92FF920F931F93CF93DF931F92FA
:10AB00001F92CDB7DEB77C01062FB72E4901B901E0
:10AB1000675E7F4F81EA99E049835A830E94B34B75
:10AB200049815A81009709F490C0880E991E9401BA
:10AB300028503109B4016D517109D401169618E0FD
:10AB4000F70101900D921A95E1F7D4011E961C921F
:10AB50001E97F4017E975196FC93EE93509754966E
:10AB60009C938E935397EFEECE2EEEEBDE2EEDEA16
:10AB7000EE2EEEEDFE2EFC01C082D182E282F38247
:10AB8000C482D582E682F782C086D186E286F386C9
:10AB9000C486D586E686F78680E4F401828BD901E7
:10ABA00015961C9215971696BC92169717960C93AD
:10ABB000179780E813968C93139712961C9212970E
:10ABC00014961C92149711964C9311975C93FB0169
:10ABD000128A81E395E5938B848B8091A3099091F0
:10ABE000A409D40111969C938E939092A40980920B
:10ABF000A30982E01F968C931F9756961C921E9273
:10AC0000559758961C921E92579765EA79E0C401B1
:10AC10000E94A44CE091A709F091A809309721F473
:10AC20000FB6F8940F923FCF8091A5099091A60995
:10AC3000E817F90769F082E087870FB6F8940F925A
:10AC40000E9439550F900FBE03C080E090E001C014
:10AC5000C4010F900F90DF91CF911F910F91FF9042
:10AC6000EF90DF90CF90BF909F908F900895BC01A0
:10AC700080E090E0A1EEB0E080934E0990934F0900
:10AC8000A0935009B0935109E0E7F0E090819D7FD7
:10AC900090831092B20092E09093B00085E0809390
:10ACA000B10082E78093B30095BB40E050E08EE4B2
:10ACB00093E00C940B5D6AEE73E080E090E0089501
:10ACC000611520E872072EE38207910558F028EEFF
:10ACD00033E040E050E00E94F762AAEEB3E00E9449
:10ACE0005E630895AAEEB3E09B01AC010E945E632F
:10ACF00069517C4F8F4F9F4F28EE33E040E050E08A
:10AD00000E94F762CA01B9010895FB012091700009
:10AD10002270309170003D7F30937000803191053A
:10AD2000A9F02CF4009771F0019769F023C08231EB
:10AD3000910569F14CF18097E9F488E090E0918306
:10AD4000808315C020E082E087BB11C0B99B05C09D
:10AD500081E090E09183808302C0118210822223DF
:10AD6000B1F0808191818068918380830DC080E003
:10AD700090E002C08FEF9FEF222359F020917000E6
:10AD8000226020937000089580E090E0F7CF80E08B
:10AD900090E008951F920F920FB60F9211240BB6F8
:10ADA0000F922F933F934F935F936F937F938F9364
:10ADB0009F93AF93BF93EF93FF938EE493E00E9432
:10ADC000005DFF91EF91BF91AF919F918F917F9126
:10ADD0006F915F914F913F912F910F900BBE0F900C
:10ADE0000FBE0F901F9018950FB6F8940F9288EB36
:10ADF0008093C1000F900FBE08958091C20083FD23
:10AE000002C081E0089582E008952091540924FB56
:10AE1000882780F990E0A0E0B0E023FD826022FD69
:10AE2000846020915309222321F026FDA26027FD92
:10AE3000A860A1FFA160A3FFA46020915209222372
:10AE400011F0A06401C0A0682091C000BC01CD0138
:10AE500020FF02C08061089580620895CF92DF9242
:10AE6000EF92FF926B017C01809153098823D9F006
:10AE70000FB6F8940F92E0FE02C08F7B03C0E1FE94
:10AE800003C0806480935309E2FE04C0809153099B
:10AE90008F7705C0E3FE05C08091530980688093D9
:10AEA00053090F900FBEE6FE03C081E08093520964
:10AEB000E7FC10925209E4FE05C08091C000816059
:10AEC0008093C000E5FE05C08091C0008E7F809316
:10AED000C000C0FE05C0809154098F7E8093540944
:10AEE000C1FE05C080915409877F80935409C2FE3A
:10AEF00005C0809154098B7F809354090E940557A7
:10AF0000DC01CB01887F21E030E08C159D05AE058A
:10AF1000BF0511F420E030E088279927821B930BAE
:10AF2000FF90EF90DF90CF900895809153098111A9
:10AF300004C060E070E0CB01089560E270E080E062
:10AF400090E00895CF92DF92EF92FF926B017C0127
:10AF500065FF0BC08091530981110EC00FB6F894A4
:10AF60000F9281E48093530905C00FB6F8940F92B5
:10AF7000109253090F900FBE0E94955721E030E0C8
:10AF8000C616D706E806F90611F420E030E0882757
:10AF90009927821B930BFF90EF90DF90CF9008953D
:10AFA000E1ECF0E08081806280830895CF93DF93AD
:10AFB0000FB6F8940F92C1ECD0E088818F77888328
:10AFC00088818F7B888388818F7D88830F900FBED7
:10AFD0008AE00E94D34E88818F7E88838881877F14
:10AFE0008883DF91CF910895CF93C82F0E94D657C1
:10AFF000C13021F48091C200877F05C0C23029F49E
:10B000008091C20088608093C2000E94F4560E9422
:10B01000FD5621E030E0C81302C020E030E0882770
:10B020009927821B930BCF9108958F929F92AF9295
:10B03000BF92CF92DF92EF92FF92CF93DF93209156
:10B04000C4008091C50030E0E901D82B8091C20096
:10B0500086FD0AC08091C00081FD0CC020E1C22E97
:10B06000D12CE12CF12C0BC092E0C92ED12CE12C7B
:10B07000F12C05C088E0C82ED12CE12CF12C0E94C7
:10B0800015514B015C01CE01A0E0B0E09C01AD0187
:10B090002F5F3F4F4F4F5F4FC701B6010E94B36212
:10B0A0009B01AC01C501B4010E94F762CA01B9015C
:10B0B000DF91CF91FF90EF90DF90CF90BF90AF9056
:10B0C0009F908F900895CF93DF9300D01F92CDB7BC
:10B0D000DEB79B01AC0169833A834B835C830E949A
:10B0E000D6578091C20029813A814B815C8186FDCF
:10B0F00013C08091C00081FF08C072E0220F331F8F
:10B10000441F551F7A95D1F707C063E0220F331F04
:10B11000441F551F6A95D1F729833A834B835C837B
:10B120000E94155129813A814B815C810E94F7620E
:10B13000DA01C9010196A11DB11DB695A795979594
:10B1400087959C01215031092093C4003093C5009C
:10B150000E94F45680E090E00F900F900F900F90B7
:10B16000DF91CF91089540E050E060E070E08EED17
:10B1700093E00E940B5D40E050E060E070E084EE00
:10B1800093E00E940B5D80E090E00895FC01A281B5
:10B19000B38180915309982F9073B9F084FF07C051
:10B1A00083E18093C60080915309806406C081E1E9
:10B1B0008093C600809153098F7B809353098091BF
:10B1C00053098F7C80935309089587FF06C08091AF
:10B1D000C1008F7D8093C100089582859385892B5E
:10B1E00031F18285938501979387828780915209F7
:10B1F000882321F08091C100816003C08091C1004B
:10B200008E7F8093C1008D918093C6008681978147
:10B21000A817B90711F4A481B581B383A28322854D
:10B220003385848595852817390719F507C08091DE
:10B23000C1008F7D8093C10013861286A089B189D9
:10B24000109729F48FEF9FEF918B808B0DC0AF3F4C
:10B250008FEFB80749F014968D919C911597019640
:10B2600015969C938E93149762E0868997890C9427
:10B27000203D0895EF92FF921F93CF93DF93EC014F
:10B280009091C00080915409982B9093540910918B
:10B29000C600809153098823C1F0133149F480918D
:10B2A000C1008F7D8093C1008091530980680AC0DE
:10B2B000113159F48091C10080628093C100809166
:10B2C00053098F778093530955C02A853B8548855C
:10B2D00059852417350720F09860909354094AC087
:10B2E00079019FEFE91AF90A232BC1F4E889F9895A
:10B2F000309729F48FEF9FEF998B888B09C0EF3F30
:10B300008FEFF80729F084819581019695838483D6
:10B3100061E08E899F890E94203D18C08823B1F08A
:10B320002E853F85E216F30688F086FD0FC09091CA
:10B33000C00095FF08C083E18093C6008091530947
:10B340008F7D806401C0806280935309E881F98118
:10B35000CF010196998388831083288139818E815A
:10B360009F812817390721F48C819D8199838883D7
:10B37000FB86EA86DF91CF911F91FF90EF900895B1
:10B380008091C10082FD10C08091C20082FF06C082
:10B390008091C20081FD0AC087E008958091C200BB
:10B3A00081FD06C085E0089589E0089588E008954C
:10B3B00086E00895CF93C82F0E94D6578091C10090
:10B3C0008B7F8093C1008091C2008D7F8093C200EB
:10B3D0008091C2008B7F8093C200C730A9F030F407
:10B3E000C630B9F48091C200826011C0C83039F013
:10B3F000C93079F48091C10084608093C10080914C
:10B40000C20082608093C2008091C20084608093F9
:10B41000C2000E94F4560E94C05921E030E0C813D7
:10B4200002C020E030E088279927821B930BCF9140
:10B4300008959091C200892F807295FF07C0809176
:10B44000C20084FD02C082E0089581E00895CF9398
:10B45000C82F0E94D657C13081F030F0C230B9F405
:10B460008091C2008F7E0CC08091C2008F7E80933D
:10B47000C2008091C2008F7D08C08091C2008061AF
:10B480008093C2008091C20080628093C2000E94BB
:10B49000F4560E94195A21E030E0C81302C020E09F
:10B4A00030E088279927821B930BCF9108958091D4
:10B4B000C20086FF0BC06A9B02C083E001C081E02E
:10B4C0009091C20090FF09C0846008958091C000EF
:10B4D00081FF02C080E2089580E00895CF93C82FD5
:10B4E0000E94D657C0FF17C0C1FF02C06A9A01C0B0
:10B4F0006A988091C200C2FF02C0816001C08E7F45
:10B500008093C2008091C0008D7F8093C0008091A5
:10B51000C200806411C08091C000C5FF02C082607B
:10B5200001C08D7F8093C0008091C2008E7F809388
:10B53000C2008091C2008F7B8093C2000E94F456AB
:10B540000E94575A21E030E0C81302C020E030E0EA
:10B5500088279927821B930BCF91089580915309D7
:10B560008823D1F086FF18C00FB6F8940F929091FF
:10B57000C00095FF07C081E18093C6008091530908
:10B580008F7E01C0806180935309809153098F7928
:10B59000809353090F900FBE089541EA53E06AE388
:10B5A00079E58EED93E00E940B5D892B91F449E8DB
:10B5B00053E066EC78E584EE93E00E940B5D009723
:10B5C00051F040E050E060E070E08EED93E00E94CA
:10B5D0000B5D8FEF9FEF08959C01CB01B9010E9495
:10B5E000CA6580E090E008959C01CB01F999FECFF7
:10B5F000B9010E94DA6580E090E00895FB01209196
:10B60000C10020783091C1003F773093C100803174
:10B610009105B9F02CF4009771F0019769F027C0FB
:10B620008231910589F16CF1809709F580E190E014
:10B630009183808319C020E08091C6008091C6006C
:10B6400013C08091C00087FF05C081E090E0918326
:10B65000808302C0118210822223B1F08081918107
:10B660008068918380830DC080E090E002C08FEFFE
:10B670009FEF222359F02091C10020682093C10040
:10B68000089580E090E0F7CF80E090E008951F9269
:10B690000F920FB60F9211240BB60F922F933F9378
:10B6A0004F935F936F937F938F939F93AF93BF93CA
:10B6B000EF93FF938EED93E00E94005DFF91EF9179
:10B6C000BF91AF919F918F917F916F915F914F91BA
:10B6D0003F912F910F900BBE0F900FBE0F901F90B8
:10B6E0001895FB012091C10020723091C1003F7D6F
:10B6F0003093C1008131910579F12CF4009779F1F3
:10B70000409769F01FC08231910549F18097D1F4CB
:10B7100080E190E09183808380E090E015C080918B
:10B72000C00085FF05C081E090E09183808302C066
:10B7300011821082222399F0808191818068918307
:10B7400080830AC08FEF9FEF222359F02091C10020
:10B7500020622093C100089580E090E0F7CF80E060
:10B7600090E008951F920F920FB60F9211240BB61E
:10B770000F922F933F934F935F936F937F938F938A
:10B780009F93AF93BF93EF93FF9384EE93E00E9458
:10B79000005DFF91EF91BF91AF919F918F917F914C
:10B7A0006F915F914F913F912F910F900BBE0F9032
:10B7B0000FBE0F901F901895EF92FF920F931F935B
:10B7C000CF93DF938C01EB01EB80FC80C7010E96D9
:10B7D00098878F838D819E810E979A8789878EE0C7
:10B7E00090E09E838D83E091C209F091C309309768
:10B7F000B9F4F70184859585082E892F902D811540
:10B80000F8E09F07C1F086309840F9F4BE01C80106
:10B81000DF91CF911F910F91FF90EF900C948E5C70
:10B82000C8011995892B29F7DF91CF911F910F91AD
:10B83000FF90EF900895BE01C801DF91CF911F9155
:10B840000F91FF90EF900C942533CE01DF91CF91B3
:10B850001F910F91FF90EF900C9410538F929F9235
:10B86000AF92BF92CF92DF92EF92FF920F931F930E
:10B87000CF93DF936C01EB014A0189014EE050E068
:10B8800060E1C9010E944D53892BC9F1D80113967B
:10B89000ED90FC901497F601A784B088D701169616
:10B8A000F501359686E001900D928A95E1F78114B5
:10B8B000910441F086E0F401D70101900D928A9540
:10B8C000E1F707C046E050E06FEF70E0C7010E946B
:10B8D0002765BE01062E672F702DD7011D967C931C
:10B8E0006E931C97D5019196ED91FC919297B801BA
:10B8F000C6011995009729F0C8010E9410538FEFD7
:10B900009FEFDF91CF911F910F91FF90EF90DF900C
:10B91000CF90BF90AF909F908F900895CF92DF927D
:10B92000EF92FF920F931F93CF93DF937C018B01D4
:10B93000DB0119968D919C911A974C9758F4C80188
:10B94000DF91CF911F910F91FF90EF90DF90CF90FB
:10B950000C941053FB01C781D08588819981082EF2
:10B96000892F902D019759F78A819B81082E892F65
:10B97000902D8115984019F78C81863001F78D81C3
:10B980008430E9F6D7011F96ED91FC915097488DD0
:10B99000598D6A8D7B8D83859485A585B6854817DD
:10B9A00059076A077B0759F66E01B8E0CB0ED11C28
:10B9B0004E855F85688979899601C7010E94C138E3
:10B9C0008E819F81082E892F902D019709F0B7CF86
:10B9D0004E855F8568897989960182E090E00E94B2
:10B9E000103AEC01009709F4AACFBC01C7010E94EC
:10B9F0006E3A892B09F0A3CFCE010E9410539FCF3E
:10BA0000DC011296ED91FC911397309719F08D910E
:10BA10009C9119940895EF92FF920F931F93CF93E7
:10BA2000DF93EC018B017A01EC81FD81309731F0DD
:10BA300060E070E080E090E0199502C080E090E066
:10BA4000F982E8821B830A83DF91CF911F910F91C6
:10BA5000FF90EF900895AF92BF92CF92DF92EF9256
:10BA6000FF920F931F93CF93DF93EC017A010FB6F0
:10BA7000F8940F928A8D9B8D680F791F7B8F6A8F48
:10BA80000A8D1B8D0F900FBE6E0185E4C80ED11C70
:10BA90005E01A0E2AA0EB11CE016F106A8F4D601E0
:10BAA000ED91FC9119954C855D856E857F85C5016D
:10BAB0000E946051892B41F40FB6F8940F920A8DC1
:10BAC0001B8D0F900FBEE8CFC801DF91CF911F9162
:10BAD0000F91FF90EF90DF90CF90BF90AF900895BF
:10BAE000CF92DF92EF92FF920F931F93CF93DF934A
:10BAF000EC018B016A0179018C819D812885398552
:10BB00000FB6F8940F92198618860F900FBE26175D
:10BB1000370769F0232B11F00E940146011511052A
:10BB2000F9F0C8010E94F345009719F41CC0672B77
:10BB3000B9F09D838C83998388839B838A83800F4C
:10BB4000911F9F838E83DD86CC86FF86EE861B86C3
:10BB50001A860FB6F8940F92198708870F900FBEB8
:10BB600080E090E002C08FEF9FEFDF91CF911F91B7
:10BB70000F91FF90EF90DF90CF9008958F929F925A
:10BB8000AF92BF92CF92DF92EF92FF920F931F93EB
:10BB9000CF93DF93EC016B015A01490188819981B0
:10BBA000AA81BB8194FF18C07DA36CA35BA34AA3A9
:10BBB000FE01EB5BFF4F0190F081E02D19954C8564
:10BBC0005D856E857F85CE0180960E94C451009769
:10BBD00009F09BC0C50199C0288D398D232B09F42C
:10BBE00090C0672B99F440E050E060E070E0CE0137
:10BBF000DF91CF911F910F91FF90EF90DF90CF9049
:10BC0000BF90AF909F908F900C942B5D8C019D0105
:10BC100049E036952795179507954A95D1F7017014
:10BC200057E0B695A795979587955A95D1F7182F10
:10BC300011700FB6F8940F928A8D9B8D0F900FBEE6
:10BC400060E070E0E12CF12CEA14FB040CF045C03C
:10BC50004E8D5F8D9C01260F371F2417350768F026
:10BC60004C8D5D8DCE010E942B5D2C8D3D8D281756
:10BC7000390708F449C060E070E0F60181149104CE
:10BC800011F0449101C04081113041F44A3049F42F
:10BC90004DE012E0013059F402E009C0123009F41D
:10BCA00011E0FFEFCF1ADF0A2FEFE21AF20AE8895C
:10BCB000F9899F012F5F3F4F398B288B408348893B
:10BCC00059892E893F894217530721F42C893D89D0
:10BCD000398B288B6F5F7F4FB7CF61157105A1F04E
:10BCE0000FB6F8940F928A8D9B8D680F791F7B8F0A
:10BCF0006A8F0F900FBECB5BDF4FE881F9811995FA
:10BD000003C08FEF9FEF01C0C701DF91CF911F915B
:10BD10000F91FF90EF90DF90CF90BF90AF909F90EA
:10BD20008F9008950F931F93CF93DF93FC01C189E8
:10BD3000D289FE01EF5BFF4F0190F081E02D199554
:10BD40008C01892B49F4C35BDF4FE881F98160E006
:10BD500072EC81E090E01995C801DF91CF911F91BD
:10BD60000F910895AF92BF92CF92DF92EF92FF9220
:10BD70000F931F93CF93DF938B016A01DC01ED9149
:10BD8000FC91C189D28988819981AA81BB8193FF65
:10BD90000BC07DAF6CAF5BAF4AAFC95BDF4FE881D3
:10BDA000F9811995C601BBC068A979A9611571050A
:10BDB00019F48FEF9FEFB3C00115110571F42EA98F
:10BDC0003FA94CA95DA9CE0188960E94705DC95B10
:10BDD000DF4FE881F9811995A0C07E01B7E4EB0E31
:10BDE000F11C5E0128E3A20EB11C0FB6F8940F926D
:10BDF0004AA95BA90F900FBE4115510599F4D701CF
:10BE0000ED91FC911995488559856A857B85C50119
:10BE10000E946051892B09F080C088A999A9892BBB
:10BE200021F7C7CF888187FF3AC080E090E0E12CFE
:10BE3000F12CFE01E05CFF4F6AE0EC14FD0408F019
:10BE400050C08417950709F44EC0AAA5BBA59D0153
:10BE50002F5F3F4F3BA72AA72C91AAA4BBA4AEA556
:10BE6000BFA5AA16BB0621F4ACA5BDA5BBA7AAA772
:10BE700001962D3011F02A3049F43081332311F02E
:10BE80002313DBCF2083D8016C9303C01082D80129
:10BE90002C93BFEFEB1AFB0A0F5F1F4FCECF7A0137
:10BEA000C416D50608F47601F801C8018E0D9F1D51
:10BEB000E817F907A9F0AAA5BBA59D012F5F3F4F81
:10BEC0003BA72AA72C9121934AA55BA52EA53FA5A8
:10BED0004217530769F72CA53DA53BA72AA7E8CF32
:10BEE000C7010097C1F00FB6F8940F922AA93BA999
:10BEF000A901481B590B5BAB4AAB0F900FBE2AA997
:10BF00003BA98CA99DA92817390728F4C95BDF4FE5
:10BF1000E881F9811995C70102C080E090E0DF91C6
:10BF2000CF911F910F91FF90EF90DF90CF90BF9036
:10BF3000AF900895DC01ED91FC9120E030E0818923
:10BF400092890C94BE5DDC01ED91FC9121E030E022
:10BF5000818992890C94BE5DEF92FF920F931F939B
:10BF6000CF93DF938C01DC01ED91FC91C189D289E3
:10BF700040E050E060E070E0CE010E942B5D7C016B
:10BF8000FE01E35AFF4F0190F081E02D60E072E086
:10BF900080E090E01995C8010E94014620E030E061
:10BFA00040E050E060E070E0CE0140960E94705D9D
:10BFB00020E030E040E050E060E070E0CE018896A4
:10BFC0000E94705DCE01C8960E946D5261E08EADF8
:10BFD0009FAD0E94013D62E08EA19FA10E94013DA4
:10BFE00081E090E0EF2811F480E090E09195819558
:10BFF0009109DF91CF911F910F91FF90EF900895DC
:10C00000AF92BF92CF92DF92EF92FF920F931F9366
:10C01000CF93DF936C015A01FC01C189D2897A0167
:10C02000F3E0EF22FF24E114F10479F420EF30E093
:10C0300040ED50E060E071E0CE0188960E94705DB6
:10C04000892B99F08C899D891DC028E330E048E256
:10C0500050E060E470E0CE0140960E94705D892B54
:10C06000A1F521E0E216F10409F784E090E00E94D6
:10C07000F3458C01892B49F48C899D890E940146E6
:10C080008CA59DA50E94014620C0AA2480ECB82260
:10C0900088819981AA81BB81A114E0E8BE0611F4D0
:10C0A0008F7701C0806888839983AA83BB83F80156
:10C0B000D182C08213821282EA94EF2849F0C95BD0
:10C0C000DF4FE881F981199503C08FEF9FEF01C021
:10C0D000C801DF91CF911F910F91FF90EF90DF90FA
:10C0E000CF90BF90AF900895AF92BF92CF92DF9262
:10C0F000EF92FF920F931F93CF93DF931F921F92A4
:10C10000CDB7DEB78A01FA01C080D180E280F3802A
:10C110002C2DFC01A188B288FB01E150F140E333F2
:10C12000F10508F0BCC18827EE56FF4F8F4F0C94E5
:10C130003863F501E35BFF4F0190F081E02DC7010B
:10C14000B6015BC0F501E15BFF4FE4C0F501EF5ABA
:10C15000FF4F07C0F501ED5AFF4F17C0F501EB5A2D
:10C16000FF4F0190F081E02D8C2D0F900F90DF910B
:10C17000CF911F910F91FF90EF90DF90CF90BF90E4
:10C18000AF901994F501E95AFF4F0190F081E02D2D
:10C19000199590E07CC1F501E75AFF4FE2CFF50118
:10C1A000E55AFF4FF2CFC6FE12C0F50126A937A906
:10C1B00044A955A960A971A9C50188960E94705D1E
:10C1C000F501E95BFF4F0190F081E02D1995C7FE65
:10C1D0000BC0F501268D378D448D558D608D718D89
:10C1E000C50140960E94705DC701B6016F73F501ED
:10C1F000E35AFF4F0190F081E02D0F900F90DF91F7
:10C20000CF911F910F91FF90EF90DF90CF90BF9053
:10C21000AF901994F501E15AFF4F0190F081E02DA4
:10C220001995F8016083718382839383F50122A9B4
:10C2300033A9232B41F4DC01CB018064F801808316
:10C240009183A283B383F501828D938D892B09F0AD
:10C2500029C1F80180819181A281B3816CC0F5016F
:10C26000C086D186E286F3861DC1F5018085918561
:10C27000A285B3850EC1F501C486D586E686F7860C
:10C2800011C1F50184859585A685B78502C1F501A3
:10C29000C080D180E280F380222319F06894C6F830
:10C2A00070C0E894C6F86DC0F501808186FF09C0B2
:10C2B00081E090E0A0E0B0E0ECC0F501808187FD76
:10C2C000F7CFF8011082118212821382EBC0F501C0
:10C2D000C080D180E280F38055C0F501C080D1805C
:10C2E000E280F380222319F06894D3F84AC0E894DE
:10C2F000D3F847C0F501C080D180E280F3802223CB
:10C3000019F06894D4F83DC0E894D4F83AC0F50127
:10C31000E55BFF4F0190F081E02D1995F8016083F6
:10C32000718382839383BEC0F50180819181A28154
:10C33000B381CC2011F08068ADC08F77F501AAC021
:10C34000F501C080D180E280F380222319F0689447
:10C35000D2F817C0E894D2F814C0F5018081918119
:10C36000A281B38192FDA4CFACCFF501C080D18072
:10C37000E280F380222319F06894D5F802C0E89493
:10C38000D5F8F501E75BFF4F0190F081E02DC70183
:10C39000B6011995009709F087C0F501C082D182D6
:10C3A000E282F38281C0F50180819181A281B38113
:10C3B00095FD7ECF86CFF501EF59FF4FD2CEF50127
:10C3C000ED59FF4FE2CEF501268D378D448D558D09
:10C3D000B601C50140960E94705D009709F064C0E7
:10C3E000F501E95BFF4F0190F081E02D89839A838D
:10C3F000199589819A8158C0F501808D918D47C02A
:10C40000F50126A937A944A955A9B601C501889601
:10C410000F900F90DF91CF911F910F91FF90EF90B0
:10C42000DF90CF90BF90AF900C94705DF50180A924
:10C4300091A92DC00FB6F8940F92F501D58EC48E38
:10C4400020C0F501848D958D22C00FB6F8940F920F
:10C45000F501D78EC68E15C0F501868D978D17C054
:10C460000FB6F8940F92F501D5AAC4AA0AC0F50137
:10C4700084A995A90CC00FB6F8940F92F501D7AA1C
:10C48000C6AA0F900FBE0EC0F50186A997A9A0E01D
:10C49000B0E0F80180839183A283B38303C08FEF60
:10C4A0009FEF02C080E090E00F900F90DF91CF915E
:10C4B0001F910F91FF90EF90DF90CF90BF90AF90C2
:10C4C0000895DC01ED91FC910188F289E02D0FB611
:10C4D000F8940F9262A973A90F900FBE80E090E0CC
:10C4E0000895CF92DF92EF92FF920F931F93CF9315
:10C4F000DF938B017A016901DC01ED91FC91C18927
:10C50000D289AB0141705527B701CE01CE960E946A
:10C51000473DA801427055279601B701CE01869686
:10C520000E94473D0FB6F8940F928AA99BA931E06B
:10C5300020E0892B09F430E0832F922F4A8D5B8D08
:10C54000288D398D4217530708F482600F900FBE73
:10C5500080239123DF91CF911F910F91FF90EF9056
:10C56000DF90CF900895DB018F939F930E945E63CD
:10C57000BF91AF91A29F800D911DA39F900DB29F7F
:10C58000900D11240895991B79E004C0991F961706
:10C5900008F0961B881F7A95C9F780950895AA1B05
:10C5A000BB1B51E107C0AA1FBB1FA617B70710F09E
:10C5B000A61BB70B881F991F5A95A9F780959095D0
:10C5C000BC01CD01089597FB072E16F4009407D007
:10C5D00077FD09D00E94CF6207FC05D03EF490950C
:10C5E00081959F4F0895709561957F4F0895A1E2C1
:10C5F0001A2EAA1BBB1BFD010DC0AA1FBB1FEE1FDD
:10C60000FF1FA217B307E407F50720F0A21BB30B27
:10C61000E40BF50B661F771F881F991F1A9469F7A3
:10C6200060957095809590959B01AC01BD01CF01FF
:10C630000895052E97FB1EF400940E94306357FD69
:10C6400007D00E94F76207FC03D04EF40C943063CD
:10C6500050954095309521953F4F4F4F5F4F08952E
:10C6600090958095709561957F4F8F4F9F4F08955E
:10C67000EE0FFF1F881F8BBF0790F691E02D1994D6
:10C680000E944863332312F48A1B9B0B0C9459635A
:10C69000A29FB001B39FC001A39F700D811D112403
:10C6A000911DB29F700D811D1124911D08950E944E
:10C6B0004863B7FF0895821B930B08950E94486357
:10C6C000A59F900DB49F900DA49F800D911D1124E6
:10C6D0000895B7FF0C945E630E945E63821B930B08
:10C6E00008953F924F925F926F927F928F929F92A6
:10C6F000AF92BF92CF92DF92EF92FF920F931F9370
:10C70000CF93DF935C016B017A016115710519F01C
:10C71000FB0191838083E114F10429F0C7010297A2
:10C72000839708F0E5C0E5012196F5011081812F7E
:10C7300090E00E94D164892B11F05E01F4CF1D328C
:10C7400029F42196F501118101E007C01B3221F483
:10C75000E5012296F501118100E0E114F10409F1EF
:10C76000F0E1EF16F10429F43FC010E3E114F10405
:10C7700021F128E0E216F10401F154F4E2E0EE16B2
:10C78000F10421F5812C912CA12CB0E4BB2E3EC0EC
:10C79000FAE0EF16F10439F020E1E216F104B1F409
:10C7A00030C0103319F1FAE0EF2EF12CACEC8A2EE8
:10C7B000982CA82CACE0BA2E29C078E0E72EF12CFA
:10C7C000812C912CA12CE0E1BE2E20C060E070E015
:10C7D00080E090E897010F2C000C440B550B0E9451
:10C7E000F76249015A0112C0103359F488818F7DD4
:10C7F000883509F0BACF19812296026080E1E82ECF
:10C80000F12C812C912CA12C68E0B62E40E060E048
:10C8100070E0CB0127010F2C000C66087708FE01A1
:10C8200050ED352E310E29E0231570F42FEB210F3A
:10C830002A3118F439EC332E06C02FE9210F2A31A2
:10C8400018F529EA322E310E232D30E02E153F0542
:10C85000DCF447FD16C086169706A806B90670F0E8
:10C86000A30192010E94B362630D711D811D911D90
:10C8700061307105810520E8920710F04FEF01C08B
:10C8800041E021961081CBCF202F2170C114D1041B
:10C8900071F0442329F02197F601D183C08307C0AA
:10C8A00001FF19C02297F601D183C08314C047FF4E
:10C8B00012C0222329F060E070E080E090E804C01C
:10C8C0006FEF7FEF8FEF9FE722E230E03093A00918
:10C8D00020939F0909C0222381F09095809570953F
:10C8E00061957F4F8F4F9F4F462F372F282F12C0B4
:10C8F00040E030E020E090E00DC097FFF5CF82E20D
:10C9000090E09093A00980939F096FEF7FEF8FEFE6
:10C910009FE7EACF642F732F822FDF91CF911F9172
:10C920000F91FF90EF90DF90CF90BF90AF909F90CE
:10C930008F907F906F905F904F903F9008951F93DE
:10C94000FC0199278827BC01E89411911032E9F382
:10C95000193010F01E30C8F31B3251F01D3249F46B
:10C96000689406C00E94B265610F711D811D911D02
:10C97000119110531A30B0F33EF490958095709554
:10C9800061957F4F8F4F9F4F1F91089585FD0C94A8
:10C99000C765806291110C94C76581568A51D8F79A
:10C9A000089591110C94C765803219F08950855013
:10C9B000C8F708959111089581548A5108F4805E52
:10C9C000855A0895FB01DC0102C005900D9241508B
:10C9D0005040D8F70895FB01DC018D910590801936
:10C9E0000110D9F3990B0895FB01DC0105900D921C
:10C9F0000020E1F70895FC0105900020E9F78095FB
:10CA000090958E0F9F1F0895FC014150504030F0CB
:10CA100001900616D1F73197CF01089588279927FD
:10CA20000895FB01DC0104C08D910190801921F46F
:10CA300041505040C8F7881B990B0895FB01DC0159
:10CA400002C001900D9241505040D8F70895DC018A
:10CA500001C06D9341505040E0F70895FB01DC01A7
:10CA60008D9181341CF08B350CF4805E61916134C2
:10CA70001CF06B350CF4605E861B611189F3990B19
:10CA80000895FB01DC010D900020E9F7119701905A
:10CA90000D920020E1F70895FC018191861721F0A5
:10CAA0008823D9F7992708953197CF010895FB017D
:10CAB000DC018D91019080190110D9F3990B089533
:10CAC000FB01DC0101900D920020E1F70895FB01CC
:10CAD000DC014150504088F08D9181341CF08B3541
:10CAE0000CF4805E619161341CF06B350CF4605E77
:10CAF000861B611171F3990B0895881BFCCFFB0114
:10CB0000DC014150504030F08D910190801919F4B2
:10CB10000020B9F7881B990B0895FC0181E090E093
:10CB20000190061609F4CF010020D1F7019708956E
:10CB3000FB0151915523A9F0BF01DC014D9145172F
:10CB40004111E1F759F4CD010190002049F04D91D8
:10CB500040154111C9F3FB014111EFCF81E090E095
:10CB600001970895592F482F372F262F660F771FCB
:10CB7000881F991F660F771F881F991F620F731FE9
:10CB8000841F951F660F771F881F991F0895992787
:10CB900088270895DC01CB01FC01F999FECF06C07E
:10CBA000F2BDE1BDF89A319600B40D92415050406B
:10CBB000B8F70895DC01A40FB51F4150504048F06C
:10CBC000CB01840F951F2E910E94EB654150504080
:10CBD000D0F70895262FF999FECF92BD81BDF89A1E
:10CBE000019700B4021639F01FBA20BD0FB6F894B1
:0CCBF000FA9AF99A0FBE0895F894FFCF4E
:10CBFC0002020000B6033B00C103FF46064B0600D1
:10CC0C0000A407F1050000BD07F1050000E407F1E1
:10CC1C00050000B207F105000056065B0600006532
:10CC2C00066A06000075067A06000084068906006E
:10CC3C0000930698060000A806AC060000C506CABC
:10CC4C00060000E506EA060000F306F806000001FF
:10CC5C00070607000000000000000045068507914C
:10CC6C00079C07AA07B707C407D107DC0700000019
:10CC7C000055524F4D000000000001000000000064
:10CC8C0000000000CA3B983B233C2D3B3D3B0E3C37
:10CC9C00303B000001000200030000000000000017
:10CCAC0000000000FFFF1E003A00590077009600BC
:10CCBC00B400D300F20010012F014D016C01FFFFF5
:10CCCC001E003B005A0078009700B500D400F3001A
:10CCDC00110130014E016D0150460000F0F1FFFFD3
:10CCEC000100FFFF000000000000FFFF000000003B
:10CCFC0000000000657468300000000000030000B4
:10CD0C0000270300002E550000000000000000006A
:10CD1C000000000000000006000000000000000001
:10CD2C000000000000000000000000000000DC0516
:10CD3C00000000000000DC5B2B552E5C00000000A6
:10CD4C00000085560000756172743000000000050B
:10CD5C0000000000007903925E7460B25E9A5FA3DB
:10CD6C005F0060AC5F616271620000000000000057
:10CD7C0000000000000000000000000000000000A7
:10CD8C000000000000000000000000000000000097
:10CD9C000000000000000000000000000000000087
:10CDAC0000000000000000000000CD5AB358D0571E
:10CDBC00AE5AA257955763581558DA59C059275A85
:10CDCC00195AF457FD562E5705576E5A575A0000EC
:10CDDC000000FE5A00000000715B0F14070D2407C1
:10CDEC000000000E32070C4107064E0704550711D0
:10CDFC005A07076C070A74070D081108150819085B
:10CE0C001D082108250829082D083108350839087E
:10CE1C003D084108450849084D08510855080200CD
:10CE2C0000000000330041002A003D0028002D00C6
:10CE3C003300400033003300410033004100410017
:10CE4C004100410077000A0A53696D706C652048F7
:10CE5C00545450204461656D6F6E2072756E6E690E
:10CE6C006E67206F6E204E75742F4F532025730AFA
:10CE7C00006574683000436F6E6669677572652073
:10CE8C0025732E2E2E006661696C65642E2043611D
:10CE9C006E6E6F7420726567697374657220457469
:10CEAC006865726E6574206465766963652E0066CC
:10CEBC0061696C65642E2043616E6E6F7420636FC4
:10CECC006E666967757265206E6574776F726B2E0E
:10CEDC000A5573652065646974636F6E662E002550
:10CEEC00732072656164790A0052656769737465B1
:10CEFC00722055524F4D2066696C6520737973749E
:10CF0C00656D2E2E2E006661696C65642E004F4B8C
:10CF1C002E004572726F72202564206372656174F5
:10CF2C00696E6720736F636B65742E0A004C6973AE
:10CF3C0074656E696E672E2E2E00436F6E6E656380
:10CF4C007465642E2E2E00722B62004572726F7205
:10CF5C00202564206372656174696E672073747236
:10CF6C0065616D2E0A00446973636F6E6E65637440
:10CF7C006564006D61696E0069646C65006468636A
:10CF8C00706300446174653A20257320474D540D3D
:10CF9C000A004E6F74204D6F6469666965640042C7
:10CFAC006164205265717565737400556E6175749A
:10CFBC00686F72697A6564004E6F7420466F756E87
:10CFCC006400496E7465726E616C204572726F728A
:10CFDC00004E6F7420496D706C656D656E74656480
:10CFEC0000746578742F68746D6C00474554004864
:10CFFC0045414400504F535400485454502F312E47
:10D00C00300046726920466562202036203230316D
:10D01C00362032333A31333A3438004F6B004C619E
:10D02C0073742D4D6F6469666965643A20257320AD
:10D03C00474D540D0A002E74787400746578742F63
:10D04C00706C61696E002E67696600696D61676559
:10D05C002F676966002E6A706700696D6167652FBE
:10D06C006A706567002E706E6700696D6167652F69
:10D07C00706E67002E626D7000696D6167652F625E
:10D08C006D70002E706466006170706C6963617401
:10D09C00696F6E2F706466002E6A73006170706C1D
:10D0AC0069636174696F6E2F782D6A617661736341
:10D0BC0072697074002E6A6172006170706C6963C1
:10D0CC006174696F6E2F782D6A6176612D61726360
:10D0DC0068697665002E63737300746578742F63CA
:10D0EC007373002E786D6C00746578742F786D6C8A
:10D0FC00002E73766700696D6167652F7376672BF9
:10D10C00786D6C006163636570742D656E636F641C
:10D11C00696E6700617574686F72697A6174696FA2
:10D12C006E00636F6E74656E742D6C656E677468DB
:10D13C0000636F6E74656E742D7479706500636F27
:10D14C006F6B696500686F73740069662D6D6F6431
:10D15C0069666965642D73696E63650072656665E1
:10D16C0072657200757365722D6167656E7400551A
:10D17C00524F4D3A002F696E6465782E68746D6C51
:10D18C00002F696E6465782E68746D002F64656677
:10D19C0061756C742E68746D6C002F6465666175B6
:10D1AC006C742E68746D002F696E6465782E7368CC
:10D1BC00746D6C002F696E6465782E7868746D6C74
:10D1CC00002F696E6465782E617370002F6465663C
:10D1DC0061756C742E61737000474D540025732C6F
:10D1EC0020253032642025732025303464202530EE
:10D1FC0032643A253032643A25303264004A616E2A
:10D20C0000466562004D617200417072004D61799B
:10D21C00004A756E004A756C004175670053657065
:10D22C00004F6374004E6F76004465630053756E57
:10D23C00004D6F6E00547565005765640054687539
:10D24C000046726900536174004261736963200087
:10D25C006367692D62696E2F00746370736D0028AB
:10D26C006E756C6C2900352E322E342E30004F53D7
:0AD27C000065746865726E75740039
:00000001FF
